 vncviewer

 Timestamp is 477787d2 (Sun Dec 30 06:58:10 2007)

 Preferred load address is 00400000

 Start         Length     Name                   Class
 0001:00000000 00035c95H .text                   CODE
 0001:00035ca0 00001915H .text$x                 CODE
 0001:000375b5 00017b0bH .textbss                CODE
 0002:00000000 000046a0H .rdata                  DATA
 0002:000046a0 00000151H .rdata$r                DATA
 0002:000047f8 00001258H .xdata$x                DATA
 0002:00005a50 00000000H .edata                  DATA
 0003:00000000 00000104H .CRT$XCA                DATA
 0003:00000104 00000172H .CRT$XCU                DATA
 0003:00000278 00000104H .CRT$XCZ                DATA
 0003:0000037c 00000104H .CRT$XIA                DATA
 0003:00000480 0000010eH .CRT$XIC                DATA
 0003:00000590 00000104H .CRT$XIY                DATA
 0003:00000694 00000104H .CRT$XIZ                DATA
 0003:00000798 00000104H .CRT$XPA                DATA
 0003:0000089c 00000104H .CRT$XPX                DATA
 0003:000009a0 00000104H .CRT$XPZ                DATA
 0003:00000aa4 00000104H .CRT$XTA                DATA
 0003:00000ba8 00000104H .CRT$XTB                DATA
 0003:00000cac 00000104H .CRT$XTZ                DATA
 0003:00000db0 00004d62H .data                   DATA
 0003:00005b18 00001e68H .bss                    DATA
 0004:00000000 000000a0H .idata$2                DATA
 0004:000000a0 00000014H .idata$3                DATA
 0004:000000b4 000005dcH .idata$4                DATA
 0004:00000690 000005dcH .idata$5                DATA
 0004:00000c6c 000011f0H .idata$6                DATA
 0005:00000000 000007d3H .rsrc$01                DATA
 0005:000007e0 0000f9a9H .rsrc$02                DATA

  Address         Publics by Value              Rva+Base     Lib:Object

 0001:000007b0       ?ShowAboutBox@@YAXXZ       004017b0 f   AboutBox.obj
 0001:000008d0       ??0AuthDialog@@QAE@XZ      004018d0 f   AuthDialog.obj
 0001:00000900       ??_GAuthDialog@@UAEPAXI@Z  00401900 f i AuthDialog.obj
 0001:00000900       ??_EAuthDialog@@UAEPAXI@Z  00401900 f i AuthDialog.obj
 0001:00000950       ??1AuthDialog@@UAE@XZ      00401950 f   AuthDialog.obj
 0001:00000980       ?DoDialog@AuthDialog@@QAEHXZ 00401980 f   AuthDialog.obj
 0001:000009d0       ?DlgProc@AuthDialog@@SGHPAUHWND__@@IIJ@Z 004019d0 f   AuthDialog.obj
 0001:00000b60       ??0ClientConnection@@QAE@PAVVNCviewerApp@@@Z 00401b60 f   ClientConnection.obj
 0001:00000c90       ?run@omni_thread@@EAEXPAX@Z 00401c90 f i ClientConnection.obj
 0001:00000cb0       ??_EClientConnection@@UAEPAXI@Z 00401cb0 f i ClientConnection.obj
 0001:00000cb0       ??_GClientConnection@@UAEPAXI@Z 00401cb0 f i ClientConnection.obj
 0001:00000d00       ??0ClientConnection@@QAE@PAVVNCviewerApp@@I@Z 00401d00 f   ClientConnection.obj
 0001:00000f00       ??0ClientConnection@@QAE@PAVVNCviewerApp@@PADH@Z 00401f00 f   ClientConnection.obj
 0001:00001060       ?Init@ClientConnection@@AAEXPAVVNCviewerApp@@@Z 00402060 f   ClientConnection.obj
 0001:00001200       ?Run@ClientConnection@@QAEXXZ 00402200 f   ClientConnection.obj
 0001:000012b0       ?CreateDisplay@ClientConnection@@AAEXXZ 004022b0 f   ClientConnection.obj
 0001:00001930       ?Print@Log@@QAAXHPADZZ     00402930 f i ClientConnection.obj
 0001:00001980       ?GetConnectDetails@ClientConnection@@AAEXXZ 00402980 f   ClientConnection.obj
 0001:00001ae0       ??0QuietException@@QAE@ABV0@@Z 00402ae0 f i ClientConnection.obj
 0001:00001b20       ??0Exception@@QAE@ABV0@@Z  00402b20 f i ClientConnection.obj
 0001:00001b60       ??_GQuietException@@UAEPAXI@Z 00402b60 f i ClientConnection.obj
 0001:00001b60       ??_EQuietException@@UAEPAXI@Z 00402b60 f i ClientConnection.obj
 0001:00001bb0       ??_EException@@UAEPAXI@Z   00402bb0 f i ClientConnection.obj
 0001:00001bb0       ??_GException@@UAEPAXI@Z   00402bb0 f i ClientConnection.obj
 0001:00001c00       ?Connect@ClientConnection@@AAEXXZ 00402c00 f   ClientConnection.obj
 0001:00001d70       ??0WarningException@@QAE@ABV0@@Z 00402d70 f i ClientConnection.obj
 0001:00001dc0       ??_GWarningException@@UAEPAXI@Z 00402dc0 f i ClientConnection.obj
 0001:00001dc0       ??_EWarningException@@UAEPAXI@Z 00402dc0 f i ClientConnection.obj
 0001:00001e10       ?SetSocketOptions@ClientConnection@@AAEXXZ 00402e10 f   ClientConnection.obj
 0001:00001e80       ?NegotiateProtocolVersion@ClientConnection@@AAEXXZ 00402e80 f   ClientConnection.obj
 0001:00002080       ?Authenticate@ClientConnection@@AAEXXZ 00403080 f   ClientConnection.obj
 0001:00002770       ??0ErrorException@@QAE@ABV0@@Z 00403770 f i ClientConnection.obj
 0001:000027b0       ??_EErrorException@@UAEPAXI@Z 004037b0 f i ClientConnection.obj
 0001:000027b0       ??_GErrorException@@UAEPAXI@Z 004037b0 f i ClientConnection.obj
 0001:00002800       ?SendClientInit@ClientConnection@@AAEXXZ 00403800 f   ClientConnection.obj
 0001:00002840       ?ReadServerInit@ClientConnection@@AAEXXZ 00403840 f   ClientConnection.obj
 0001:00002b40       ?SizeWindow@ClientConnection@@AAEXXZ 00403b40 f   ClientConnection.obj
 0001:00002d80       ?CreateLocalFramebuffer@ClientConnection@@AAEXXZ 00403d80 f   ClientConnection.obj
 0001:00003030       ??0omni_mutex_lock@@QAE@AAVomni_mutex@@@Z 00404030 f i ClientConnection.obj
 0001:00003070       ??1omni_mutex_lock@@QAE@XZ 00404070 f i ClientConnection.obj
 0001:000030a0       ?FillSolidRect@ClientConnection@@AAEXPAUtagRECT@@K@Z 004040a0 f i ClientConnection.obj
 0001:00003100       ??0ObjectSelector@@QAE@PAUHDC__@@PAX@Z 00404100 f i ClientConnection.obj
 0001:00003150       ??1ObjectSelector@@QAE@XZ  00404150 f i ClientConnection.obj
 0001:00003190       ??0PaletteSelector@@QAE@PAUHDC__@@PAUHPALETTE__@@@Z 00404190 f i ClientConnection.obj
 0001:000031e0       ??1PaletteSelector@@QAE@XZ 004041e0 f i ClientConnection.obj
 0001:00003230       ??0TempDC@@QAE@PAUHWND__@@@Z 00404230 f i ClientConnection.obj
 0001:00003270       ??1TempDC@@QAE@XZ          00404270 f i ClientConnection.obj
 0001:000032a0       ??BTempDC@@QAEPAUHDC__@@XZ 004042a0 f i ClientConnection.obj
 0001:000032c0       ?SetupPixelFormat@ClientConnection@@AAEXXZ 004042c0 f   ClientConnection.obj
 0001:000034e0       ?SetFormatAndEncodings@ClientConnection@@AAEXXZ 004044e0 f   ClientConnection.obj
 0001:00003820       ?KillThread@ClientConnection@@QAEXXZ 00404820 f   ClientConnection.obj
 0001:000038a0       ??1ClientConnection@@UAE@XZ 004048a0 f   ClientConnection.obj
 0001:00003af0       ?ScrollScreen@ClientConnection@@AAE_NHH@Z 00404af0 f   ClientConnection.obj
 0001:00003cf0       ?WndProc@ClientConnection@@CGJPAUHWND__@@IIJ@Z 00404cf0 f   ClientConnection.obj
 0001:00005360       ?ProcessPointerEvent@ClientConnection@@AAEXHHKI@Z 00406360 f   ClientConnection.obj
 0001:00005700       ?SubProcessPointerEvent@ClientConnection@@AAEXHHK@Z 00406700 f i ClientConnection.obj
 0001:00005880       ?SendPointerEvent@ClientConnection@@AAEXHHH@Z 00406880 f i ClientConnection.obj
 0001:00005930       ?ProcessKeyEvent@ClientConnection@@AAEXHK@Z 00406930 f i ClientConnection.obj
 0001:00005c90       ?SendKeyEvent@ClientConnection@@AAEXK_N@Z 00406c90 f i ClientConnection.obj
 0001:00005d70       ?SendClientCutText@ClientConnection@@AAEXPADH@Z 00406d70 f   ClientConnection.obj
 0001:00005e20       ?DoBlit@ClientConnection@@AAEXXZ 00406e20 f i ClientConnection.obj
 0001:00006220       ?UpdateScrollbars@ClientConnection@@AAEXXZ 00407220 f i ClientConnection.obj
 0001:00006340       ?ShowConnInfo@ClientConnection@@AAEXXZ 00407340 f   ClientConnection.obj
 0001:00006420       ?run_undetached@ClientConnection@@EAEPAXPAX@Z 00407420 f   ClientConnection.obj
 0001:00006730       ?SendFullFramebufferUpdateRequest@ClientConnection@@AAEXXZ 00407730 f i ClientConnection.obj
 0001:00006780       ?SendFramebufferUpdateRequest@ClientConnection@@AAEXHHHH_N@Z 00407780 f i ClientConnection.obj
 0001:000068a0       ?SendAppropriateFramebufferUpdateRequest@ClientConnection@@AAEXXZ 004078a0 f   ClientConnection.obj
 0001:00006990       ?SendIncrementalFramebufferUpdateRequest@ClientConnection@@AAEXXZ 00407990 f i ClientConnection.obj
 0001:000069e0       ?ReadScreenUpdate@ClientConnection@@AAEXXZ 004079e0 f   ClientConnection.obj
 0001:00006e30       ?SetDormant@ClientConnection@@AAEX_N@Z 00407e30 f   ClientConnection.obj
 0001:00006ec0       ?ReadServerCutText@ClientConnection@@AAEXXZ 00407ec0 f   ClientConnection.obj
 0001:00006fb0       ?ReadBell@ClientConnection@@AAEXXZ 00407fb0 f   ClientConnection.obj
 0001:00007070       ?ReadExact@ClientConnection@@AAEXPADH@Z 00408070 f i ClientConnection.obj
 0001:000071f0       ?ReadString@ClientConnection@@AAEXPADH@Z 004081f0 f i ClientConnection.obj
 0001:00007250       ?WriteExact@ClientConnection@@AAEXPADH@Z 00408250 f i ClientConnection.obj
 0001:000073f0       ?CheckBufferSize@ClientConnection@@AAEXH@Z 004083f0 f i ClientConnection.obj
 0001:00007580       ?ProcessLocalClipboardChange@ClientConnection@@AAEXXZ 00408580 f   ClientConnectionClipboard.obj
 0001:000078a0       ?UpdateLocalClipboard@ClientConnection@@AAEXPADH@Z 004088a0 f   ClientConnectionClipboard.obj
 0001:00007b50       ?ReadCopyRect@ClientConnection@@AAEXPAUrfbFramebufferUpdateRectHeader@@@Z 00408b50 f   ClientConnectionCopyRect.obj
 0001:00007d80       ?ReadCoRRERect@ClientConnection@@AAEXPAUrfbFramebufferUpdateRectHeader@@@Z 00408d80 f   ClientConnectionCoRRE.obj
 0001:000086d0       ?FillSolidRect@ClientConnection@@AAEXHHHHK@Z 004096d0 f i ClientConnectionCoRRE.obj
 0001:00008770       ?ofnInit@@YAXXZ            00409770 f   ClientConnectionFile.obj
 0001:000087e0       ?SaveConnection@ClientConnection@@AAEXXZ 004097e0 f   ClientConnectionFile.obj
 0001:00008b00       ?LoadConnection@ClientConnection@@AAEHPAD@Z 00409b00 f   ClientConnectionFile.obj
 0001:00008cb0       ?InFullScreenMode@ClientConnection@@AAE_NXZ 00409cb0 f   ClientConnectionFullScreen.obj
 0001:00008ce0       ?SetFullScreenMode@ClientConnection@@AAEX_N@Z 00409ce0 f   ClientConnectionFullScreen.obj
 0001:00008d20       ?RealiseFullScreenMode@ClientConnection@@AAEXXZ 00409d20 f   ClientConnectionFullScreen.obj
 0001:00008f70       ?BumpScroll@ClientConnection@@AAE_NHH@Z 00409f70 f   ClientConnectionFullScreen.obj
 0001:00009110       ?ReadHextileRect@ClientConnection@@AAEXPAUrfbFramebufferUpdateRectHeader@@@Z 0040a110 f   ClientConnectionHextile.obj
 0001:00009210       ?HandleHextileEncoding8@ClientConnection@@AAEXHHHH@Z 0040a210 f   ClientConnectionHextile.obj
 0001:00009b60       ?HandleHextileEncoding16@ClientConnection@@AAEXHHHH@Z 0040ab60 f   ClientConnectionHextile.obj
 0001:0000a4b0       ?HandleHextileEncoding32@ClientConnection@@AAEXHHHH@Z 0040b4b0 f   ClientConnectionHextile.obj
 0001:0000ae10       ?ReadRawRect@ClientConnection@@AAEXPAUrfbFramebufferUpdateRectHeader@@@Z 0040be10 f   ClientConnectionRaw.obj
 0001:0000b5d0       ?ReadRRERect@ClientConnection@@AAEXPAUrfbFramebufferUpdateRectHeader@@@Z 0040c5d0 f   ClientConnectionRRE.obj
 0001:0000bff0       _deskey                    0040cff0 f   d3des.obj
 0001:0000c420       _cpkey                     0040d420 f   d3des.obj
 0001:0000c480       _usekey                    0040d480 f   d3des.obj
 0001:0000c4e0       _des                       0040d4e0 f   d3des.obj
 0001:0000cd10       ??0Daemon@@QAE@H@Z         0040dd10 f   Daemon.obj
 0001:0000d030       ??_EDaemon@@UAEPAXI@Z      0040e030 f i Daemon.obj
 0001:0000d030       ??_GDaemon@@UAEPAXI@Z      0040e030 f i Daemon.obj
 0001:0000d080       ?AddTrayIcon@Daemon@@IAEXXZ 0040e080 f   Daemon.obj
 0001:0000d0c0       ?CheckTrayIcon@Daemon@@IAEXXZ 0040e0c0 f   Daemon.obj
 0001:0000d130       ?RemoveTrayIcon@Daemon@@IAEXXZ 0040e130 f   Daemon.obj
 0001:0000d170       ?SendTrayMsg@Daemon@@IAE_NK@Z 0040e170 f   Daemon.obj
 0001:0000d250       ?WndProc@Daemon@@SGJPAUHWND__@@IIJ@Z 0040e250 f   Daemon.obj
 0001:0000d600       ??1Daemon@@UAE@XZ          0040e600 f   Daemon.obj
 0001:0000d680       ??0Exception@@QAE@PBD@Z    0040e680 f   Exception.obj
 0001:0000d720       ??1Exception@@UAE@XZ       0040e720 f   Exception.obj
 0001:0000d760       ?Report@Exception@@UAEXXZ  0040e760 f   Exception.obj
 0001:0000d7b0       ??0QuietException@@QAE@PBD@Z 0040e7b0 f   Exception.obj
 0001:0000d7f0       ??1QuietException@@UAE@XZ  0040e7f0 f   Exception.obj
 0001:0000d820       ?Report@QuietException@@UAEXXZ 0040e820 f   Exception.obj
 0001:0000d870       ??0WarningException@@QAE@PBD_N@Z 0040e870 f   Exception.obj
 0001:0000d8c0       ??1WarningException@@UAE@XZ 0040e8c0 f   Exception.obj
 0001:0000d8f0       ?Report@WarningException@@UAEXXZ 0040e8f0 f   Exception.obj
 0001:0000d960       ??0ErrorException@@QAE@PBD@Z 0040e960 f   Exception.obj
 0001:0000d9a0       ??1ErrorException@@UAE@XZ  0040e9a0 f   Exception.obj
 0001:0000d9d0       ?Report@ErrorException@@UAEXXZ 0040e9d0 f   Exception.obj
 0001:0000da80       ??0Flasher@@QAE@H@Z        0040ea80 f   Flasher.obj
 0001:0000de00       ??_GFlasher@@UAEPAXI@Z     0040ee00 f i Flasher.obj
 0001:0000de00       ??_EFlasher@@UAEPAXI@Z     0040ee00 f i Flasher.obj
 0001:0000de50       ?KillScreenSaverFunc@@YGHPAUHWND__@@J@Z 0040ee50 f   Flasher.obj
 0001:0000de80       ?WndProc@Flasher@@SGJPAUHWND__@@IIJ@Z 0040ee80 f   Flasher.obj
 0001:0000e4a0       ?scalechar@@YAHD@Z         0040f4a0 f i Flasher.obj
 0001:0000e4e0       ?CloseScreenSaver@Flasher@@SAXXZ 0040f4e0 f   Flasher.obj
 0001:0000e5f0       ??1Flasher@@UAE@XZ         0040f5f0 f   Flasher.obj
 0001:0000e6a0       ??0KeyMap@@QAE@XZ          0040f6a0 f   KeyMap.obj
 0001:0000e6c0       ?PCtoX@KeyMap@@QAE?AUKeyActionSpec@@IK@Z 0040f6c0 f   KeyMap.obj
 0001:0000ec80       ??0Log@@QAE@HHPAD_N@Z      0040fc80 f   Log.obj
 0001:0000ed00       ??_GLog@@UAEPAXI@Z         0040fd00 f i Log.obj
 0001:0000ed00       ??_ELog@@UAEPAXI@Z         0040fd00 f i Log.obj
 0001:0000ed50       ?SetMode@Log@@QAEXH@Z      0040fd50 f   Log.obj
 0001:0000edf0       ?SetLevel@Log@@QAEXH@Z     0040fdf0 f   Log.obj
 0001:0000ee20       ?SetFile@Log@@QAEXPAD_N@Z  0040fe20 f   Log.obj
 0001:0000eef0       ?CloseFile@Log@@AAEXXZ     0040fef0 f   Log.obj
 0001:0000ef30       ?ReallyPrint@Log@@AAEXPAD0@Z 0040ff30 f   Log.obj
 0001:0000f030       ??1Log@@UAE@XZ             00410030 f   Log.obj
 0001:0000f100       ??0MRU@@QAE@PADI@Z         00410100 f   MRU.obj
 0001:0000f1a0       ??_EMRU@@UAEPAXI@Z         004101a0 f i MRU.obj
 0001:0000f1a0       ??_GMRU@@UAEPAXI@Z         004101a0 f i MRU.obj
 0001:0000f1f0       ?AddItem@MRU@@QAEXPAD@Z    004101f0 f   MRU.obj
 0001:0000f440       ?NumItems@MRU@@QAEHXZ      00410440 f   MRU.obj
 0001:0000f480       ?GetItem@MRU@@QAEHHPADH@Z  00410480 f   MRU.obj
 0001:0000f530       ?RemoveItem@MRU@@QAEXPAD@Z 00410530 f   MRU.obj
 0001:0000f5f0       ?RemoveItem@MRU@@QAEXH@Z   004105f0 f   MRU.obj
 0001:0000f6b0       ?ReadIndex@MRU@@AAEXXZ     004106b0 f   MRU.obj
 0001:0000f720       ?WriteIndex@MRU@@IAEXXZ    00410720 f   MRU.obj
 0001:0000f790       ?Tidy@MRU@@AAEXXZ          00410790 f   MRU.obj
 0001:0000fbd0       ??1MRU@@UAE@XZ             00410bd0 f   MRU.obj
 0001:0000fc70       ??0SessionDialog@@QAE@PAVVNCOptions@@@Z 00410c70 f   SessionDialog.obj
 0001:0000fd30       ??_ESessionDialog@@UAEPAXI@Z 00410d30 f i SessionDialog.obj
 0001:0000fd30       ??_GSessionDialog@@UAEPAXI@Z 00410d30 f i SessionDialog.obj
 0001:0000fd80       ??1SessionDialog@@UAE@XZ   00410d80 f   SessionDialog.obj
 0001:0000fde0       ?DoDialog@SessionDialog@@QAEHXZ 00410de0 f   SessionDialog.obj
 0001:0000fe30       ?SessDlgProc@SessionDialog@@CGHPAUHWND__@@IIJ@Z 00410e30 f   SessionDialog.obj
 0001:00010110       _vncEncryptBytes           00411110 f   vncauth.obj
 0001:000101d0       _vncEncryptPasswd          004111d0 f   vncauth.obj
 0001:00010270       _vncDecryptPasswd          00411270 f   vncauth.obj
 0001:00010360       ??0VNCOptions@@QAE@XZ      00411360 f   VNCOptions.obj
 0001:00010540       ??_EVNCOptions@@UAEPAXI@Z  00411540 f i VNCOptions.obj
 0001:00010540       ??_GVNCOptions@@UAEPAXI@Z  00411540 f i VNCOptions.obj
 0001:00010590       ??4VNCOptions@@QAEAAV0@AAV0@@Z 00411590 f   VNCOptions.obj
 0001:00010890       ??1VNCOptions@@UAE@XZ      00411890 f   VNCOptions.obj
 0001:000108c0       ?gcd@@YAHHH@Z              004118c0 f   VNCOptions.obj
 0001:00010920       ?FixScaling@VNCOptions@@AAEXXZ 00411920 f   VNCOptions.obj
 0001:00010a00       ?SetFromCommandLine@VNCOptions@@QAEXPAD@Z 00411a00 f   VNCOptions.obj
 0001:00011650       ?SwitchMatch@@YA_NPBD0@Z   00412650 f i VNCOptions.obj
 0001:000116f0       ?saveInt@@YAXPADH0@Z       004126f0 f   VNCOptions.obj
 0001:00011740       ?readInt@@YAHPADH0@Z       00412740 f   VNCOptions.obj
 0001:00011770       ?Save@VNCOptions@@QAEXPAD@Z 00412770 f   VNCOptions.obj
 0001:00011a10       ?Load@VNCOptions@@QAEXPAD@Z 00412a10 f   VNCOptions.obj
 0001:00011db0       ?Register@VNCOptions@@AAEXXZ 00412db0 f   VNCOptions.obj
 0001:00012030       ?ShowUsage@VNCOptions@@AAEXPAD@Z 00413030 f   VNCOptions.obj
 0001:000120b0       ?DoDialog@VNCOptions@@QAEH_N@Z 004130b0 f   VNCOptions.obj
 0001:00012110       ?OptDlgProc@VNCOptions@@SGHPAUHWND__@@IIJ@Z 00413110 f   VNCOptions.obj
 0001:00012a00       _WinMain@16                00413a00 f   vncviewer.obj
 0001:00012b90       ?CentreWindow@@YAXPAUHWND__@@@Z 00413b90 f   vncviewer.obj
 0001:00012c90       ?ParseDisplay@@YA_NPAD0HPAH@Z 00413c90 f   vncviewer.obj
 0001:00012dc0       ??0VNCviewerApp@@QAE@PAUHINSTANCE__@@PAD@Z 00413dc0 f   VNCviewerApp.obj
 0001:00012fa0       ?RegisterConnection@VNCviewerApp@@QAEXPAVClientConnection@@@Z 00413fa0 f   VNCviewerApp.obj
 0001:000130d0       ?DeregisterConnection@VNCviewerApp@@QAEXPAVClientConnection@@@Z 004140d0 f   VNCviewerApp.obj
 0001:00013270       ??1VNCviewerApp@@QAE@XZ    00414270 f   VNCviewerApp.obj
 0001:00013310       ??0VNCviewerApp32@@QAE@PAUHINSTANCE__@@PAD@Z 00414310 f   VNCviewerApp32.obj
 0001:000135d0       ?NewConnection@VNCviewerApp32@@UAEXXZ 004145d0 f   VNCviewerApp32.obj
 0001:000136e0       ?NewConnection@VNCviewerApp32@@UAEXPADH@Z 004146e0 f   VNCviewerApp32.obj
 0001:000137f0       ?NewConnection@VNCviewerApp32@@UAEXI@Z 004147f0 f   VNCviewerApp32.obj
 0001:00013900       ?RegisterSounds@VNCviewerApp32@@AAEXXZ 00414900 f   VNCviewerApp32.obj
 0001:00013b40       ??1VNCviewerApp32@@QAE@XZ  00414b40 f   VNCviewerApp32.obj
 0001:00013c80       _PlaySoundA@12             00414c80 f   winmm:WINMM.dll
 0001:00013c90       ??0omni_mutex@@QAE@XZ      00414c90 f   omnithread:nt.obj
 0001:00013ca8       ??1omni_mutex@@QAE@XZ      00414ca8 f   omnithread:nt.obj
 0001:00013cbd       ?lock@omni_mutex@@QAEXXZ   00414cbd f   omnithread:nt.obj
 0001:00013cd2       ?unlock@omni_mutex@@QAEXXZ 00414cd2 f   omnithread:nt.obj
 0001:00013d43       ??0omni_condition@@QAE@PAVomni_mutex@@@Z 00414d43 f   omnithread:nt.obj
 0001:00013d7c       ??1omni_condition@@QAE@XZ  00414d7c f   omnithread:nt.obj
 0001:00013d94       ?wait@omni_condition@@QAEXXZ 00414d94 f   omnithread:nt.obj
 0001:00013eb2       ?timedwait@omni_condition@@QAEHKK@Z 00414eb2 f   omnithread:nt.obj
 0001:00014138       ?signal@omni_condition@@QAEXXZ 00415138 f   omnithread:nt.obj
 0001:00014210       ?broadcast@omni_condition@@QAEXXZ 00415210 f   omnithread:nt.obj
 0001:000142d4       ??0omni_semaphore@@QAE@I@Z 004152d4 f   omnithread:nt.obj
 0001:00014328       ??1omni_semaphore@@QAE@XZ  00415328 f   omnithread:nt.obj
 0001:00014367       ?wait@omni_semaphore@@QAEXXZ 00415367 f   omnithread:nt.obj
 0001:000143a8       ?trywait@omni_semaphore@@QAEHXZ 004153a8 f   omnithread:nt.obj
 0001:00014404       ?post@omni_semaphore@@QAEXXZ 00415404 f   omnithread:nt.obj
 0001:00014447       ??0init_t@omni_thread@@QAE@XZ 00415447 f   omnithread:nt.obj
 0001:0001462a       _omni_thread_wrapper@4     0041562a f   omnithread:nt.obj
 0001:00014708       ??0omni_thread@@QAE@P6AXPAX@Z0W4priority_t@0@@Z 00415708 f   omnithread:nt.obj
 0001:0001477e       ??0omni_thread@@QAE@P6APAXPAX@Z0W4priority_t@0@@Z 0041577e f   omnithread:nt.obj
 0001:000147f4       ??0omni_thread@@IAE@PAXW4priority_t@0@@Z 004157f4 f   omnithread:nt.obj
 0001:0001486b       ?common_constructor@omni_thread@@AAEXPAXW4priority_t@1@H@Z 0041586b f   omnithread:nt.obj
 0001:0001493a       ??1omni_thread@@MAE@XZ     0041593a f   omnithread:nt.obj
 0001:000149f7       ?start@omni_thread@@QAEXXZ 004159f7 f   omnithread:nt.obj
 0001:00014b32       ?start_undetached@omni_thread@@IAEXXZ 00415b32 f   omnithread:nt.obj
 0001:00014b77       ?join@omni_thread@@QAEXPAPAX@Z 00415b77 f   omnithread:nt.obj
 0001:00014c78       ?set_priority@omni_thread@@QAEXW4priority_t@1@@Z 00415c78 f   omnithread:nt.obj
 0001:00014d31       ?create@omni_thread@@SAPAV1@P6AXPAX@Z0W4priority_t@1@@Z 00415d31 f   omnithread:nt.obj
 0001:00014db2       ?create@omni_thread@@SAPAV1@P6APAXPAX@Z0W4priority_t@1@@Z 00415db2 f   omnithread:nt.obj
 0001:00014e33       ?exit@omni_thread@@SAXPAX@Z 00415e33 f   omnithread:nt.obj
 0001:00014eb3       ?self@omni_thread@@SAPAV1@XZ 00415eb3 f   omnithread:nt.obj
 0001:00014ecd       ?yield@omni_thread@@SAXXZ  00415ecd f   omnithread:nt.obj
 0001:00014eda       ?sleep@omni_thread@@SAXKK@Z 00415eda f   omnithread:nt.obj
 0001:00014f6e       ?get_time@omni_thread@@SAXPAK0KK@Z 00415f6e f   omnithread:nt.obj
 0001:00014fc2       ?nt_priority@omni_thread@@CAHW4priority_t@1@@Z 00415fc2 f   omnithread:nt.obj
 0001:000150f0       ??0_internal_omni_thread_helper@@QAE@XZ 004160f0 f i omnithread:nt.obj
 0001:000151d0       ??0_internal_omni_thread_dummy@@QAE@XZ 004161d0 f i omnithread:nt.obj
 0001:00015200       ??_E_internal_omni_thread_dummy@@UAEPAXI@Z 00416200 f i omnithread:nt.obj
 0001:00015200       ??_G_internal_omni_thread_dummy@@UAEPAXI@Z 00416200 f i omnithread:nt.obj
 0001:00015230       ??1_internal_omni_thread_dummy@@UAE@XZ 00416230 f i omnithread:nt.obj
 0001:00015250       ??1_internal_omni_thread_helper@@QAE@XZ 00416250 f i omnithread:nt.obj
 0001:000152a0       ??B_internal_omni_thread_helper@@QAEPAVomni_thread@@XZ 004162a0 f i omnithread:nt.obj
 0001:000152c0       ??C_internal_omni_thread_helper@@QAEPAVomni_thread@@XZ 004162c0 f i omnithread:nt.obj
 0001:000152e0       ??0omni_thread_fatal@@QAE@H@Z 004162e0 f i omnithread:nt.obj
 0001:00015300       ?run_undetached@omni_thread@@EAEPAXPAX@Z 00416300 f i omnithread:nt.obj
 0001:00015310       ??_Eomni_thread@@MAEPAXI@Z 00416310 f i omnithread:nt.obj
 0001:00015310       ??_Gomni_thread@@MAEPAXI@Z 00416310 f i omnithread:nt.obj
 0001:0001533e       _GetLastError@0            0041633e f   kernel32:KERNEL32.dll
 0001:00015344       _Sleep@4                   00416344 f   kernel32:KERNEL32.dll
 0001:0001534a       _Beep@8                    0041634a f   kernel32:KERNEL32.dll
 0001:00015350       _LocalFree@4               00416350 f   kernel32:KERNEL32.dll
 0001:00015356       _FormatMessageA@28         00416356 f   kernel32:KERNEL32.dll
 0001:0001535c       _GlobalUnlock@4            0041635c f   kernel32:KERNEL32.dll
 0001:00015362       _GlobalLock@4              00416362 f   kernel32:KERNEL32.dll
 0001:00015368       _GlobalAlloc@8             00416368 f   kernel32:KERNEL32.dll
 0001:0001536e       _WritePrivateProfileStringA@16 0041636e f   kernel32:KERNEL32.dll
 0001:00015374       _GetPrivateProfileIntA@16  00416374 f   kernel32:KERNEL32.dll
 0001:0001537a       _GetPrivateProfileStringA@24 0041637a f   kernel32:KERNEL32.dll
 0001:00015380       _GetVersionExA@4           00416380 f   kernel32:KERNEL32.dll
 0001:00015386       _AllocConsole@0            00416386 f   kernel32:KERNEL32.dll
 0001:0001538c       _SetEndOfFile@4            0041638c f   kernel32:KERNEL32.dll
 0001:00015392       _SetFilePointer@16         00416392 f   kernel32:KERNEL32.dll
 0001:00015398       _CreateFileA@28            00416398 f   kernel32:KERNEL32.dll
 0001:0001539e       _CloseHandle@4             0041639e f   kernel32:KERNEL32.dll
 0001:000153a4       _WriteFile@20              004163a4 f   kernel32:KERNEL32.dll
 0001:000153aa       _WriteConsoleA@20          004163aa f   kernel32:KERNEL32.dll
 0001:000153b0       _GetStdHandle@4            004163b0 f   kernel32:KERNEL32.dll
 0001:000153b6       _OutputDebugStringA@4      004163b6 f   kernel32:KERNEL32.dll
 0001:000153bc       _GetModuleFileNameA@12     004163bc f   kernel32:KERNEL32.dll
 0001:000153c2       _InitializeCriticalSection@4 004163c2 f   kernel32:KERNEL32.dll
 0001:000153c8       _DeleteCriticalSection@4   004163c8 f   kernel32:KERNEL32.dll
 0001:000153ce       _EnterCriticalSection@4    004163ce f   kernel32:KERNEL32.dll
 0001:000153d4       _LeaveCriticalSection@4    004163d4 f   kernel32:KERNEL32.dll
 0001:000153da       _WaitForSingleObject@8     004163da f   kernel32:KERNEL32.dll
 0001:000153e0       _ReleaseSemaphore@12       004163e0 f   kernel32:KERNEL32.dll
 0001:000153e6       _CreateSemaphoreA@16       004163e6 f   kernel32:KERNEL32.dll
 0001:000153ec       _SetThreadPriority@8       004163ec f   kernel32:KERNEL32.dll
 0001:000153f2       _TlsSetValue@8             004163f2 f   kernel32:KERNEL32.dll
 0001:000153f8       _GetCurrentThreadId@0      004163f8 f   kernel32:KERNEL32.dll
 0001:000153fe       _DuplicateHandle@28        004163fe f   kernel32:KERNEL32.dll
 0001:00015404       _GetCurrentThread@0        00416404 f   kernel32:KERNEL32.dll
 0001:0001540a       _GetCurrentProcess@0       0041640a f   kernel32:KERNEL32.dll
 0001:00015410       _TlsAlloc@0                00416410 f   kernel32:KERNEL32.dll
 0001:00015416       _ResumeThread@4            00416416 f   kernel32:KERNEL32.dll
 0001:0001541c       _TlsGetValue@4             0041641c f   kernel32:KERNEL32.dll
 0001:00015422       _GetSystemTime@4           00416422 f   kernel32:KERNEL32.dll
 0001:00015428       _DialogBoxParamA@20        00416428 f   user32:USER32.dll
 0001:0001542e       _EndDialog@8               0041642e f   user32:USER32.dll
 0001:00015434       _GetDlgItemTextA@16        00416434 f   user32:USER32.dll
 0001:0001543a       _SetDlgItemTextA@12        0041643a f   user32:USER32.dll
 0001:00015440       _SetWindowLongA@12         00416440 f   user32:USER32.dll
 0001:00015446       _GetWindowLongA@8          00416446 f   user32:USER32.dll
 0001:0001544c       _SetClipboardViewer@4      0041644c f   user32:USER32.dll
 0001:00015452       _DrawMenuBar@4             00416452 f   user32:USER32.dll
 0001:00015458       _AppendMenuA@16            00416458 f   user32:USER32.dll
 0001:0001545e       _GetSystemMenu@8           0041645e f   user32:USER32.dll
 0001:00015464       _ShowWindow@8              00416464 f   user32:USER32.dll
 0001:0001546a       _CreateWindowExA@48        0041646a f   user32:USER32.dll
 0001:00015470       _RegisterClassA@4          00416470 f   user32:USER32.dll
 0001:00015476       _LoadCursorA@8             00416476 f   user32:USER32.dll
 0001:0001547c       _LoadIconA@8               0041647c f   user32:USER32.dll
 0001:00015482       _MessageBoxA@16            00416482 f   user32:USER32.dll
 0001:00015488       _SetWindowTextA@8          00416488 f   user32:USER32.dll
 0001:0001548e       _SetForegroundWindow@4     0041648e f   user32:USER32.dll
 0001:00015494       _SetWindowPos@28           00416494 f   user32:USER32.dll
 0001:0001549a       _AdjustWindowRectEx@16     0041649a f   user32:USER32.dll
 0001:000154a0       _SetRect@20                004164a0 f   user32:USER32.dll
 0001:000154a6       _SystemParametersInfoA@16  004164a6 f   user32:USER32.dll
 0001:000154ac       _InvalidateRect@12         004164ac f   user32:USER32.dll
 0001:000154b2       _DrawTextA@20              004164b2 f   user32:USER32.dll
 0001:000154b8       _GetDC@4                   004164b8 f   user32:USER32.dll
 0001:000154be       _ReleaseDC@8               004164be f   user32:USER32.dll
 0001:000154c4       _DestroyWindow@4           004164c4 f   user32:USER32.dll
 0001:000154ca       _UpdateWindow@4            004164ca f   user32:USER32.dll
 0001:000154d0       _ScrollWindowEx@32         004164d0 f   user32:USER32.dll
 0001:000154d6       _GetClientRect@8           004164d6 f   user32:USER32.dll
 0001:000154dc       _DefWindowProcA@16         004164dc f   user32:USER32.dll
 0001:000154e2       _SendMessageA@16           004164e2 f   user32:USER32.dll
 0001:000154e8       _PostQuitMessage@4         004164e8 f   user32:USER32.dll
 0001:000154ee       _SetCursor@4               004164ee f   user32:USER32.dll
 0001:000154f4       _ShowScrollBar@12          004164f4 f   user32:USER32.dll
 0001:000154fa       _GetWindowRect@8           004164fa f   user32:USER32.dll
 0001:00015500       _ChangeClipboardChain@8    00416500 f   user32:USER32.dll
 0001:00015506       _GetWindow@8               00416506 f   user32:USER32.dll
 0001:0001550c       _GetForegroundWindow@0     0041650c f   user32:USER32.dll
 0001:00015512       _GetFocus@0                00416512 f   user32:USER32.dll
 0001:00015518       _KillTimer@8               00416518 f   user32:USER32.dll
 0001:0001551e       _PostMessageA@16           0041651e f   user32:USER32.dll
 0001:00015524       _SetTimer@16               00416524 f   user32:USER32.dll
 0001:0001552a       _GetKeyNameTextA@12        0041652a f   user32:USER32.dll
 0001:00015530       _EndPaint@8                00416530 f   user32:USER32.dll
 0001:00015536       _BeginPaint@8              00416536 f   user32:USER32.dll
 0001:0001553c       _SetScrollInfo@16          0041653c f   user32:USER32.dll
 0001:00015542       _GetKeyboardLayoutNameA@4  00416542 f   user32:USER32.dll
 0001:00015548       _IsIconic@4                00416548 f   user32:USER32.dll
 0001:0001554e       _CloseClipboard@0          0041654e f   user32:USER32.dll
 0001:00015554       _GetClipboardData@4        00416554 f   user32:USER32.dll
 0001:0001555a       _OpenClipboard@4           0041655a f   user32:USER32.dll
 0001:00015560       _GetClipboardOwner@0       00416560 f   user32:USER32.dll
 0001:00015566       _SetClipboardData@8        00416566 f   user32:USER32.dll
 0001:0001556c       _EmptyClipboard@0          0041656c f   user32:USER32.dll
 0001:00015572       _CheckMenuItem@12          00416572 f   user32:USER32.dll
 0001:00015578       _GetSystemMetrics@4        00416578 f   user32:USER32.dll
 0001:0001557e       _SetCursorPos@8            0041657e f   user32:USER32.dll
 0001:00015584       _GetCursorPos@4            00416584 f   user32:USER32.dll
 0001:0001558a       _LoadMenuA@8               0041658a f   user32:USER32.dll
 0001:00015590       _RegisterClassExA@4        00416590 f   user32:USER32.dll
 0001:00015596       _LoadStringA@16            00416596 f   user32:USER32.dll
 0001:0001559c       _TrackPopupMenu@28         0041659c f   user32:USER32.dll
 0001:000155a2       _SetMenuDefaultItem@12     004165a2 f   user32:USER32.dll
 0001:000155a8       _GetMenuItemID@8           004165a8 f   user32:USER32.dll
 0001:000155ae       _GetSubMenu@8              004165ae f   user32:USER32.dll
 0001:000155b4       _DestroyMenu@4             004165b4 f   user32:USER32.dll
 0001:000155ba       _CloseDesktop@4            004165ba f   user32:USER32.dll
 0001:000155c0       _EnumDesktopWindows@12     004165c0 f   user32:USER32.dll
 0001:000155c6       _OpenDesktopA@16           004165c6 f   user32:USER32.dll
 0001:000155cc       _FindWindowA@8             004165cc f   user32:USER32.dll
 0001:000155d2       _GetKeyState@4             004165d2 f   user32:USER32.dll
 0001:000155d8       _ToAscii@20                004165d8 f   user32:USER32.dll
 0001:000155de       _GetKeyboardState@4        004165de f   user32:USER32.dll
 0001:000155e4       _GetDlgItem@8              004165e4 f   user32:USER32.dll
 0001:000155ea       _GetDlgItemInt@16          004165ea f   user32:USER32.dll
 0001:000155f0       _SetDlgItemInt@16          004165f0 f   user32:USER32.dll
 0001:000155f6       _EnableWindow@8            004165f6 f   user32:USER32.dll
 0001:000155fc       _DispatchMessageA@4        004165fc f   user32:USER32.dll
 0001:00015602       _GetMessageA@16            00416602 f   user32:USER32.dll
 0001:00015608       _LoadKeyboardLayoutA@8     00416608 f   user32:USER32.dll
 0001:0001560e       _CreatePalette@4           0041660e f   gdi32:GDI32.dll
 0001:00015614       _GetDeviceCaps@8           00416614 f   gdi32:GDI32.dll
 0001:0001561a       _CreateCompatibleDC@4      0041661a f   gdi32:GDI32.dll
 0001:00015620       _GetStockObject@4          00416620 f   gdi32:GDI32.dll
 0001:00015626       _SetTextColor@8            00416626 f   gdi32:GDI32.dll
 0001:0001562c       _SetBkColor@8              0041662c f   gdi32:GDI32.dll
 0001:00015632       _CreateCompatibleBitmap@12 00416632 f   gdi32:GDI32.dll
 0001:00015638       _ExtTextOutA@32            00416638 f   gdi32:GDI32.dll
 0001:0001563e       _SelectObject@8            0041663e f   gdi32:GDI32.dll
 0001:00015644       _RealizePalette@4          00416644 f   gdi32:GDI32.dll
 0001:0001564a       _SelectPalette@12          0041664a f   gdi32:GDI32.dll
 0001:00015650       _DeleteObject@4            00416650 f   gdi32:GDI32.dll
 0001:00015656       _DeleteDC@4                00416656 f   gdi32:GDI32.dll
 0001:0001565c       _UpdateColors@4            0041665c f   gdi32:GDI32.dll
 0001:00015662       _BitBlt@36                 00416662 f   gdi32:GDI32.dll
 0001:00015668       _StretchBlt@44             00416668 f   gdi32:GDI32.dll
 0001:0001566e       _SetBrushOrgEx@16          0041666e f   gdi32:GDI32.dll
 0001:00015674       _SetStretchBltMode@8       00416674 f   gdi32:GDI32.dll
 0001:0001567a       _SetPixelV@16              0041667a f   gdi32:GDI32.dll
 0001:00015680       _CreateFontIndirectA@4     00416680 f   gdi32:GDI32.dll
 0001:00015686       _GdiFlush@0                00416686 f   gdi32:GDI32.dll
 0001:0001568c       _SetBkMode@8               0041668c f   gdi32:GDI32.dll
 0001:00015692       _Rectangle@20              00416692 f   gdi32:GDI32.dll
 0001:00015698       _GetClipBox@8              00416698 f   gdi32:GDI32.dll
 0001:0001569e       _CommDlgExtendedError@0    0041669e f   comdlg32:comdlg32.dll
 0001:000156a4       _GetSaveFileNameA@4        004166a4 f   comdlg32:comdlg32.dll
 0001:000156aa       _RegCloseKey@4             004166aa f   advapi32:ADVAPI32.dll
 0001:000156b0       _RegSetValueExA@24         004166b0 f   advapi32:ADVAPI32.dll
 0001:000156b6       _RegQueryValueExA@24       004166b6 f   advapi32:ADVAPI32.dll
 0001:000156bc       _RegCreateKeyExA@36        004166bc f   advapi32:ADVAPI32.dll
 0001:000156c2       _RegCreateKeyA@12          004166c2 f   advapi32:ADVAPI32.dll
 0001:000156c8       _RegDeleteValueA@8         004166c8 f   advapi32:ADVAPI32.dll
 0001:000156ce       _RegEnumValueA@32          004166ce f   advapi32:ADVAPI32.dll
 0001:000156d4       _RegQueryInfoKeyA@48       004166d4 f   advapi32:ADVAPI32.dll
 0001:000156da       _RegSetValueA@20           004166da f   advapi32:ADVAPI32.dll
 0001:000156e0       _RegOpenKeyA@12            004166e0 f   advapi32:ADVAPI32.dll
 0001:000156e6       _Shell_NotifyIconA@8       004166e6 f   shell32:SHELL32.dll
 0001:000156ec       _getpeername@12            004166ec f   wsock32:WSOCK32.dll
 0001:000156f2       _connect@12                004166f2 f   wsock32:WSOCK32.dll
 0001:000156f8       _htons@4                   004166f8 f   wsock32:WSOCK32.dll
 0001:000156fe       _gethostbyname@4           004166fe f   wsock32:WSOCK32.dll
 0001:00015704       _inet_addr@4               00416704 f   wsock32:WSOCK32.dll
 0001:0001570a       _socket@12                 0041670a f   wsock32:WSOCK32.dll
 0001:00015710       _setsockopt@20             00416710 f   wsock32:WSOCK32.dll
 0001:00015716       _closesocket@4             00416716 f   wsock32:WSOCK32.dll
 0001:0001571c       _shutdown@8                0041671c f   wsock32:WSOCK32.dll
 0001:00015722       _WSAGetLastError@0         00416722 f   wsock32:WSOCK32.dll
 0001:00015728       _recv@16                   00416728 f   wsock32:WSOCK32.dll
 0001:0001572e       _send@16                   0041672e f   wsock32:WSOCK32.dll
 0001:00015734       _WSAAsyncSelect@16         00416734 f   wsock32:WSOCK32.dll
 0001:0001573a       _listen@8                  0041673a f   wsock32:WSOCK32.dll
 0001:00015740       _bind@12                   00416740 f   wsock32:WSOCK32.dll
 0001:00015746       _ioctlsocket@12            00416746 f   wsock32:WSOCK32.dll
 0001:0001574c       _accept@12                 0041674c f   wsock32:WSOCK32.dll
 0001:00015752       _WSACleanup@0              00416752 f   wsock32:WSOCK32.dll
 0001:00015758       _WSAStartup@8              00416758 f   wsock32:WSOCK32.dll
 0001:00015760       ??3@YAXPAX@Z               00416760 f   LIBCMTD:dbgdel.obj
 0001:00015810       ?_JumpToContinuation@@YGXPAXPAUEHRegistrationNode@@@Z 00416810 f   LIBCMTD:trnsctrl.obj
 0001:00015850       ?_CallMemberFunction0@@YGXPAX0@Z 00416850 f   LIBCMTD:trnsctrl.obj
 0001:00015860       ?_CallMemberFunction1@@YGXPAX00@Z 00416860 f   LIBCMTD:trnsctrl.obj
 0001:00015870       ?_CallMemberFunction2@@YGXPAX00H@Z 00416870 f   LIBCMTD:trnsctrl.obj
 0001:00015880       ?_UnwindNestedFrames@@YGXPAUEHRegistrationNode@@PAUEHExceptionRecord@@@Z 00416880 f   LIBCMTD:trnsctrl.obj
 0001:000158e0       ___CxxFrameHandler         004168e0 f   LIBCMTD:trnsctrl.obj
 0001:00015920       ___CxxLongjmpUnwind@4      00416920 f   LIBCMTD:trnsctrl.obj
 0001:00015950       ?_CallCatchBlock2@@YAPAXPAUEHRegistrationNode@@PBU_s_FuncInfo@@PAXHK@Z 00416950 f   LIBCMTD:trnsctrl.obj
 0001:00015a00       ?_CallSETranslator@@YAHPAUEHExceptionRecord@@PAUEHRegistrationNode@@PAX2PBU_s_FuncInfo@@H1@Z 00416a00 f   LIBCMTD:trnsctrl.obj
 0001:00015b60       ?_GetRangeOfTrysToCheck@@YAPBU_s_TryBlockMapEntry@@PBU_s_FuncInfo@@HHPAI1@Z 00416b60 f   LIBCMTD:trnsctrl.obj
 0001:00015bf0       __global_unwind2           00416bf0 f   LIBCMTD:exsup.obj
 0001:00015c32       __local_unwind2            00416c32 f   LIBCMTD:exsup.obj
 0001:00015c8a       __NLG_Return2              00416c8a f   LIBCMTD:exsup.obj
 0001:00015c9a       __abnormal_termination     00416c9a f   LIBCMTD:exsup.obj
 0001:00015cbd       __NLG_Notify1              00416cbd f   LIBCMTD:exsup.obj
 0001:00015cc6       __NLG_Notify               00416cc6 f   LIBCMTD:exsup.obj
 0001:00015cd9       __NLG_Dispatch             00416cd9 f   LIBCMTD:exsup.obj
 0001:00015ce0       _strcpy                    00416ce0 f   LIBCMTD:strcat.obj
 0001:00015cf0       _strcat                    00416cf0 f   LIBCMTD:strcat.obj
 0001:00015dd0       _sprintf                   00416dd0 f   LIBCMTD:sprintf.obj
 0001:00015ed0       _strncpy                   00416ed0 f   LIBCMTD:strncpy.obj
 0001:00015fd0       ??1type_info@@UAE@XZ       00416fd0 f   LIBCMTD:typinfo.obj
 0001:00016010       ??_Gtype_info@@UAEPAXI@Z   00417010 f i LIBCMTD:typinfo.obj
 0001:00016010       ??_Etype_info@@UAEPAXI@Z   00417010 f i LIBCMTD:typinfo.obj
 0001:00016040       ??8type_info@@QBEHABV0@@Z  00417040 f   LIBCMTD:typinfo.obj
 0001:00016070       ??9type_info@@QBEHABV0@@Z  00417070 f   LIBCMTD:typinfo.obj
 0001:000160a0       ?before@type_info@@QBEHABV1@@Z 004170a0 f   LIBCMTD:typinfo.obj
 0001:000160d0       ?raw_name@type_info@@QBEPBDXZ 004170d0 f   LIBCMTD:typinfo.obj
 0001:000160f0       ??0type_info@@AAE@ABV0@@Z  004170f0 f   LIBCMTD:typinfo.obj
 0001:00016110       ??4type_info@@AAEAAV0@ABV0@@Z 00417110 f   LIBCMTD:typinfo.obj
 0001:00016120       __CxxThrowException@8      00417120 f   LIBCMTD:throw.obj
 0001:00016170       _sscanf                    00417170 f   LIBCMTD:sscanf.obj
 0001:00016230       _malloc                    00417230 f   LIBCMTD:dbgheap.obj
 0001:00016260       __malloc_dbg               00417260 f   LIBCMTD:dbgheap.obj
 0001:00016290       __nh_malloc                00417290 f   LIBCMTD:dbgheap.obj
 0001:000162b0       __nh_malloc_dbg            004172b0 f   LIBCMTD:dbgheap.obj
 0001:00016350       __heap_alloc               00417350 f   LIBCMTD:dbgheap.obj
 0001:00016370       __heap_alloc_dbg           00417370 f   LIBCMTD:dbgheap.obj
 0001:00016690       _calloc                    00417690 f   LIBCMTD:dbgheap.obj
 0001:000166c0       __calloc_dbg               004176c0 f   LIBCMTD:dbgheap.obj
 0001:00016720       _realloc                   00417720 f   LIBCMTD:dbgheap.obj
 0001:00016750       __realloc_dbg              00417750 f   LIBCMTD:dbgheap.obj
 0001:00016d00       __expand                   00417d00 f   LIBCMTD:dbgheap.obj
 0001:00016d30       __expand_dbg               00417d30 f   LIBCMTD:dbgheap.obj
 0001:00016dc0       _free                      00417dc0 f   LIBCMTD:dbgheap.obj
 0001:00016de0       __free_lk                  00417de0 f   LIBCMTD:dbgheap.obj
 0001:00016e00       __free_dbg                 00417e00 f   LIBCMTD:dbgheap.obj
 0001:00016e70       __free_dbg_lk              00417e70 f   LIBCMTD:dbgheap.obj
 0001:00017260       __msize                    00418260 f   LIBCMTD:dbgheap.obj
 0001:00017280       __msize_dbg                00418280 f   LIBCMTD:dbgheap.obj
 0001:00017410       __CrtSetBreakAlloc         00418410 f   LIBCMTD:dbgheap.obj
 0001:00017430       __CrtSetDbgBlockType       00418430 f   LIBCMTD:dbgheap.obj
 0001:00017510       __CrtSetAllocHook          00418510 f   LIBCMTD:dbgheap.obj
 0001:000175c0       __CrtCheckMemory           004185c0 f   LIBCMTD:dbgheap.obj
 0001:00017970       __CrtSetDbgFlag            00418970 f   LIBCMTD:dbgheap.obj
 0001:000179a0       __CrtDoForAllClientObjects 004189a0 f   LIBCMTD:dbgheap.obj
 0001:00017a50       __CrtIsValidPointer        00418a50 f   LIBCMTD:dbgheap.obj
 0001:00017aa0       __CrtIsValidHeapPointer    00418aa0 f   LIBCMTD:dbgheap.obj
 0001:00017bd0       __CrtIsMemoryBlock         00418bd0 f   LIBCMTD:dbgheap.obj
 0001:00017d00       __CrtSetDumpClient         00418d00 f   LIBCMTD:dbgheap.obj
 0001:00017d20       __CrtMemCheckpoint         00418d20 f   LIBCMTD:dbgheap.obj
 0001:00017ed0       __CrtMemDifference         00418ed0 f   LIBCMTD:dbgheap.obj
 0001:00018000       __CrtMemDumpAllObjectsSince 00419000 f   LIBCMTD:dbgheap.obj
 0001:00018420       __CrtDumpMemoryLeaks       00419420 f   LIBCMTD:dbgheap.obj
 0001:000184a0       __CrtMemDumpStatistics     004194a0 f   LIBCMTD:dbgheap.obj
 0001:00018570       _strlen                    00419570 f   LIBCMTD:strlen.obj
 0001:000185f0       ??2@YAPAXI@Z               004195f0 f   LIBCMTD:new.obj
 0001:00018610       _abs                       00419610 f   LIBCMTD:abs.obj
 0001:00018640       _memcmp                    00419640 f   LIBCMTD:memcmp.obj
 0001:000186f0       _memcpy                    004196f0 f   LIBCMTD:memcpy.obj
 0001:00018a30       _memset                    00419a30 f   LIBCMTD:memset.obj
 0001:00018a90       __assert                   00419a90 f   LIBCMTD:assert.obj
 0001:00018e10       __CrtDbgBreak              00419e10 f   LIBCMTD:dbgrpt.obj
 0001:00018e20       __CrtSetReportMode         00419e20 f   LIBCMTD:dbgrpt.obj
 0001:00018e80       __CrtSetReportFile         00419e80 f   LIBCMTD:dbgrpt.obj
 0001:00018f00       __CrtSetReportHook         00419f00 f   LIBCMTD:dbgrpt.obj
 0001:00018f20       __CrtDbgReport             00419f20 f   LIBCMTD:dbgrpt.obj
 0001:000195c0       _vsprintf                  0041a5c0 f   LIBCMTD:vsprintf.obj
 0001:000196c0       __onexit                   0041a6c0 f   LIBCMTD:onexit.obj
 0001:00019780       _atexit                    0041a780 f   LIBCMTD:onexit.obj
 0001:000197a0       ___onexitinit              0041a7a0 f   LIBCMTD:onexit.obj
 0001:000197f0       _strcmp                    0041a7f0 f   LIBCMTD:strcmp.obj
 0001:00019890       _strchr                    0041a890 f   LIBCMTD:strchr.obj
 0001:00019896       ___from_strstr_to_strchr   0041a896 f   LIBCMTD:strchr.obj
 0001:00019950       __strdup                   0041a950 f   LIBCMTD:strdup.obj
 0001:000199a0       __access                   0041a9a0 f   LIBCMTD:access.obj
 0001:00019a00       __fullpath                 0041aa00 f   LIBCMTD:fullpath.obj
 0001:00019ae0       __strcmpi                  0041aae0 f   LIBCMTD:stricmp.obj
 0001:00019ae0       __stricmp                  0041aae0 f   LIBCMTD:stricmp.obj
 0001:00019bb0       __purecall                 0041abb0 f   LIBCMTD:purevirt.obj
 0001:00019bc0       __cinit                    0041abc0 f   LIBCMTD:crt0dat.obj
 0001:00019c00       _exit                      0041ac00 f   LIBCMTD:crt0dat.obj
 0001:00019c20       __exit                     0041ac20 f   LIBCMTD:crt0dat.obj
 0001:00019c40       __cexit                    0041ac40 f   LIBCMTD:crt0dat.obj
 0001:00019c60       __c_exit                   0041ac60 f   LIBCMTD:crt0dat.obj
 0001:00019d70       __lockexit                 0041ad70 f   LIBCMTD:crt0dat.obj
 0001:00019d80       __unlockexit               0041ad80 f   LIBCMTD:crt0dat.obj
 0001:00019dc0       _WinMainCRTStartup         0041adc0 f   LIBCMTD:wincrt0.obj
 0001:00019f30       __amsg_exit                0041af30 f   LIBCMTD:wincrt0.obj
 0001:00019f90       __beginthreadex            0041af90 f   LIBCMTD:threadex.obj
 0001:0001a150       __endthreadex              0041b150 f   LIBCMTD:threadex.obj
 0001:0001a1a0       __mtinitlocks              0041b1a0 f   LIBCMTD:mlock.obj
 0001:0001a1e0       __mtdeletelocks            0041b1e0 f   LIBCMTD:mlock.obj
 0001:0001a280       __lock                     0041b280 f   LIBCMTD:mlock.obj
 0001:0001a320       __unlock                   0041b320 f   LIBCMTD:mlock.obj
 0001:0001a340       __lockerr_exit             0041b340 f   LIBCMTD:mlock.obj
 0001:0001a360       ___InternalCxxFrameHandler 0041b360 f   LIBCMTD:frame.obj
 0001:0001a8d0       ___FrameUnwindToState      0041b8d0 f   LIBCMTD:frame.obj
 0001:0001aee0       ?_DestructExceptionObject@@YAXPAUEHExceptionRecord@@E@Z 0041bee0 f   LIBCMTD:frame.obj
 0001:0001afc0       __CallSettingFrame@12      0041bfc0 f   LIBCMTD:lowhelpr.obj
 0001:0001afe7       __NLG_Return               0041bfe7 f   LIBCMTD:lowhelpr.obj
 0001:0001b010       __mtinit                   0041c010 f   LIBCMTD:tidtable.obj
 0001:0001b0a0       __mtterm                   0041c0a0 f   LIBCMTD:tidtable.obj
 0001:0001b0d0       __initptd                  0041c0d0 f   LIBCMTD:tidtable.obj
 0001:0001b0f0       __getptd                   0041c0f0 f   LIBCMTD:tidtable.obj
 0001:0001b190       __freeptd                  0041c190 f   LIBCMTD:tidtable.obj
 0001:0001b2a0       ___threadid                0041c2a0 f   LIBCMTD:tidtable.obj
 0001:0001b2b0       ___threadhandle            0041c2b0 f   LIBCMTD:tidtable.obj
 0001:0001b2c0       ?terminate@@YAXXZ          0041c2c0 f   LIBCMTD:hooks.obj
 0001:0001b350       ?unexpected@@YAXXZ         0041c350 f   LIBCMTD:hooks.obj
 0001:0001b370       ?_inconsistency@@YAXXZ     0041c370 f   LIBCMTD:hooks.obj
 0001:0001b400       __flsbuf                   0041c400 f   LIBCMTD:_flsbuf.obj
 0001:0001b680       __output                   0041c680 f   LIBCMTD:output.obj
 0001:0001c5b0       __free_base                0041d5b0 f   LIBCMTD:free.obj
 0001:0001c700       ?__CxxUnhandledExceptionFilter@@YGJPAU_EXCEPTION_POINTERS@@@Z 0041d700 f   LIBCMTD:unhandld.obj
 0001:0001c760       ?__CxxSetUnhandledExceptionFilter@@YAXXZ 0041d760 f   LIBCMTD:unhandld.obj
 0001:0001c780       ?__CxxRestoreUnhandledExceptionFilter@@YAXXZ 0041d780 f   LIBCMTD:unhandld.obj
 0001:0001c7a0       __input                    0041d7a0 f   LIBCMTD:input.obj
 0001:0001dca0       ?_set_new_handler@@YAP6AHI@ZP6AHI@Z@Z 0041eca0 f   LIBCMTD:handler.obj
 0001:0001dcd0       ?_query_new_handler@@YAP6AHI@ZXZ 0041ecd0 f   LIBCMTD:handler.obj
 0001:0001dce0       __callnewh                 0041ece0 f   LIBCMTD:handler.obj
 0001:0001dd18       __except_handler3          0041ed18 f   LIBCMTD:exsup3.obj
 0001:0001ddd5       __seh_longjmp_unwind@4     0041edd5 f   LIBCMTD:exsup3.obj
 0001:0001ddf0       __malloc_base              0041edf0 f   LIBCMTD:malloc.obj
 0001:0001de10       __nh_malloc_base           0041ee10 f   LIBCMTD:malloc.obj
 0001:0001de70       __heap_alloc_base          0041ee70 f   LIBCMTD:malloc.obj
 0001:0001dfc0       __CrtDefaultAllocHook      0041efc0 f   LIBCMTD:dbghook.obj
 0001:0001dfd0       __expand_base              0041efd0 f   LIBCMTD:expand.obj
 0001:0001e1e0       __realloc_base             0041f1e0 f   LIBCMTD:realloc.obj
 0001:0001e680       __heapchk                  0041f680 f   LIBCMTD:heapchk.obj
 0001:0001e790       __heapset                  0041f790 f   LIBCMTD:heapchk.obj
 0001:0001e7a0       __get_sbh_threshold        0041f7a0 f   LIBCMTD:sbheap.obj
 0001:0001e7d0       __set_sbh_threshold        0041f7d0 f   LIBCMTD:sbheap.obj
 0001:0001e8e0       ___sbh_heap_init           0041f8e0 f   LIBCMTD:sbheap.obj
 0001:0001e950       ___sbh_find_block          0041f950 f   LIBCMTD:sbheap.obj
 0001:0001e9b0       ___sbh_verify_block        0041f9b0 f   LIBCMTD:sbheap.obj
 0001:0001ea10       ___sbh_free_block          0041fa10 f   LIBCMTD:sbheap.obj
 0001:0001eff0       ___sbh_alloc_block         0041fff0 f   LIBCMTD:sbheap.obj
 0001:0001f530       ___sbh_alloc_new_region    00420530 f   LIBCMTD:sbheap.obj
 0001:0001f640       ___sbh_alloc_new_group     00420640 f   LIBCMTD:sbheap.obj
 0001:0001f830       ___sbh_resize_block        00420830 f   LIBCMTD:sbheap.obj
 0001:0001fe20       ___sbh_heapmin             00420e20 f   LIBCMTD:sbheap.obj
 0001:0001ff50       ___sbh_heap_check          00420f50 f   LIBCMTD:sbheap.obj
 0001:00020570       __get_old_sbh_threshold    00421570 f   LIBCMTD:sbheap.obj
 0001:00020580       __set_old_sbh_threshold    00421580 f   LIBCMTD:sbheap.obj
 0001:000205b0       ___old_sbh_new_region      004215b0 f   LIBCMTD:sbheap.obj
 0001:00020790       ___old_sbh_release_region  00421790 f   LIBCMTD:sbheap.obj
 0001:00020810       ___old_sbh_decommit_pages  00421810 f   LIBCMTD:sbheap.obj
 0001:00020970       ___old_sbh_find_block      00421970 f   LIBCMTD:sbheap.obj
 0001:00020a00       ___old_sbh_free_block      00421a00 f   LIBCMTD:sbheap.obj
 0001:00020a70       ___old_sbh_alloc_block     00421a70 f   LIBCMTD:sbheap.obj
 0001:00020e30       ___old_sbh_alloc_block_from_page 00421e30 f   LIBCMTD:sbheap.obj
 0001:000210e0       ___old_sbh_resize_block    004220e0 f   LIBCMTD:sbheap.obj
 0001:00021250       ___old_sbh_heap_check      00422250 f   LIBCMTD:sbheap.obj
 0001:00021490       __GetLinkerVersion         00422490 f   LIBCMTD:heapinit.obj
 0001:000214f0       ___heap_select             004224f0 f   LIBCMTD:heapinit.obj
 0001:00021720       __heap_init                00422720 f   LIBCMTD:heapinit.obj
 0001:000217b0       __heap_term                004227b0 f   LIBCMTD:heapinit.obj
 0001:000218a0       __isctype                  004228a0 f   LIBCMTD:isctype.obj
 0001:00021960       _abort                     00422960 f   LIBCMTD:abort.obj
 0001:00021980       _signal                    00422980 f   LIBCMTD:winsig.obj
 0001:00021c50       _raise                     00422c50 f   LIBCMTD:winsig.obj
 0001:00021ef0       ___fpecode                 00422ef0 f   LIBCMTD:winsig.obj
 0001:00021f00       ___pxcptinfoptrs           00422f00 f   LIBCMTD:winsig.obj
 0001:00021f10       ___crtMessageBoxA          00422f10 f   LIBCMTD:crtmbox.obj
 0001:00021fd0       __itoa                     00422fd0 f   LIBCMTD:xtoa.obj
 0001:000220f0       __ltoa                     004230f0 f   LIBCMTD:xtoa.obj
 0001:00022130       __ultoa                    00423130 f   LIBCMTD:xtoa.obj
 0001:00022150       __i64toa                   00423150 f   LIBCMTD:xtoa.obj
 0001:000222a0       __ui64toa                  004232a0 f   LIBCMTD:xtoa.obj
 0001:000222c0       _strncat                   004232c0 f   LIBCMTD:strncat.obj
 0001:000223f0       _fflush                    004233f0 f   LIBCMTD:fflush.obj
 0001:00022440       __fflush_lk                00423440 f   LIBCMTD:fflush.obj
 0001:00022490       __flush                    00423490 f   LIBCMTD:fflush.obj
 0001:00022550       __flushall                 00423550 f   LIBCMTD:fflush.obj
 0001:000226a0       _fprintf                   004236a0 f   LIBCMTD:fprintf.obj
 0001:00022770       _setvbuf                   00423770 f   LIBCMTD:setvbuf.obj
 0001:000228e0       ___initstdio               004238e0 f   LIBCMTD:_file.obj
 0001:00022a10       ___endstdio                00423a10 f   LIBCMTD:_file.obj
 0001:00022a30       __lock_file                00423a30 f   LIBCMTD:_file.obj
 0001:00022a70       __lock_file2               00423a70 f   LIBCMTD:_file.obj
 0001:00022aa0       __unlock_file              00423aa0 f   LIBCMTD:_file.obj
 0001:00022ae0       __unlock_file2             00423ae0 f   LIBCMTD:_file.obj
 0001:00022b10       __snprintf                 00423b10 f   LIBCMTD:snprintf.obj
 0001:00022c10       __vsnprintf                00423c10 f   LIBCMTD:vsnprint.obj
 0001:00022d10       __alloca_probe             00423d10 f   LIBCMTD:chkstk.obj
 0001:00022d10       __chkstk                   00423d10 f   LIBCMTD:chkstk.obj
 0001:00022d40       __dosmaperr                00423d40 f   LIBCMTD:dosmap.obj
 0001:00022de0       __errno                    00423de0 f   LIBCMTD:dosmap.obj
 0001:00022df0       ___doserrno                00423df0 f   LIBCMTD:dosmap.obj
 0001:00022e00       __getcwd                   00423e00 f   LIBCMTD:getcwd.obj
 0001:00022e40       __getdcwd                  00423e40 f   LIBCMTD:getcwd.obj
 0001:00022e80       __getdcwd_lk               00423e80 f   LIBCMTD:getcwd.obj
 0001:00022fa0       __validdrive               00423fa0 f   LIBCMTD:getcwd.obj
 0001:00022ff0       _setlocale                 00423ff0 f   LIBCMTD:setlocal.obj
 0001:00023680       __expandlocale             00424680 f   LIBCMTD:setlocal.obj
 0001:00023810       ___init_dummy              00424810 f   LIBCMTD:setlocal.obj
 0001:00023820       __strcats                  00424820 f   LIBCMTD:setlocal.obj
 0001:00023870       ___lc_strtolc              00424870 f   LIBCMTD:setlocal.obj
 0001:000239d0       ___lc_lctostr              004249d0 f   LIBCMTD:setlocal.obj
 0001:00023a40       __tolower                  00424a40 f   LIBCMTD:tolower.obj
 0001:00023a50       _tolower                   00424a50 f   LIBCMTD:tolower.obj
 0001:00023af0       __tolower_lk               00424af0 f   LIBCMTD:tolower.obj
 0001:00023c20       __XcptFilter               00424c20 f   LIBCMTD:winxfltr.obj
 0001:00023e40       __wincmdln                 00424e40 f   LIBCMTD:wincmdln.obj
 0001:00023f00       __setenvp                  00424f00 f   LIBCMTD:stdenvp.obj
 0001:00024050       __setargv                  00425050 f   LIBCMTD:stdargv.obj
 0001:00024560       ___crtGetEnvironmentStringsA 00425560 f   LIBCMTD:a_env.obj
 0001:00024780       __ioinit                   00425780 f   LIBCMTD:ioinit.obj
 0001:00024ab0       __ioterm                   00425ab0 f   LIBCMTD:ioinit.obj
 0001:00024b50       __FF_MSGBANNER             00425b50 f   LIBCMTD:crt0msg.obj
 0001:00024ba0       __NMSG_WRITE               00425ba0 f   LIBCMTD:crt0msg.obj
 0001:00024d60       __GET_RTERRMSG             00425d60 f   LIBCMTD:crt0msg.obj
 0001:00024db0       ?_ValidateRead@@YAHPBXI@Z  00425db0 f   LIBCMTD:validate.obj
 0001:00024de0       ?_ValidateWrite@@YAHPAXI@Z 00425de0 f   LIBCMTD:validate.obj
 0001:00024e10       ?_ValidateExecute@@YAHP6GHXZ@Z 00425e10 f   LIBCMTD:validate.obj
 0001:00024e40       _memmove                   00425e40 f   LIBCMTD:memmove.obj
 0001:00025180       __lseek                    00426180 f   LIBCMTD:lseek.obj
 0001:00025210       __lseek_lk                 00426210 f   LIBCMTD:lseek.obj
 0001:000252d0       __write                    004262d0 f   LIBCMTD:write.obj
 0001:00025360       __write_lk                 00426360 f   LIBCMTD:write.obj
 0001:000255e0       __getbuf                   004265e0 f   LIBCMTD:_getbuf.obj
 0001:000256b0       __isatty                   004266b0 f   LIBCMTD:isatty.obj
 0001:000256f0       _wctomb                    004266f0 f   LIBCMTD:wctomb.obj
 0001:00025770       __wctomb_lk                00426770 f   LIBCMTD:wctomb.obj
 0001:00025810       __aulldiv                  00426810 f   LIBCMTD:ulldiv.obj
 0001:00025880       __aullrem                  00426880 f   LIBCMTD:ullrem.obj
 0001:00025900       _mbtowc                    00426900 f   LIBCMTD:mbtowc.obj
 0001:00025980       __mbtowc_lk                00426980 f   LIBCMTD:mbtowc.obj
 0001:00025ae0       _isalpha                   00426ae0 f   LIBCMTD:_ctype.obj
 0001:00025b30       _isupper                   00426b30 f   LIBCMTD:_ctype.obj
 0001:00025b70       _islower                   00426b70 f   LIBCMTD:_ctype.obj
 0001:00025bb0       _isdigit                   00426bb0 f   LIBCMTD:_ctype.obj
 0001:00025bf0       _isxdigit                  00426bf0 f   LIBCMTD:_ctype.obj
 0001:00025c40       _isspace                   00426c40 f   LIBCMTD:_ctype.obj
 0001:00025c80       _ispunct                   00426c80 f   LIBCMTD:_ctype.obj
 0001:00025cc0       _isalnum                   00426cc0 f   LIBCMTD:_ctype.obj
 0001:00025d10       _isprint                   00426d10 f   LIBCMTD:_ctype.obj
 0001:00025d60       _isgraph                   00426d60 f   LIBCMTD:_ctype.obj
 0001:00025db0       _iscntrl                   00426db0 f   LIBCMTD:_ctype.obj
 0001:00025df0       ___isascii                 00426df0 f   LIBCMTD:_ctype.obj
 0001:00025e00       ___toascii                 00426e00 f   LIBCMTD:_ctype.obj
 0001:00025e10       ___iscsymf                 00426e10 f   LIBCMTD:_ctype.obj
 0001:00025e70       ___iscsym                  00426e70 f   LIBCMTD:_ctype.obj
 0001:00025ed0       __allshl                   00426ed0 f   LIBCMTD:llshl.obj
 0001:00025ef0       __filbuf                   00426ef0 f   LIBCMTD:_filbuf.obj
 0001:000260e0       _ungetc                    004270e0 f   LIBCMTD:ungetc.obj
 0001:00026150       __ungetc_lk                00427150 f   LIBCMTD:ungetc.obj
 0001:00026290       _strtol                    00427290 f   LIBCMTD:strtol.obj
 0001:000265f0       _strtoul                   004275f0 f   LIBCMTD:strtol.obj
 0001:00026610       _strstr                    00427610 f   LIBCMTD:strstr.obj
 0001:00026690       _strncmp                   00427690 f   LIBCMTD:strncmp.obj
 0001:000266d0       ___crtGetStringTypeA       004276d0 f   LIBCMTD:a_str.obj
 0001:00026890       __commit                   00427890 f   LIBCMTD:commit.obj
 0001:00026970       __stbuf                    00427970 f   LIBCMTD:_sftbuf.obj
 0001:00026ad0       __ftbuf                    00427ad0 f   LIBCMTD:_sftbuf.obj
 0001:00026b70       __freebuf                  00427b70 f   LIBCMTD:_freebuf.obj
 0001:00026c10       __fcloseall                00427c10 f   LIBCMTD:closeall.obj
 0001:00026cf0       ___init_time               00427cf0 f   LIBCMTD:inittime.obj
 0001:00027670       ___init_numeric            00428670 f   LIBCMTD:initnum.obj
 0001:000279a0       ___init_monetary           004289a0 f   LIBCMTD:initmon.obj
 0001:00027e00       ___init_ctype              00428e00 f   LIBCMTD:initctyp.obj
 0001:000281a0       ___init_collate            004291a0 f   LIBCMTD:initcoll.obj
 0001:000281b0       _strcspn                   004291b0 f   LIBCMTD:strcspn.obj
 0001:000281f0       _strpbrk                   004291f0 f   LIBCMTD:strpbrk.obj
 0001:00028230       ___get_qualified_locale    00429230 f   LIBCMTD:getqloc.obj
 0001:00028fd0       ___crtLCMapStringA         00429fd0 f   LIBCMTD:a_map.obj
 0001:00029330       __ismbbkalnum              0042a330 f   LIBCMTD:ismbbyte.obj
 0001:00029350       __ismbbkprint              0042a350 f   LIBCMTD:ismbbyte.obj
 0001:00029370       __ismbbkpunct              0042a370 f   LIBCMTD:ismbbyte.obj
 0001:00029390       __ismbbalnum               0042a390 f   LIBCMTD:ismbbyte.obj
 0001:000293b0       __ismbbalpha               0042a3b0 f   LIBCMTD:ismbbyte.obj
 0001:000293d0       __ismbbgraph               0042a3d0 f   LIBCMTD:ismbbyte.obj
 0001:000293f0       __ismbbprint               0042a3f0 f   LIBCMTD:ismbbyte.obj
 0001:00029410       __ismbbpunct               0042a410 f   LIBCMTD:ismbbyte.obj
 0001:00029430       __ismbblead                0042a430 f   LIBCMTD:ismbbyte.obj
 0001:00029450       __ismbbtrail               0042a450 f   LIBCMTD:ismbbyte.obj
 0001:00029470       __ismbbkana                0042a470 f   LIBCMTD:ismbbyte.obj
 0001:00029520       __setmbcp                  0042a520 f   LIBCMTD:mbctype.obj
 0001:00029ce0       __getmbcp                  0042ace0 f   LIBCMTD:mbctype.obj
 0001:00029d00       ___initmbctable            0042ad00 f   LIBCMTD:mbctype.obj
 0001:00029d30       __alloc_osfhnd             0042ad30 f   LIBCMTD:osfinfo.obj
 0001:00029f20       __set_osfhnd               0042af20 f   LIBCMTD:osfinfo.obj
 0001:00029fe0       __free_osfhnd              0042afe0 f   LIBCMTD:osfinfo.obj
 0001:0002a0c0       __get_osfhandle            0042b0c0 f   LIBCMTD:osfinfo.obj
 0001:0002a130       __open_osfhandle           0042b130 f   LIBCMTD:osfinfo.obj
 0001:0002a240       __lock_fhandle             0042b240 f   LIBCMTD:osfinfo.obj
 0001:0002a2d0       __unlock_fhandle           0042b2d0 f   LIBCMTD:osfinfo.obj
 0001:0002a300       __fptrap                   0042b300 f   LIBCMTD:crt0fp.obj
 0001:0002a310       __read                     0042b310 f   LIBCMTD:read.obj
 0001:0002a3a0       __read_lk                  0042b3a0 f   LIBCMTD:read.obj
 0001:0002a7f0       __toupper                  0042b7f0 f   LIBCMTD:toupper.obj
 0001:0002a800       _toupper                   0042b800 f   LIBCMTD:toupper.obj
 0001:0002a8a0       __toupper_lk               0042b8a0 f   LIBCMTD:toupper.obj
 0001:0002a9d0       _fclose                    0042b9d0 f   LIBCMTD:fclose.obj
 0001:0002aa60       __fclose_lk                0042ba60 f   LIBCMTD:fclose.obj
 0001:0002ab20       __Getdays                  0042bb20 f   LIBCMTD:strftime.obj
 0001:0002ac50       __Getmonths                0042bc50 f   LIBCMTD:strftime.obj
 0001:0002ad80       __Gettnames                0042bd80 f   LIBCMTD:strftime.obj
 0001:0002b0f0       _strftime                  0042c0f0 f   LIBCMTD:strftime.obj
 0001:0002b110       __Strftime                 0042c110 f   LIBCMTD:strftime.obj
 0001:0002c030       ___getlocaleinfo           0042d030 f   LIBCMTD:inithelp.obj
 0001:0002c2c0       _localeconv                0042d2c0 f   LIBCMTD:lconv.obj
 0001:0002c2d0       ___crtGetStringTypeW       0042d2d0 f   LIBCMTD:w_str.obj
 0001:0002c540       __strnicmp                 0042d540 f   LIBCMTD:strnicmp.obj
 0001:0002c650       _atol                      0042d650 f   LIBCMTD:atox.obj
 0001:0002c750       _atoi                      0042d750 f   LIBCMTD:atox.obj
 0001:0002c770       __atoi64                   0042d770 f   LIBCMTD:atox.obj
 0001:0002c8a0       __close                    0042d8a0 f   LIBCMTD:close.obj
 0001:0002c920       __close_lk                 0042d920 f   LIBCMTD:close.obj
 0001:0002c9d0       ___tzset                   0042d9d0 f   LIBCMTD:tzset.obj
 0001:0002ca10       __tzset                    0042da10 f   LIBCMTD:tzset.obj
 0001:0002cde0       __isindst                  0042dde0 f   LIBCMTD:tzset.obj
 0001:0002d310       ___crtGetLocaleInfoW       0042e310 f   LIBCMTD:w_loc.obj
 0001:0002d4b0       ___crtGetLocaleInfoA       0042e4b0 f   LIBCMTD:a_loc.obj
 0001:0002d660       __allmul                   0042e660 f   LIBCMTD:llmul.obj
 0001:0002d6a0       _getenv                    0042e6a0 f   LIBCMTD:getenv.obj
 0001:0002d6d0       __getenv_lk                0042e6d0 f   LIBCMTD:getenv.obj
 0001:0002d7a0       __mbsnbicoll               0042e7a0 f   LIBCMTD:mbsnbico.obj
 0001:0002d7f0       ___wtomb_environ           0042e7f0 f   LIBCMTD:wtombenv.obj
 0001:0002d8a0       ___crtCompareStringA       0042e8a0 f   LIBCMTD:a_cmp.obj
 0001:0002dcf0       ___crtsetenv               0042ecf0 f   LIBCMTD:setenv.obj
 0001:0002e140       __mbschr                   0042f140 f   LIBCMTD:mbschr.obj
 0001:0002e22e       _RtlUnwind@16              0042f22e f   kernel32:KERNEL32.dll
 0001:0002e234       _RaiseException@16         0042f234 f   kernel32:KERNEL32.dll
 0001:0002e23a       _IsBadWritePtr@8           0042f23a f   kernel32:KERNEL32.dll
 0001:0002e240       _IsBadReadPtr@8            0042f240 f   kernel32:KERNEL32.dll
 0001:0002e246       _HeapValidate@12           0042f246 f   kernel32:KERNEL32.dll
 0001:0002e24c       _DebugBreak@0              0042f24c f   kernel32:KERNEL32.dll
 0001:0002e252       _InterlockedDecrement@4    0042f252 f   kernel32:KERNEL32.dll
 0001:0002e258       _GetProcAddress@8          0042f258 f   kernel32:KERNEL32.dll
 0001:0002e25e       _LoadLibraryA@4            0042f25e f   kernel32:KERNEL32.dll
 0001:0002e264       _InterlockedIncrement@4    0042f264 f   kernel32:KERNEL32.dll
 0001:0002e26a       _GetFileAttributesA@4      0042f26a f   kernel32:KERNEL32.dll
 0001:0002e270       _GetFullPathNameA@16       0042f270 f   kernel32:KERNEL32.dll
 0001:0002e276       _ExitProcess@4             0042f276 f   kernel32:KERNEL32.dll
 0001:0002e27c       _TerminateProcess@8        0042f27c f   kernel32:KERNEL32.dll
 0001:0002e282       _GetModuleHandleA@4        0042f282 f   kernel32:KERNEL32.dll
 0001:0002e288       _GetStartupInfoA@4         0042f288 f   kernel32:KERNEL32.dll
 0001:0002e28e       _GetCommandLineA@0         0042f28e f   kernel32:KERNEL32.dll
 0001:0002e294       _GetVersion@0              0042f294 f   kernel32:KERNEL32.dll
 0001:0002e29a       _CreateThread@24           0042f29a f   kernel32:KERNEL32.dll
 0001:0002e2a0       _ExitThread@4              0042f2a0 f   kernel32:KERNEL32.dll
 0001:0002e2a6       _FatalAppExitA@8           0042f2a6 f   kernel32:KERNEL32.dll
 0001:0002e2ac       _TlsFree@4                 0042f2ac f   kernel32:KERNEL32.dll
 0001:0002e2b2       _SetLastError@4            0042f2b2 f   kernel32:KERNEL32.dll
 0001:0002e2b8       _HeapFree@12               0042f2b8 f   kernel32:KERNEL32.dll
 0001:0002e2be       _SetUnhandledExceptionFilter@4 0042f2be f   kernel32:KERNEL32.dll
 0001:0002e2c4       _HeapAlloc@12              0042f2c4 f   kernel32:KERNEL32.dll
 0001:0002e2ca       _HeapReAlloc@16            0042f2ca f   kernel32:KERNEL32.dll
 0001:0002e2d0       _VirtualFree@12            0042f2d0 f   kernel32:KERNEL32.dll
 0001:0002e2d6       _VirtualAlloc@16           0042f2d6 f   kernel32:KERNEL32.dll
 0001:0002e2dc       _GetEnvironmentVariableA@12 0042f2dc f   kernel32:KERNEL32.dll
 0001:0002e2e2       _HeapDestroy@4             0042f2e2 f   kernel32:KERNEL32.dll
 0001:0002e2e8       _HeapCreate@12             0042f2e8 f   kernel32:KERNEL32.dll
 0001:0002e2ee       _SetConsoleCtrlHandler@8   0042f2ee f   kernel32:KERNEL32.dll
 0001:0002e2f4       _GetCurrentDirectoryA@8    0042f2f4 f   kernel32:KERNEL32.dll
 0001:0002e2fa       _GetDriveTypeA@4           0042f2fa f   kernel32:KERNEL32.dll
 0001:0002e300       _UnhandledExceptionFilter@4 0042f300 f   kernel32:KERNEL32.dll
 0001:0002e306       _FreeEnvironmentStringsA@4 0042f306 f   kernel32:KERNEL32.dll
 0001:0002e30c       _FreeEnvironmentStringsW@4 0042f30c f   kernel32:KERNEL32.dll
 0001:0002e312       _WideCharToMultiByte@32    0042f312 f   kernel32:KERNEL32.dll
 0001:0002e318       _GetEnvironmentStrings@0   0042f318 f   kernel32:KERNEL32.dll
 0001:0002e31e       _GetEnvironmentStringsW@0  0042f31e f   kernel32:KERNEL32.dll
 0001:0002e324       _SetHandleCount@4          0042f324 f   kernel32:KERNEL32.dll
 0001:0002e32a       _GetFileType@4             0042f32a f   kernel32:KERNEL32.dll
 0001:0002e330       _IsBadCodePtr@4            0042f330 f   kernel32:KERNEL32.dll
 0001:0002e336       _MultiByteToWideChar@24    0042f336 f   kernel32:KERNEL32.dll
 0001:0002e33c       _GetStringTypeA@20         0042f33c f   kernel32:KERNEL32.dll
 0001:0002e342       _GetStringTypeW@16         0042f342 f   kernel32:KERNEL32.dll
 0001:0002e348       _FlushFileBuffers@4        0042f348 f   kernel32:KERNEL32.dll
 0001:0002e34e       _GetCPInfo@8               0042f34e f   kernel32:KERNEL32.dll
 0001:0002e354       _IsValidLocale@8           0042f354 f   kernel32:KERNEL32.dll
 0001:0002e35a       _IsValidCodePage@4         0042f35a f   kernel32:KERNEL32.dll
 0001:0002e360       _GetLocaleInfoA@16         0042f360 f   kernel32:KERNEL32.dll
 0001:0002e366       _EnumSystemLocalesA@8      0042f366 f   kernel32:KERNEL32.dll
 0001:0002e36c       _GetUserDefaultLCID@0      0042f36c f   kernel32:KERNEL32.dll
 0001:0002e372       _LCMapStringA@24           0042f372 f   kernel32:KERNEL32.dll
 0001:0002e378       _LCMapStringW@24           0042f378 f   kernel32:KERNEL32.dll
 0001:0002e37e       _GetACP@0                  0042f37e f   kernel32:KERNEL32.dll
 0001:0002e384       _GetOEMCP@0                0042f384 f   kernel32:KERNEL32.dll
 0001:0002e38a       _SetStdHandle@8            0042f38a f   kernel32:KERNEL32.dll
 0001:0002e390       _ReadFile@20               0042f390 f   kernel32:KERNEL32.dll
 0001:0002e396       _GetTimeZoneInformation@4  0042f396 f   kernel32:KERNEL32.dll
 0001:0002e39c       _GetLocaleInfoW@16         0042f39c f   kernel32:KERNEL32.dll
 0001:0002e3a2       _CompareStringA@24         0042f3a2 f   kernel32:KERNEL32.dll
 0001:0002e3a8       _CompareStringW@24         0042f3a8 f   kernel32:KERNEL32.dll
 0001:0002e3ae       _SetEnvironmentVariableA@8 0042f3ae f   kernel32:KERNEL32.dll
 0001:000375c0       __enc$textbss$begin        004385c0     <linker-defined>
 0001:0004f0c0       __enc$textbss$end          004500c0     <linker-defined>
 0002:0000001c       ??_7AuthDialog@@6B@        0045101c     AuthDialog.obj
 0002:00000048       ??_7ClientConnection@@6B@  00451048     ClientConnection.obj
 0002:00000058       ??_C@_09DPKL@?$CIunknown?$CJ?$AA@ 00451058     ClientConnection.obj
 0002:00000064       ??_C@_0M@IBML@?$CFd?4?$CFd?4?$CFd?4?$CFd?$AA@ 00451064     ClientConnection.obj
 0002:00000074       ??_C@_0BI@CPFE@Close?5listening?5?$CGdaemon?$AA@ 00451074     ClientConnection.obj
 0002:00000090       ??_C@_0BE@EJE@?$CGAbout?5VNCviewer?4?4?4?$AA@ 00451090     ClientConnection.obj
 0002:000000a8       ??_C@_0BM@OAKP@Save?5connection?5info?5?$CGas?4?4?4?$AA@ 004510a8     ClientConnection.obj
 0002:000000cc       ??_C@_0BD@HJOM@Ne?$CGw?5connection?4?4?4?$AA@ 004510cc     ClientConnection.obj
 0002:000000e4       ??_C@_06NPMP@Alt?5Up?$AA@  004510e4     ClientConnection.obj
 0002:000000ec       ??_C@_08COAO@Alt?5Down?$AA@ 004510ec     ClientConnection.obj
 0002:000000f8       ??_C@_07JICO@Ctrl?5Up?$AA@ 004510f8     ClientConnection.obj
 0002:00000104       ??_C@_09JIPL@Ctrl?5Down?$AA@ 00451104     ClientConnection.obj
 0002:00000110       ??_C@_0BB@DGEO@Send?5Ctl?9Alt?9Del?$AA@ 00451110     ClientConnection.obj
 0002:00000124       ??_C@_0N@LCLK@?$CGFull?5screen?$AA@ 00451124     ClientConnection.obj
 0002:00000134       ??_C@_0BI@PINC@Request?5screen?5?$CGrefresh?$AA@ 00451134     ClientConnection.obj
 0002:00000150       ??_C@_0BB@PGON@Connection?5?$CGinfo?$AA@ 00451150     ClientConnection.obj
 0002:00000164       ??_C@_0BH@PPMK@Connection?5?$CGoptions?4?4?4?$AA@ 00451164     ClientConnection.obj
 0002:00000180       ??_C@_0DB@MDPF@Palette?9based?5display?5?9?5?$CFd?5entri@ 00451180     ClientConnection.obj
 0002:000001bc       ??_C@_09GOMH@VNCviewer?$AA@ 004511bc     ClientConnection.obj
 0002:000001c8       ??_C@_0P@MAMH@User?5Cancelled?$AA@ 004511c8     ClientConnection.obj
 0002:000001dc       ??_7QuietException@@6B@    004511dc     ClientConnection.obj
 0002:000001e8       ??_7Exception@@6B@         004511e8     ClientConnection.obj
 0002:000001f4       ??_C@_0BJ@KCOG@Connected?5to?5?$CFs?5port?5?$CFd?6?$AA@ 004511f4     ClientConnection.obj
 0002:00000214       ??_C@_0BM@PFHD@Failed?5to?5connect?5to?5server?$AA@ 00451214     ClientConnection.obj
 0002:00000238       ??_C@_0EF@BHPE@Failed?5to?5get?5server?5address?4?6?$AND@ 00451238     ClientConnection.obj
 0002:0000028c       ??_C@_0BG@FKAK@Error?5creating?5socket?$AA@ 0045128c     ClientConnection.obj
 0002:000002a8       ??_7WarningException@@6B@  004512a8     ClientConnection.obj
 0002:000002b4       ??_C@_0CC@FLED@Error?5disabling?5Nagle?8s?5algorith@ 004512b4     ClientConnection.obj
 0002:000002dc       ??_C@_0DH@EKOD@Connected?5to?5RFB?5server?0?5using?5p@ 004512dc     ClientConnection.obj
 0002:00000320       ??_C@_0BP@BMKL@Can?8t?5use?5IDEA?5authentication?6?$AA@ 00451320     ClientConnection.obj
 0002:00000348       ??_C@_0CM@IKPM@RFB?5server?5supports?5protocol?5ver@ 00451348     ClientConnection.obj
 0002:0000037c       ??_C@_0BB@NFD@Invalid?5protocol?$AA@ 0045137c     ClientConnection.obj
 0002:00000390       ??_C@_0P@KEED@RFB?5?$CF03d?4?$CF03d?6?$AA@ 00451390     ClientConnection.obj
 0002:000003a4       ??_C@_0CE@MNA@Error?5reading?5protocol?5version?3?5@ 004513a4     ClientConnection.obj
 0002:000003d0       ??_C@_0BP@HHDB@Unknown?5authentication?5scheme?$CB?$AA@ 004513d0     ClientConnection.obj
 0002:000003f8       ??_C@_0DD@NBHF@Unknown?5authentication?5scheme?5fr@ 004513f8     ClientConnection.obj
 0002:00000438       ??_C@_0CD@NBKC@Unknown?5VNC?5authentication?5resul@ 00451438     ClientConnection.obj
 0002:00000464       ??_C@_0CH@KEON@Unknown?5VNC?5authentication?5resul@ 00451464     ClientConnection.obj
 0002:00000494       ??_C@_0CM@FFF@VNC?5authentication?5failed?5?9?5too?5@ 00451494     ClientConnection.obj
 0002:000004c8       ??_C@_0BL@PDDO@VNC?5authentication?5failed?$CB?$AA@ 004514c8     ClientConnection.obj
 0002:000004e8       ??_C@_0BO@JDGC@VNC?5authentication?5succeeded?6?$AA@ 004514e8     ClientConnection.obj
 0002:0000050c       ??_C@_0P@KGPO@Empty?5password?$AA@ 0045150c     ClientConnection.obj
 0002:00000520       ??_C@_0BK@NKCI@Password?5had?5zero?5length?6?$AA@ 00451520     ClientConnection.obj
 0002:00000540       ??_C@_03IBNE@Psw?$AA@      00451540     ClientConnection.obj
 0002:00000544       ??_C@_0BH@EON@Software?2ORL?2VNCviewer?$AA@ 00451544     ClientConnection.obj
 0002:00000560       ??_C@_0CI@CLKJ@Can?8t?5use?5IDEA?5authentication?5an@ 00451560     ClientConnection.obj
 0002:00000590       ??_C@_0FH@HGAD@Sorry?5?9?5this?5server?5uses?5an?5olde@ 00451590     ClientConnection.obj
 0002:000005f8       ??_C@_0BH@HKCE@Protocol?5Version?5error?$AA@ 004515f8     ClientConnection.obj
 0002:00000614       ??_C@_0BK@OLN@No?5authentication?5needed?6?$AA@ 00451614     ClientConnection.obj
 0002:00000634       ??_C@_0CD@BDDP@RFB?5connection?5failed?0?5reason?3?5?$CF@ 00451634     ClientConnection.obj
 0002:00000660       ??_7ErrorException@@6B@    00451660     ClientConnection.obj
 0002:0000066c       ??_C@_0BL@JKHA@Geometry?5?$CFd?5x?5?$CFd?5depth?5?$CFd?6?$AA@ 0045166c     ClientConnection.obj
 0002:0000068c       ??_C@_0BD@LPM@Desktop?5name?5?$CC?$CFs?$CC?6?$AA@ 0045168c     ClientConnection.obj
 0002:000006a4       ??_C@_0BN@BBNE@Screen?5work?5area?5is?5?$CFd?5x?5?$CFd?6?$AA@ 004516a4     ClientConnection.obj
 0002:000006c8       ??_C@_0CF@GEJN@Please?5wait?5?9?5initial?5screen?5loa@ 004516c8     ClientConnection.obj
 0002:000006f4       ??_C@_0CG@MJJB@Error?5creating?5local?5image?5of?5sc@ 004516f4     ClientConnection.obj
 0002:00000724       ??_C@_0DB@JOD@Memory?5DC?5has?5depth?5of?5?$CFd?5and?5?$CFs@ 00451724     ClientConnection.obj
 0002:00000760       ??_C@_06EFGN@is?5not?$AA@  00451760     ClientConnection.obj
 0002:00000768       ??_C@_02HNOA@is?$AA@       00451768     ClientConnection.obj
 0002:0000076c       ??_C@_0BO@JHHG@Requesting?516?9bit?5truecolour?6?$AA@ 0045176c     ClientConnection.obj
 0002:00000790       ??_C@_0BN@OMFB@Requesting?58?9bit?5truecolour?6?$AA@ 00451790     ClientConnection.obj
 0002:000007b4       ??_C@_0BP@NFEE@Are?5you?5sure?5you?5want?5to?5exit?$DP?$AA@ 004517b4     ClientConnection.obj
 0002:000007dc       ??_C@_0BC@BDCK@Closing?5VNCviewer?$AA@ 004517dc     ClientConnection.obj
 0002:000007f4       ??_C@_0CF@OOFP@Losing?5focus?5?9?5cancelling?5modifi@ 004517f4     ClientConnection.obj
 0002:00000820       ??_C@_0CP@KKFB@Failed?5to?5create?5timer?5for?5emula@ 00451820     ClientConnection.obj
 0002:00000858       ??_C@_0BF@MFIE@fake?5L?5Ctrl?5pressed?6?$AA@ 00451858     ClientConnection.obj
 0002:00000874       ??_C@_0BE@LPDE@fake?5L?5Alt?5pressed?6?$AA@ 00451874     ClientConnection.obj
 0002:0000088c       ??_C@_0BF@HFEC@fake?5R?5Ctrl?5pressed?6?$AA@ 0045188c     ClientConnection.obj
 0002:000008a8       ??_C@_0BE@HJEO@fake?5R?5Alt?5pressed?6?$AA@ 004518a8     ClientConnection.obj
 0002:000008c0       ??_C@_0BH@EEMM@Sent?5keysym?5?$CF04x?5?$CI?$CFs?$CJ?6?$AA@ 004518c0     ClientConnection.obj
 0002:000008dc       ??_C@_07FCDP@release?$AA@  004518dc     ClientConnection.obj
 0002:000008e8       ??_C@_05LMJC@press?$AA@    004518e8     ClientConnection.obj
 0002:000008f0       ??_C@_0BD@GHJH@fake?5R?5Alt?5raised?6?$AA@ 004518f0     ClientConnection.obj
 0002:00000908       ??_C@_0BE@GLAH@fake?5R?5Ctrl?5raised?6?$AA@ 00451908     ClientConnection.obj
 0002:00000920       ??_C@_0BD@BNEK@fake?5L?5Alt?5raised?6?$AA@ 00451920     ClientConnection.obj
 0002:00000938       ??_C@_0BE@KNHN@fake?5L?5Ctrl?5raised?6?$AA@ 00451938     ClientConnection.obj
 0002:00000950       ??_C@_0CB@LGPL@Process?5key?3?5?$CFs?5?$CIkeyData?5?$CF04x?$CJ?3?5@ 00451950     ClientConnection.obj
 0002:00000978       ??_C@_0CH@EEGE@SendKeyEvent?3?5key?5?$DN?5x?$CF04x?5status@ 00451978     ClientConnection.obj
 0002:000009a8       ??_C@_02HAO@up?$AA@        004519a8     ClientConnection.obj
 0002:000009ac       ??_C@_04KKMF@down?$AA@     004519ac     ClientConnection.obj
 0002:000009b4       ??_C@_0BM@OMDB@Sent?5?$CFd?5bytes?5of?5clipboard?6?$AA@ 004519b4     ClientConnection.obj
 0002:000009d8       ??_C@_0P@OOLN@Blit?5error?5?$CFd?6?$AA@ 004519d8     ClientConnection.obj
 0002:000009ec       ??_C@_0BE@FHLH@VNC?5connection?5info?$AA@ 004519ec     ClientConnection.obj
 0002:00000a04       ??_C@_0JI@OCPB@Connected?5to?3?5?$CFs?3?6?$ANHost?3?5?$CFs?5port@ 00451a04     ClientConnection.obj
 0002:00000abc       ??_C@_0CE@OIAC@Update?9processing?5thread?5finishi@ 00451abc     ClientConnection.obj
 0002:00000ae8       ??_C@_0CC@MAEB@Unhandled?5message?5type?5received?$CB@ 00451ae8     ClientConnection.obj
 0002:00000b10       ??_C@_0BM@ONNK@Unknown?5message?5type?5x?$CF02x?6?$AA@ 00451b10     ClientConnection.obj
 0002:00000b34       ??_C@_0CO@CECF@Unhandled?5SetColormap?5message?5ty@ 00451b34     ClientConnection.obj
 0002:00000b6c       ??_C@_0CP@EHPI@rfbSetColourMapEntries?5read?5but?5@ 00451b6c     ClientConnection.obj
 0002:00000ba4       ??_C@_0CH@LOLC@Error?5while?5waiting?5for?5server?5m@ 00451ba4     ClientConnection.obj
 0002:00000bd4       ??_C@_0CC@LLPM@Socket?5error?5reading?5message?3?5?$CFd@ 00451bd4     ClientConnection.obj
 0002:00000bfc       ??_C@_0N@HODA@SocketClosed?$AA@ 00451bfc     ClientConnection.obj
 0002:00000c0c       ??_C@_0P@GLHK@Socket?5closed?6?$AA@ 00451c0c     ClientConnection.obj
 0002:00000c20       ??_C@_0CC@HAGC@Update?9processing?5thread?5started@ 00451c20     ClientConnection.obj
 0002:00000c48       ??_C@_0BD@CLDJ@Request?5?$CFs?5update?6?$AA@ 00451c48     ClientConnection.obj
 0002:00000c60       ??_C@_04EELP@full?$AA@     00451c60     ClientConnection.obj
 0002:00000c68       ??_C@_0M@CCLI@incremental?$AA@ 00451c68     ClientConnection.obj
 0002:00000c78       ??_C@_0BN@LAND@Requesting?5new?5pixel?5format?6?$AA@ 00451c78     ClientConnection.obj
 0002:00000c9c       ??_C@_0CG@MKLP@Unknown?5encoding?5?$CFd?5?9?5not?5suppor@ 00451c9c     ClientConnection.obj
 0002:00000ccc       ??_C@_0BB@BPFP@?$CFs?5dormant?5mode?6?$AA@ 00451ccc     ClientConnection.obj
 0002:00000ce0       ??_C@_07LHCK@Leaving?$AA@  00451ce0     ClientConnection.obj
 0002:00000cec       ??_C@_08IBPL@Entering?$AA@ 00451cec     ClientConnection.obj
 0002:00000cf8       ??_C@_0BO@PAHH@Read?5remote?5clipboard?5change?6?$AA@ 00451cf8     ClientConnection.obj
 0002:00000d1c       ??_C@_06PCOG@Bell?$CB?6?$AA@ 00451d1c     ClientConnection.obj
 0002:00000d24       ??_C@_0O@FDIC@VNCViewerBell?$AA@ 00451d24     ClientConnection.obj
 0002:00000d34       ??_C@_0CH@CKMF@ReadExact?3?5Socket?5error?5while?5re@ 00451d34     ClientConnection.obj
 0002:00000d64       ??_C@_0BP@CNJA@Socket?5error?5while?5reading?5?$CFd?6?$AA@ 00451d64     ClientConnection.obj
 0002:00000d8c       ??_C@_0BD@MCJ@Connection?5closed?4?$AA@ 00451d8c     ClientConnection.obj
 0002:00000da4       ??_C@_0BE@JDB@?5?5reading?5?$CFd?5bytes?6?$AA@ 00451da4     ClientConnection.obj
 0002:00000dbc       ??_C@_0BH@EDMG@Read?5a?5?$CFd?9byte?5string?6?$AA@ 00451dbc     ClientConnection.obj
 0002:00000dd8       ??_C@_0CI@ENOK@WriteExact?3?5Socket?5error?5while?5w@ 00451dd8     ClientConnection.obj
 0002:00000e08       ??_C@_0BF@GDOM@Socket?5error?5?$CFd?3?5?$CFs?6?$AA@ 00451e08     ClientConnection.obj
 0002:00000e24       ??_C@_0BE@MEOE@?5?5writing?5?$CFd?5bytes?6?$AA@ 00451e24     ClientConnection.obj
 0002:00000e3c       ??_C@_0BI@OJJJ@bufsize?5expanded?5to?5?$CFd?6?$AA@ 00451e3c     ClientConnection.obj
 0002:00000e58       ??_C@_0DA@KKJB@Insufficient?5memory?5to?5allocate?5@ 00451e58     ClientConnection.obj
 0002:00000e94       ??_C@_0CN@JLHC@Exception?5while?5sending?5clipboar@ 00451e94     ClientConnectionClipboard.obj
 0002:00000ecc       ??_C@_0BP@FEOC@Don?8t?5send?5initial?5clipboard?$CB?6?$AA@ 00451ecc     ClientConnectionClipboard.obj
 0002:00000ef4       ??_C@_0BJ@BOIJ@We?5changed?5it?5?9?5ignore?$CB?6?$AA@ 00451ef4     ClientConnectionClipboard.obj
 0002:00000f14       ??_C@_0BD@OMOO@Clipboard?5changed?6?$AA@ 00451f14     ClientConnectionClipboard.obj
 0002:00000f2c       ??_C@_0BL@DOGP@Failed?5to?5close?5clipboard?6?$AA@ 00451f2c     ClientConnectionClipboard.obj
 0002:00000f4c       ??_C@_0BL@OODM@Failed?5to?5empty?5clipboard?6?$AA@ 00451f4c     ClientConnectionClipboard.obj
 0002:00000f6c       ??_C@_0BK@BEMC@Failed?5to?5open?5clipboard?6?$AA@ 00451f6c     ClientConnectionClipboard.obj
 0002:00000f8c       ??_C@_0CN@KALO@Error?5in?5blit?5in?5ClientConnectio@ 00451f8c     ClientConnectionCopyRect.obj
 0002:00000fc4       ??_C@_03LPKH@vnc?$AA@      00451fc4     ClientConnectionFile.obj
 0002:00000fc8       ??_C@_08NPHI@password?$AA@ 00451fc8     ClientConnectionFile.obj
 0002:00000fd4       ??_C@_04OBKB@?$CF02x?$AA@  00451fd4     ClientConnectionFile.obj
 0002:00000fdc       ??_C@_0KJ@JPHD@Do?5you?5want?5to?5save?5the?5password@ 00451fdc     ClientConnectionFile.obj
 0002:000010a8       ??_C@_0BB@JPLH@Security?5warning?$AA@ 004520a8     ClientConnectionFile.obj
 0002:000010bc       ??_C@_04IOEK@port?$AA@     004520bc     ClientConnectionFile.obj
 0002:000010c4       ??_C@_02MECO@?$CFd?$AA@    004520c4     ClientConnectionFile.obj
 0002:000010c8       ??_C@_0L@DLBA@connection?$AA@ 004520c8     ClientConnectionFile.obj
 0002:000010d8       ??_C@_04OHFB@host?$AA@     004520d8     ClientConnectionFile.obj
 0002:000010e0       ??_C@_0O@MJGN@Saving?5to?5?$CFs?6?$AA@ 004520e0     ClientConnectionFile.obj
 0002:000010f0       ??_C@_0BP@GFOK@Error?5?$CFd?5from?5GetSaveFileName?6?$AA@ 004520f0     ClientConnectionFile.obj
 0002:00001118       ??_C@_0BC@GKLE@Error?5saving?5file?$AA@ 00452118     ClientConnectionFile.obj
 0002:00001130       ??_C@_0BB@JPIB@Invalid?5filename?$AA@ 00452130     ClientConnectionFile.obj
 0002:00001144       ??_C@_0N@IHHO@?$CF?410s?9?$CFd?4vnc?$AA@ 00452144     ClientConnectionFile.obj
 0002:00001154       ??_C@_0BI@GHNP@Saving?5connection?5info?6?$AA@ 00452154     ClientConnectionFile.obj
 0002:00001170       ??_C@_03MANP@?$CF2x?$AA@   00452170     ClientConnectionFile.obj
 0002:00001174       ??_C@_0CE@IIFK@Error?5reading?5port?5number?5from?5f@ 00452174     ClientConnectionFile.obj
 0002:000011a0       ??_C@_0CC@FFF@Error?5reading?5host?5name?5from?5fil@ 004521a0     ClientConnectionFile.obj
 0002:000011c8       ??_C@_0BC@OP@Config?5file?5error?$AA@ 004521c8     ClientConnectionFile.obj
 0002:000011e0       ??_C@_00A@?$AA@            004521e0     ClientConnectionFile.obj
 0002:000011e4       ??_C@_0HF@GONJ@To?5exit?5from?5full?9screen?5mode?0?5u@ 004521e4     ClientConnectionFullScreen.obj
 0002:00001270       ??_C@_0BL@LBBI@VNCviewer?5full?9screen?5mode?$AA@ 00452270     ClientConnectionFullScreen.obj
 0002:00001290       ??_C@_0BF@NAIK@SkipFullScreenPrompt?$AA@ 00452290     ClientConnectionFullScreen.obj
 0002:000012ac       ??_C@_0CA@JIDA@Software?2ORL?2VNCviewer?2Settings?$AA@ 004522ac     ClientConnectionFullScreen.obj
 0002:000012d4       ??_C@_0CG@BMKM@Invalid?5number?5of?5bits?5per?5pixel@ 004522d4     ClientConnectionRaw.obj
 0002:00001304       ??_C@_0BK@KODL@Error?5when?5Daemon?5listens?$AA@ 00452304     Daemon.obj
 0002:00001324       ??_C@_0BM@JHCL@Error?5binding?5Daemon?5socket?$AA@ 00452324     Daemon.obj
 0002:00001348       ??_C@_0BN@BNEE@Error?5creating?5Daemon?5socket?$AA@ 00452348     Daemon.obj
 0002:0000136c       ??_C@_0BB@HMEH@VNCviewer?5Daemon?$AA@ 0045236c     Daemon.obj
 0002:00001380       ??_7Daemon@@6B@            00452380     Daemon.obj
 0002:00001384       ??_C@_0BC@BKGH@Adding?5tray?5icon?6?$AA@ 00452384     Daemon.obj
 0002:0000139c       ??_C@_0CE@EEFA@Tray?5icon?5not?5there?5?9?5reinstalli@ 0045239c     Daemon.obj
 0002:000013c8       ??_C@_0BE@BIJI@Checking?5tray?5icon?6?$AA@ 004523c8     Daemon.obj
 0002:000013e0       ??_C@_0BE@OMLC@Deleting?5tray?5icon?6?$AA@ 004523e0     Daemon.obj
 0002:000013f8       ??_C@_0BE@KHGJ@No?5systray?5submenu?6?$AA@ 004523f8     Daemon.obj
 0002:00001410       ??_C@_0BK@CPNI@Daemon?5connection?5closed?6?$AA@ 00452410     Daemon.obj
 0002:00001430       ??_C@_0BE@IIOH@HIWORD?$CIlParam?$CJ?5?$DN?$DN?50?$AA@ 00452430     Daemon.obj
 0002:00001448       ??_C@_0EL@DJJA@i?3?2sysinstall?2vnc?2vnc?93_3_3r7_x8@ 00452448     Daemon.obj
 0002:000014a4       ??_C@_0N@MOIP@info?5?$CB?$DN?5NULL?$AA@ 004524a4     Exception.obj
 0002:000014b4       ??_C@_0EO@EJKJ@I?3?2SysInstall?2Vnc?2vnc?93_3_3r7_x8@ 004524b4     Exception.obj
 0002:00001514       ??_C@_05NAGO@false?$AA@    00452514     Exception.obj
 0002:0000151c       ??_C@_0O@OMLC@Warning?5?3?5?$CFs?6?$AA@ 0045251c     Exception.obj
 0002:0000152c       ??_C@_08GJJN@VNC?5info?$AA@ 0045252c     Exception.obj
 0002:00001538       ??_C@_0CD@HEPI@Error?5when?5Flasher?5tries?5to?5list@ 00452538     Flasher.obj
 0002:00001564       ??_C@_0BN@PDKC@Error?5binding?5Flasher?5socket?$AA@ 00452564     Flasher.obj
 0002:00001588       ??_C@_0BO@FKCI@Error?5creating?5Flasher?5socket?$AA@ 00452588     Flasher.obj
 0002:000015ac       ??_C@_0CA@NMJK@FAILED?5TO?5SELECT?5FLASHER?5FONT?$CB?6?$AA@ 004525ac     Flasher.obj
 0002:000015d4       ??_C@_0BC@CGAK@VNCviewer?5Flasher?$AA@ 004525d4     Flasher.obj
 0002:000015ec       ??_7Flasher@@6B@           004525ec     Flasher.obj
 0002:000015f0       ??_C@_0BL@JJKG@Flasher?5connection?5closed?6?$AA@ 004525f0     Flasher.obj
 0002:00001610       ??_C@_0BA@CBPH@Flash?5for?5?8?$CFs?8?6?$AA@ 00452610     Flasher.obj
 0002:00001624       ??_C@_08GBPE@res?5?$DN?$DN?50?$AA@ 00452624     Flasher.obj
 0002:00001630       ??_C@_0EM@COCG@I?3?2SysInstall?2Vnc?2vnc?93_3_3r7_x8@ 00452630     Flasher.obj
 0002:0000168c       ??_C@_0N@HKMB@Screen?9saver?$AA@ 0045268c     Flasher.obj
 0002:0000169c       ??_C@_0BI@ILAB@WindowsScreenSaverClass?$AA@ 0045269c     Flasher.obj
 0002:00001974       ??_C@_0CM@PAFK@ToAscii?5?$CIwithout?5ctrl?$CJ?5returns?5?$CF@ 00452974     KeyMap.obj
 0002:000019a8       ??_C@_01BJG@?6?$AA@        004529a8     KeyMap.obj
 0002:000019ac       ??_C@_0L@GGJM@?$CF02x?5?$CI?$CFc?$CJ?5?$AA@ 004529ac     KeyMap.obj
 0002:000019bc       ??_C@_0ED@BFLB@Ctrl?9Alt?5pressed?3?5ToAscii?5?$CIwitho@ 004529bc     KeyMap.obj
 0002:00001a0c       ??_C@_0BI@DHEO@not?5in?5special?5keymap?0?5?$AA@ 00452a0c     KeyMap.obj
 0002:00001a28       ??_C@_0BG@LPJH@keymap?5gives?5?$CFu?5?$CI?$CFx?$CJ?5?$AA@ 00452a28     KeyMap.obj
 0002:00001a44       ??_C@_0N@MGCC@?5?$CIextended?$CJ?5?$AA@ 00452a44     KeyMap.obj
 0002:00001a54       ??_C@_0P@GIEG@?5keyData?5?$CF04x?5?$AA@ 00452a54     KeyMap.obj
 0002:00001a68       ?ToDebug@Log@@2HB          00452a68     Log.obj
 0002:00001a6c       ?ToFile@Log@@2HB           00452a6c     Log.obj
 0002:00001a70       ?ToConsole@Log@@2HB        00452a70     Log.obj
 0002:00001a78       ??_7Log@@6B@               00452a78     Log.obj
 0002:00001a7c       ??_C@_0BL@LLBC@Error?5opening?5log?5file?5?$CFs?6?$AA@ 00452a7c     Log.obj
 0002:00001a9c       ??_C@_05BBHA@index?$AA@    00452a9c     MRU.obj
 0002:00001aa4       ??_7MRU@@6B@               00452aa4     MRU.obj
 0002:00001aa8       ??_C@_0BL@FEIO@Software?2ORL?2VNCviewer?2MRU?$AA@ 00452aa8     SessionDialog.obj
 0002:00001ac8       ??_7SessionDialog@@6B@     00452ac8     SessionDialog.obj
 0002:00001acc       ??_C@_0EK@HIBH@Invalid?5VNC?5server?5specified?4?6?$ANS@ 00452acc     SessionDialog.obj
 0002:00001b24       ??_C@_0BB@IOAN@Connection?5setup?$AA@ 00452b24     SessionDialog.obj
 0002:00001b38       ??_7VNCOptions@@6B@        00452b38     VNCOptions.obj
 0002:00001b3c       ??_C@_0DB@NFPF@Invalid?5scale?5factor?5?9?5resetting@ 00452b3c     VNCOptions.obj
 0002:00001b78       ??_C@_0P@DNAD@Argument?5error?$AA@ 00452b78     VNCOptions.obj
 0002:00001b8c       ??_C@_0BO@DJNG@Invalid?5VNC?5server?5specified?4?$AA@ 00452b8c     VNCOptions.obj
 0002:00001bb0       ??_C@_08DFJG@register?$AA@ 00452bb0     VNCOptions.obj
 0002:00001bbc       ??_C@_0CO@CNCN@Can?8t?5open?5specified?5config?5file@ 00452bbc     VNCOptions.obj
 0002:00001bf4       ??_C@_0BJ@IPOC@No?5config?5file?5specified?$AA@ 00452bf4     VNCOptions.obj
 0002:00001c14       ??_C@_06FALM@config?$AA@   00452c14     VNCOptions.obj
 0002:00001c1c       ??_C@_0BK@FKKB@Invalid?5logfile?5specified?$AA@ 00452c1c     VNCOptions.obj
 0002:00001c3c       ??_C@_02DILL@?$CFs?$AA@    00452c3c     VNCOptions.obj
 0002:00001c40       ??_C@_0BF@PG@No?5logfile?5specified?$AA@ 00452c40     VNCOptions.obj
 0002:00001c5c       ??_C@_07OFK@logfile?$AA@   00452c5c     VNCOptions.obj
 0002:00001c68       ??_C@_07BLFM@console?$AA@  00452c68     VNCOptions.obj
 0002:00001c74       ??_C@_0BL@BHKD@Invalid?5loglevel?5specified?$AA@ 00452c74     VNCOptions.obj
 0002:00001c94       ??_C@_0BG@PCPJ@No?5loglevel?5specified?$AA@ 00452c94     VNCOptions.obj
 0002:00001cb0       ??_C@_08GDIA@loglevel?$AA@ 00452cb0     VNCOptions.obj
 0002:00001cbc       ??_C@_0BI@IPKF@Invalid?5delay?5specified?$AA@ 00452cbc     VNCOptions.obj
 0002:00001cd8       ??_C@_0BD@OCGF@No?5delay?5specified?$AA@ 00452cd8     VNCOptions.obj
 0002:00001cf0       ??_C@_05BFAE@delay?$AA@    00452cf0     VNCOptions.obj
 0002:00001cf8       ??_C@_0BB@FKMK@disableclipboard?$AA@ 00452cf8     VNCOptions.obj
 0002:00001d0c       ??_C@_0BH@NBOH@Invalid?5fuzz?5specified?$AA@ 00452d0c     VNCOptions.obj
 0002:00001d28       ??_C@_0BC@BBPE@No?5fuzz?5specified?$AA@ 00452d28     VNCOptions.obj
 0002:00001d40       ??_C@_0N@OLPA@emulate3fuzz?$AA@ 00452d40     VNCOptions.obj
 0002:00001d50       ??_C@_0BK@HEIE@Invalid?5timeout?5specified?$AA@ 00452d50     VNCOptions.obj
 0002:00001d70       ??_C@_0BF@COND@No?5timeout?5specified?$AA@ 00452d70     VNCOptions.obj
 0002:00001d8c       ??_C@_0BA@BIHK@emulate3timeout?$AA@ 00452d8c     VNCOptions.obj
 0002:00001da0       ??_C@_0BK@DPGL@Invalid?5scaling?5specified?$AA@ 00452da0     VNCOptions.obj
 0002:00001dc0       ??_C@_05OHLK@?$CFd?1?$CFd?$AA@ 00452dc0     VNCOptions.obj
 0002:00001dc8       ??_C@_0BM@MEID@No?5scaling?5factor?5specified?$AA@ 00452dc8     VNCOptions.obj
 0002:00001dec       ??_C@_05IMHO@scale?$AA@    00452dec     VNCOptions.obj
 0002:00001df4       ??_C@_0L@KKMI@noemulate3?$AA@ 00452df4     VNCOptions.obj
 0002:00001e04       ??_C@_08HKDL@emulate3?$AA@ 00452e04     VNCOptions.obj
 0002:00001e10       ??_C@_0O@LNNN@belldeiconify?$AA@ 00452e10     VNCOptions.obj
 0002:00001e20       ??_C@_0N@PNDA@normalcursor?$AA@ 00452e20     VNCOptions.obj
 0002:00001e30       ??_C@_09FNCG@dotcursor?$AA@ 00452e30     VNCOptions.obj
 0002:00001e3c       ??_C@_08CJGP@nocursor?$AA@ 00452e3c     VNCOptions.obj
 0002:00001e48       ??_C@_09DFNL@swapmouse?$AA@ 00452e48     VNCOptions.obj
 0002:00001e54       ??_C@_06MDBN@shared?$AA@   00452e54     VNCOptions.obj
 0002:00001e5c       ??_C@_04JOKE@8bit?$AA@     00452e5c     VNCOptions.obj
 0002:00001e64       ??_C@_0L@EMDO@fullscreen?$AA@ 00452e64     VNCOptions.obj
 0002:00001e74       ??_C@_08MEMD@viewonly?$AA@ 00452e74     VNCOptions.obj
 0002:00001e80       ??_C@_0L@NLGL@restricted?$AA@ 00452e80     VNCOptions.obj
 0002:00001e90       ??_C@_06IODP@listen?$AA@   00452e90     VNCOptions.obj
 0002:00001e98       ??_C@_01KDJI@h?$AA@        00452e98     VNCOptions.obj
 0002:00001e9c       ??_C@_01PKMN@?$DP?$AA@     00452e9c     VNCOptions.obj
 0002:00001ea0       ??_C@_04MHDN@help?$AA@     00452ea0     VNCOptions.obj
 0002:00001ea8       ??_C@_07MHLD@options?$AA@  00452ea8     VNCOptions.obj
 0002:00001eb4       ??_C@_09NGJ@scale_den?$AA@ 00452eb4     VNCOptions.obj
 0002:00001ec0       ??_C@_09KMOB@scale_num?$AA@ 00452ec0     VNCOptions.obj
 0002:00001ecc       ??_C@_0M@KLHF@localcursor?$AA@ 00452ecc     VNCOptions.obj
 0002:00001edc       ??_C@_0BD@ILKB@preferred_encoding?$AA@ 00452edc     VNCOptions.obj
 0002:00001ef4       ??_C@_0BA@CMPA@use_encoding_?$CFd?$AA@ 00452ef4     VNCOptions.obj
 0002:00001f08       ??_C@_0EC@GPGI@Software?2Microsoft?2Windows?2Curre@ 00452f08     VNCOptions.obj
 0002:00001f58       ??_C@_0BD@INEB@?$CC?$CFs?$CC?5?9config?5?$CC?$CF?$CF1?$CC?$AA@ 00452f58     VNCOptions.obj
 0002:00001f70       ??_C@_0BD@GFLJ@Shell?2open?2command?$AA@ 00452f70     VNCOptions.obj
 0002:00001f88       ??_C@_04MLEK@?$CFs?00?$AA@ 00452f88     VNCOptions.obj
 0002:00001f90       ??_C@_0M@JONA@DefaultIcon?$AA@ 00452f90     VNCOptions.obj
 0002:00001fa0       ??_C@_0BG@NNKJ@VNCviewer?5Config?5File?$AA@ 00452fa0     VNCOptions.obj
 0002:00001fbc       ??_C@_0O@IOBJ@Viewer?5is?5?$CFs?6?$AA@ 00452fbc     VNCOptions.obj
 0002:00001fcc       ??_C@_0CC@BAAP@Error?5getting?5vncviewer?5filename@ 00452fcc     VNCOptions.obj
 0002:00001ff4       ??_C@_0CD@CCBP@Failed?5to?5register?5?4vnc?5extensio@ 00452ff4     VNCOptions.obj
 0002:00002020       ??_C@_0BB@BPKA@VncViewer?4Config?$AA@ 00453020     VNCOptions.obj
 0002:00002034       ??_C@_04OAJJ@?4vnc?$AA@    00453034     VNCOptions.obj
 0002:0000203c       ??_C@_09INGB@VNC?5error?$AA@ 0045303c     VNCOptions.obj
 0002:00002048       ??_C@_0OJ@HAJE@?$CFs?6?$ANUsage?5includes?3?6?$AN?5?5vncviewer@ 00453048     VNCOptions.obj
 0002:00002160       ??_C@_08LHAE@Exiting?6?$AA@ 00453160     vncviewer.obj
 0002:0000216c       ??_C@_0CI@IPJG@Started?5and?5Winsock?5?$CIv?5?$CFd?$CJ?5initi@ 0045316c     VNCviewerApp.obj
 0002:0000219c       ??_C@_0CD@CBK@Error?5initialising?5sockets?5libra@ 0045319c     VNCviewerApp.obj
 0002:000021c8       ??_7VNCviewerApp@@6B@      004531c8     VNCviewerApp.obj
 0002:000021d8       ??_C@_0BG@OBBM@Client?5list?5overflow?$CB?$AA@ 004531d8     VNCviewerApp.obj
 0002:000021f4       ??_C@_0BH@BPHH@Client?5list?5overflow?$CB?6?$AA@ 004531f4     VNCviewerApp.obj
 0002:00002210       ??_C@_0CA@FMPI@Registered?5connection?5with?5app?6?$AA@ 00453210     VNCviewerApp.obj
 0002:00002238       ??_C@_0CF@CGCL@Client?5not?5found?5for?5deregisteri@ 00453238     VNCviewerApp.obj
 0002:00002264       ??_C@_0CC@OOFC@Deregistered?5connection?5from?5app@ 00453264     VNCviewerApp.obj
 0002:0000228c       ??_C@_0BJ@KFIB@VNC?5viewer?5closing?5down?6?$AA@ 0045328c     VNCviewerApp.obj
 0002:000022ac       ??_C@_0O@KLML@VNCviewerBell?$AA@ 004532ac     VNCviewerApp32.obj
 0002:000022bc       ??_C@_0CB@LLJP@AppEvents?2Schemes?2Apps?2VNCviewer@ 004532bc     VNCviewerApp32.obj
 0002:000022e4       ??_C@_0BA@HMGF@VNCviewer?5error?$AA@ 004532e4     VNCviewerApp32.obj
 0002:000022f8       ??_C@_0CL@IAMI@Error?5creating?5listening?5daemon?3@ 004532f8     VNCviewerApp32.obj
 0002:0000232c       ??_C@_0CO@IOLG@Perhaps?5another?5VNCviewer?5is?5alr@ 0045332c     VNCviewerApp32.obj
 0002:00002364       ??_C@_0CF@PCKE@In?5listening?5mode?5?9?5staring?5daem@ 00453364     VNCviewerApp32.obj
 0002:00002390       ??_C@_0CI@CIPO@Error?5loading?5specified?5keyboard@ 00453390     VNCviewerApp32.obj
 0002:000023c0       ??_7VNCviewerApp32@@6B@    004533c0     VNCviewerApp32.obj
 0002:000023d0       ??_C@_0P@LEHE@?$CFs?2?$CFs?2?4default?$AA@ 004533d0     VNCviewerApp32.obj
 0002:000023e4       ??_C@_08KNNE@ding?4wav?$AA@ 004533e4     VNCviewerApp32.obj
 0002:000023f0       ??_C@_0P@JDLG@?$CFs?2?$CFs?2?4current?$AA@ 004533f0     VNCviewerApp32.obj
 0002:00002404       ??_C@_05KEJO@?$CFs?2?$CFs?$AA@ 00453404     VNCviewerApp32.obj
 0002:0000240c       ??_C@_04FKNP@Bell?$AA@     0045340c     VNCviewerApp32.obj
 0002:00002414       ??_C@_0BJ@JMAH@AppEvents?2EventLabels?2?$CFs?$AA@ 00453414     VNCviewerApp32.obj
 0002:00002434       ??_7_internal_omni_thread_dummy@@6B@ 00453434     omnithread:nt.obj
 0002:00002440       ??_7omni_thread@@6B@       00453440     omnithread:nt.obj
 0002:0000244c       ??_C@_0L@OFGA@dbgdel?4cpp?$AA@ 0045344c     LIBCMTD:dbgdel.obj
 0002:00002458       ??_C@_0CH@PHOC@_BLOCK_TYPE_IS_VALID?$CIpHead?9?$DOnBlo@ 00453458     LIBCMTD:dbgdel.obj
 0002:00002480       ??_C@_0P@LNLA@format?5?$CB?$DN?5NULL?$AA@ 00453480     LIBCMTD:sprintf.obj
 0002:00002490       ??_C@_09NEAG@sprintf?4c?$AA@ 00453490     LIBCMTD:sprintf.obj
 0002:0000249c       ??_C@_0P@OOIN@string?5?$CB?$DN?5NULL?$AA@ 0045349c     LIBCMTD:sprintf.obj
 0002:000024b0       ??_7type_info@@6B@         004534b0     LIBCMTD:typinfo.obj
 0002:000024d8       ??_C@_08EJDA@sscanf?4c?$AA@ 004534d8     LIBCMTD:sscanf.obj
 0002:000024e4       ??_C@_06DPMO@Client?$AA@   004534e4     LIBCMTD:dbgheap.obj
 0002:000024ec       ??_C@_06BAFM@Ignore?$AA@   004534ec     LIBCMTD:dbgheap.obj
 0002:000024f4       ??_C@_03DICE@CRT?$AA@      004534f4     LIBCMTD:dbgheap.obj
 0002:000024f8       ??_C@_06BILL@Normal?$AA@   004534f8     LIBCMTD:dbgheap.obj
 0002:00002500       ??_C@_04NEN@Free?$AA@      00453500     LIBCMTD:dbgheap.obj
 0002:00002514       ??_C@_0DC@CGID@Error?3?5memory?5allocation?3?5bad?5me@ 00453514     LIBCMTD:dbgheap.obj
 0002:00002548       ??_C@_0CE@FMIA@Invalid?5allocation?5size?3?5?$CFu?5byte@ 00453548     LIBCMTD:dbgheap.obj
 0002:0000256c       ??_C@_0CB@CPBI@Client?5hook?5allocation?5failure?4?6@ 0045356c     LIBCMTD:dbgheap.obj
 0002:00002590       ??_C@_0DF@DKHF@Client?5hook?5allocation?5failure?5a@ 00453590     LIBCMTD:dbgheap.obj
 0002:000025c8       ??_C@_09IMJC@dbgheap?4c?$AA@ 004535c8     LIBCMTD:dbgheap.obj
 0002:000025d4       ??_C@_0BC@EPKL@_CrtCheckMemory?$CI?$CJ?$AA@ 004535d4     LIBCMTD:dbgheap.obj
 0002:000025f4       ??_C@_0BK@JDHA@_pFirstBlock?5?$DN?$DN?5pOldBlock?$AA@ 004535f4     LIBCMTD:dbgheap.obj
 0002:00002610       ??_C@_0BJ@NMEF@_pLastBlock?5?$DN?$DN?5pOldBlock?$AA@ 00453610     LIBCMTD:dbgheap.obj
 0002:0000262c       ??_C@_0DC@BOCN@fRealloc?5?$HM?$HM?5?$CI?$CBfRealloc?5?$CG?$CG?5pNewBl@ 0045362c     LIBCMTD:dbgheap.obj
 0002:00002660       ??_C@_0DK@DKOM@_BLOCK_TYPE?$CIpOldBlock?9?$DOnBlockUse@ 00453660     LIBCMTD:dbgheap.obj
 0002:0000269c       ??_C@_0EF@EDKM@pOldBlock?9?$DOnLine?5?$DN?$DN?5IGNORE_LINE?5@ 0045369c     LIBCMTD:dbgheap.obj
 0002:000026e4       ??_C@_0CC@GPMO@_CrtIsValidHeapPointer?$CIpUserData@ 004536e4     LIBCMTD:dbgheap.obj
 0002:00002708       ??_C@_0CN@FHGE@Allocation?5too?5large?5or?5negative@ 00453708     LIBCMTD:dbgheap.obj
 0002:00002738       ??_C@_0CE@EAMN@Client?5hook?5re?9allocation?5failur@ 00453738     LIBCMTD:dbgheap.obj
 0002:0000275c       ??_C@_0DI@KKMM@Client?5hook?5re?9allocation?5failur@ 0045375c     LIBCMTD:dbgheap.obj
 0002:000027b4       ??_C@_0BG@JCEC@_pFirstBlock?5?$DN?$DN?5pHead?$AA@ 004537b4     LIBCMTD:dbgheap.obj
 0002:000027cc       ??_C@_0BF@NLNN@_pLastBlock?5?$DN?$DN?5pHead?$AA@ 004537cc     LIBCMTD:dbgheap.obj
 0002:000027e4       ??_C@_0BO@PLHH@pHead?9?$DOnBlockUse?5?$DN?$DN?5nBlockUse?$AA@ 004537e4     LIBCMTD:dbgheap.obj
 0002:00002804       ??_C@_0DN@KKIO@pHead?9?$DOnLine?5?$DN?$DN?5IGNORE_LINE?5?$CG?$CG?5p@ 00453804     LIBCMTD:dbgheap.obj
 0002:00002844       ??_C@_0CK@OJNB@DAMAGE?3?5after?5?$CFhs?5block?5?$CI?$CD?$CFd?$CJ?5at@ 00453844     LIBCMTD:dbgheap.obj
 0002:00002870       ??_C@_0CL@IJIL@DAMAGE?3?5before?5?$CFhs?5block?5?$CI?$CD?$CFd?$CJ?5a@ 00453870     LIBCMTD:dbgheap.obj
 0002:0000289c       ??_C@_0BL@MBNA@Client?5hook?5free?5failure?4?6?$AA@ 0045389c     LIBCMTD:dbgheap.obj
 0002:000028d4       ??_C@_0DK@EKKL@memory?5check?5error?5at?50x?$CF08X?5?$DN?50@ 004538d4     LIBCMTD:dbgheap.obj
 0002:00002910       ??_C@_0CJ@GCII@?$CFhs?5located?5at?50x?$CF08X?5is?5?$CFu?5byte@ 00453910     LIBCMTD:dbgheap.obj
 0002:0000293c       ??_C@_0CA@EJPI@?$CFhs?5allocated?5at?5file?5?$CFhs?$CI?$CFd?$CJ?4?6?$AA@ 0045393c     LIBCMTD:dbgheap.obj
 0002:0000295c       ??_C@_0CJ@LHHG@DAMAGE?3?5on?5top?5of?5Free?5block?5at?5@ 0045395c     LIBCMTD:dbgheap.obj
 0002:00002988       ??_C@_07GJHM@DAMAGED?$AA@  00453988     LIBCMTD:dbgheap.obj
 0002:00002990       ??_C@_0CL@ODIE@_heapchk?5fails?5with?5unknown?5retu@ 00453990     LIBCMTD:dbgheap.obj
 0002:000029bc       ??_C@_0CC@EHNC@_heapchk?5fails?5with?5_HEAPBADPTR?4@ 004539bc     LIBCMTD:dbgheap.obj
 0002:000029e0       ??_C@_0CC@JNDP@_heapchk?5fails?5with?5_HEAPBADEND?4@ 004539e0     LIBCMTD:dbgheap.obj
 0002:00002a04       ??_C@_0CD@DNMG@_heapchk?5fails?5with?5_HEAPBADNODE@ 00453a04     LIBCMTD:dbgheap.obj
 0002:00002a28       ??_C@_0CE@JMCB@_heapchk?5fails?5with?5_HEAPBADBEGI@ 00453a28     LIBCMTD:dbgheap.obj
 0002:00002a7c       ??_C@_0CD@MEMI@Bad?5memory?5block?5found?5at?50x?$CF08X@ 00453a7c     LIBCMTD:dbgheap.obj
 0002:00002aa0       ??_C@_0CI@GMAO@_CrtMemCheckPoint?3?5NULL?5state?5po@ 00453aa0     LIBCMTD:dbgheap.obj
 0002:00002ad4       ??_C@_0CI@MNAE@_CrtMemDifference?3?5NULL?5state?5po@ 00453ad4     LIBCMTD:dbgheap.obj
 0002:00002afc       ??_C@_0BH@PKIJ@Object?5dump?5complete?4?6?$AA@ 00453afc     LIBCMTD:dbgheap.obj
 0002:00002b14       ??_C@_0DB@DBPF@crt?5block?5at?50x?$CF08X?0?5subtype?5?$CFx?0@ 00453b14     LIBCMTD:dbgheap.obj
 0002:00002b48       ??_C@_0CI@JLM@normal?5block?5at?50x?$CF08X?0?5?$CFu?5bytes@ 00453b48     LIBCMTD:dbgheap.obj
 0002:00002b70       ??_C@_0DE@PFEA@client?5block?5at?50x?$CF08X?0?5subtype?5@ 00453b70     LIBCMTD:dbgheap.obj
 0002:00002ba4       ??_C@_06MBCE@?$HL?$CFld?$HN?5?$AA@ 00453ba4     LIBCMTD:dbgheap.obj
 0002:00002bac       ??_C@_0L@BLDJ@?$CFhs?$CI?$CFd?$CJ?5?3?5?$AA@ 00453bac     LIBCMTD:dbgheap.obj
 0002:00002bb8       ??_C@_0BE@FEMA@?$CDFile?5Error?$CD?$CI?$CFd?$CJ?5?3?5?$AA@ 00453bb8     LIBCMTD:dbgheap.obj
 0002:00002bcc       ??_C@_0BE@FPPM@Dumping?5objects?5?9?$DO?6?$AA@ 00453bcc     LIBCMTD:dbgheap.obj
 0002:00002bec       ??_C@_0BA@POLM@?5Data?3?5?$DM?$CFs?$DO?5?$CFs?6?$AA@ 00453bec     LIBCMTD:dbgheap.obj
 0002:00002bfc       ??_C@_05JLAO@?$CF?42X?5?$AA@ 00453bfc     LIBCMTD:dbgheap.obj
 0002:00002c04       ??_C@_0BI@KONA@Detected?5memory?5leaks?$CB?6?$AA@ 00453c04     LIBCMTD:dbgheap.obj
 0002:00002c1c       ??_C@_0BP@LCCN@Total?5allocations?3?5?$CFld?5bytes?4?6?$AA@ 00453c1c     LIBCMTD:dbgheap.obj
 0002:00002c3c       ??_C@_0CB@COID@Largest?5number?5used?3?5?$CFld?5bytes?4?6@ 00453c3c     LIBCMTD:dbgheap.obj
 0002:00002c60       ??_C@_0BO@MEJD@?$CFld?5bytes?5in?5?$CFld?5?$CFhs?5Blocks?4?6?$AA@ 00453c60     LIBCMTD:dbgheap.obj
 0002:00002c80       ??_C@_02JJJH@?6?6?$AA@     00453c80     LIBCMTD:assert.obj
 0002:00002c84       ??_C@_03NAME@?4?4?4?$AA@   00453c84     LIBCMTD:assert.obj
 0002:00002c88       ??_C@_0CF@JPDF@Microsoft?5Visual?5C?$CL?$CL?5Runtime?5Lib@ 00453c88     LIBCMTD:assert.obj
 0002:00002cb0       ??_C@_0DN@MHHJ@?$CIPress?5Retry?5to?5debug?5the?5applic@ 00453cb0     LIBCMTD:assert.obj
 0002:00002cf0       ??_C@_0HA@EJLJ@For?5information?5on?5how?5your?5prog@ 00453cf0     LIBCMTD:assert.obj
 0002:00002d60       ??_C@_0N@NOAB@Expression?3?5?$AA@ 00453d60     LIBCMTD:assert.obj
 0002:00002d70       ??_C@_06JMOL@Line?3?5?$AA@ 00453d70     LIBCMTD:assert.obj
 0002:00002d78       ??_C@_06FAAO@File?3?5?$AA@ 00453d78     LIBCMTD:assert.obj
 0002:00002d80       ??_C@_0BH@NNCD@?$DMprogram?5name?5unknown?$DO?$AA@ 00453d80     LIBCMTD:assert.obj
 0002:00002d98       ??_C@_09PIFG@Program?3?5?$AA@ 00453d98     LIBCMTD:assert.obj
 0002:00002da4       ??_C@_0BC@OIMC@Assertion?5failed?$CB?$AA@ 00453da4     LIBCMTD:assert.obj
 0002:00002db8       ??_C@_0BB@BLL@Assertion?5Failed?$AA@ 00453db8     LIBCMTD:dbgrpt.obj
 0002:00002dcc       ??_C@_05CKBG@Error?$AA@    00453dcc     LIBCMTD:dbgrpt.obj
 0002:00002dd4       ??_C@_07JCGI@Warning?$AA@  00453dd4     LIBCMTD:dbgrpt.obj
 0002:00002ddc       ??_C@_0M@ODEP@?$CFs?$CI?$CFd?$CJ?5?3?5?$CFs?$AA@ 00453ddc     LIBCMTD:dbgrpt.obj
 0002:00002de8       ??_C@_01FEHD@?$AN?$AA@     00453de8     LIBCMTD:dbgrpt.obj
 0002:00002dec       ??_C@_0BD@BEAK@Assertion?5failed?3?5?$AA@ 00453dec     LIBCMTD:dbgrpt.obj
 0002:00002e00       ??_C@_0CL@LCCP@_CrtDbgReport?3?5String?5too?5long?5o@ 00453e00     LIBCMTD:dbgrpt.obj
 0002:00002e2c       ??_C@_0DC@EMDK@Second?5Chance?5Assertion?5Failed?3?5@ 00453e2c     LIBCMTD:dbgrpt.obj
 0002:00002e60       ??_C@_09NJAK@wsprintfA?$AA@ 00453e60     LIBCMTD:dbgrpt.obj
 0002:00002e6c       ??_C@_0L@HKL@user32?4dll?$AA@ 00453e6c     LIBCMTD:dbgrpt.obj
 0002:00002e78       ??_C@_0CD@GCMD@Microsoft?5Visual?5C?$CL?$CL?5Debug?5Libra@ 00453e78     LIBCMTD:dbgrpt.obj
 0002:00002e9c       ??_C@_0FD@EBDD@Debug?5?$CFs?$CB?6?6Program?3?5?$CFs?$CFs?$CFs?$CFs?$CFs?$CFs@ 00453e9c     LIBCMTD:dbgrpt.obj
 0002:00002ef0       ??_C@_09DCKN@?6Module?3?5?$AA@ 00453ef0     LIBCMTD:dbgrpt.obj
 0002:00002efc       ??_C@_07HJII@?6File?3?5?$AA@ 00453efc     LIBCMTD:dbgrpt.obj
 0002:00002f04       ??_C@_07LFGN@?6Line?3?5?$AA@ 00453f04     LIBCMTD:dbgrpt.obj
 0002:00002f0c       ??_C@_0HD@BHFH@?6?6For?5information?5on?5how?5your?5pr@ 00453f0c     LIBCMTD:dbgrpt.obj
 0002:00002f80       ??_C@_08GFHP@dbgrpt?4c?$AA@ 00453f80     LIBCMTD:dbgrpt.obj
 0002:00002f8c       ??_C@_0BG@FBEA@szUserMessage?5?$CB?$DN?5NULL?$AA@ 00453f8c     LIBCMTD:dbgrpt.obj
 0002:00002fa4       ??_C@_0L@HE@vsprintf?4c?$AA@ 00453fa4     LIBCMTD:vsprintf.obj
 0002:00002fb0       ??_C@_08CEA@onexit?4c?$AA@ 00453fb0     LIBCMTD:onexit.obj
 0002:00002fcc       ??_C@_0L@BOLO@threadex?4c?$AA@ 00453fcc     LIBCMTD:threadex.obj
 0002:00002fe4       ??_C@_07PDLA@mlock?4c?$AA@ 00453fe4     LIBCMTD:mlock.obj
 0002:00003034       ??_C@_0L@ENLJ@tidtable?4c?$AA@ 00454034     LIBCMTD:tidtable.obj
 0002:00003070       ??_C@_0DP@IHIN@?$CI?$CCinconsistent?5IOB?5fields?$CC?0?5stre@ 00454070     LIBCMTD:_flsbuf.obj
 0002:000030b0       ??_C@_09LGEI@_flsbuf?4c?$AA@ 004540b0     LIBCMTD:_flsbuf.obj
 0002:000030bc       ??_C@_0M@KJPK@str?5?$CB?$DN?5NULL?$AA@ 004540bc     LIBCMTD:_flsbuf.obj
 0002:000030c8       ___lookuptable             004540c8     LIBCMTD:output.obj
 0002:00003124       ??_C@_1O@POHA@?$AA?$CI?$AAn?$AAu?$AAl?$AAl?$AA?$CJ?$AA?$AA@ 00454124     LIBCMTD:output.obj
 0002:00003134       ??_C@_06ONKE@?$CInull?$CJ?$AA@ 00454134     LIBCMTD:output.obj
 0002:0000313c       ??_C@_08MIHI@output?4c?$AA@ 0045413c     LIBCMTD:output.obj
 0002:00003148       ??_C@_0P@PIHB@ch?5?$CB?$DN?5_T?$CI?8?20?8?$CJ?$AA@ 00454148     LIBCMTD:output.obj
 0002:00003170       ??_C@_0P@FHEA@stream?5?$CB?$DN?5NULL?$AA@ 00454170     LIBCMTD:input.obj
 0002:00003180       ??_C@_07IEFA@input?4c?$AA@ 00454180     LIBCMTD:input.obj
 0002:000031e8       ??_C@_0BH@PHHF@__GLOBAL_HEAP_SELECTED?$AA@ 004541e8     LIBCMTD:heapinit.obj
 0002:00003200       ??_C@_0BF@BBGL@__MSVCRT_HEAP_SELECT?$AA@ 00454200     LIBCMTD:heapinit.obj
 0002:00003218       ??_C@_08CNMA@winsig?4c?$AA@ 00454218     LIBCMTD:winsig.obj
 0002:00003224       ??_C@_0BD@NJFP@GetLastActivePopup?$AA@ 00454224     LIBCMTD:crtmbox.obj
 0002:00003238       ??_C@_0BA@GILI@GetActiveWindow?$AA@ 00454238     LIBCMTD:crtmbox.obj
 0002:00003248       ??_C@_0M@PKCK@MessageBoxA?$AA@ 00454248     LIBCMTD:crtmbox.obj
 0002:00003254       ??_C@_09DLOM@fprintf?4c?$AA@ 00454254     LIBCMTD:fprintf.obj
 0002:00003260       ??_C@_09GCII@setvbuf?4c?$AA@ 00454260     LIBCMTD:setvbuf.obj
 0002:0000326c       ??_C@_07HPAH@_file?4c?$AA@ 0045426c     LIBCMTD:_file.obj
 0002:00003274       ??_C@_07PCLE@LC_TIME?$AA@  00454274     LIBCMTD:setlocal.obj
 0002:0000327c       ??_C@_0L@NKG@LC_NUMERIC?$AA@ 0045427c     LIBCMTD:setlocal.obj
 0002:00003288       ??_C@_0M@CBIH@LC_MONETARY?$AA@ 00454288     LIBCMTD:setlocal.obj
 0002:00003294       ??_C@_08LFGE@LC_CTYPE?$AA@ 00454294     LIBCMTD:setlocal.obj
 0002:000032a0       ??_C@_0L@CFLC@LC_COLLATE?$AA@ 004542a0     LIBCMTD:setlocal.obj
 0002:000032ac       ??_C@_06GCPK@LC_ALL?$AA@   004542ac     LIBCMTD:setlocal.obj
 0002:000032b4       ??_C@_01FAJB@?$DL?$AA@     004542b4     LIBCMTD:setlocal.obj
 0002:000032b8       ??_C@_02BGDO@?$DN?$DL?$AA@ 004542b8     LIBCMTD:setlocal.obj
 0002:000032bc       ??_C@_0L@MOEE@setlocal?4c?$AA@ 004542bc     LIBCMTD:setlocal.obj
 0002:000032c8       ??_C@_01KPOD@?$DN?$AA@     004542c8     LIBCMTD:setlocal.obj
 0002:000032cc       ??_C@_03DBOJ@_?4?0?$AA@    004542cc     LIBCMTD:setlocal.obj
 0002:000032d0       ??_C@_01PJCK@?4?$AA@       004542d0     LIBCMTD:setlocal.obj
 0002:000032d4       ??_C@_01NON@_?$AA@         004542d4     LIBCMTD:setlocal.obj
 0002:000032d8       ??_C@_09IGKD@stdenvp?4c?$AA@ 004542d8     LIBCMTD:stdenvp.obj
 0002:000032e4       ??_C@_09MPMN@stdargv?4c?$AA@ 004542e4     LIBCMTD:stdargv.obj
 0002:000032f0       ??_C@_07BNNE@a_env?4c?$AA@ 004542f0     LIBCMTD:a_env.obj
 0002:000032f8       ??_C@_08KFDJ@ioinit?4c?$AA@ 004542f8     LIBCMTD:ioinit.obj
 0002:00003304       ??_C@_0P@GGKG@runtime?5error?5?$AA@ 00454304     LIBCMTD:crt0msg.obj
 0002:00003314       ??_C@_02PIMC@?$AN?6?$AA@   00454314     LIBCMTD:crt0msg.obj
 0002:00003318       ??_C@_0O@DELO@TLOSS?5error?$AN?6?$AA@ 00454318     LIBCMTD:crt0msg.obj
 0002:00003328       ??_C@_0N@OMLL@SING?5error?$AN?6?$AA@ 00454328     LIBCMTD:crt0msg.obj
 0002:00003338       ??_C@_0P@OJAK@DOMAIN?5error?$AN?6?$AA@ 00454338     LIBCMTD:crt0msg.obj
 0002:00003348       ??_C@_0CF@EANP@R6028?$AN?6?9?5unable?5to?5initialize?5he@ 00454348     LIBCMTD:crt0msg.obj
 0002:00003370       ??_C@_0DF@ECGN@R6027?$AN?6?9?5not?5enough?5space?5for?5lo@ 00454370     LIBCMTD:crt0msg.obj
 0002:000033a8       ??_C@_0DF@FKAC@R6026?$AN?6?9?5not?5enough?5space?5for?5st@ 004543a8     LIBCMTD:crt0msg.obj
 0002:000033e0       ??_C@_0CG@DPMN@R6025?$AN?6?9?5pure?5virtual?5function?5c@ 004543e0     LIBCMTD:crt0msg.obj
 0002:00003408       ??_C@_0DF@CKIP@R6024?$AN?6?9?5not?5enough?5space?5for?5_o@ 00454408     LIBCMTD:crt0msg.obj
 0002:00003440       ??_C@_0CJ@GGOE@R6019?$AN?6?9?5unable?5to?5open?5console?5@ 00454440     LIBCMTD:crt0msg.obj
 0002:0000346c       ??_C@_0CB@LBOB@R6018?$AN?6?9?5unexpected?5heap?5error?$AN?6@ 0045446c     LIBCMTD:crt0msg.obj
 0002:00003490       ??_C@_0CN@FPEG@R6017?$AN?6?9?5unexpected?5multithread?5@ 00454490     LIBCMTD:crt0msg.obj
 0002:000034c0       ??_C@_0CM@OBIC@R6016?$AN?6?9?5not?5enough?5space?5for?5th@ 004544c0     LIBCMTD:crt0msg.obj
 0002:000034ec       ??_C@_0CB@HPAL@?$AN?6abnormal?5program?5termination?$AN?6@ 004544ec     LIBCMTD:crt0msg.obj
 0002:00003510       ??_C@_0CM@JOOB@R6009?$AN?6?9?5not?5enough?5space?5for?5en@ 00454510     LIBCMTD:crt0msg.obj
 0002:0000353c       ??_C@_0CK@OIBL@R6008?$AN?6?9?5not?5enough?5space?5for?5ar@ 0045453c     LIBCMTD:crt0msg.obj
 0002:00003568       ??_C@_0CF@LKPB@R6002?$AN?6?9?5floating?5point?5not?5load@ 00454568     LIBCMTD:crt0msg.obj
 0002:00003590       ??_C@_0BK@DEOK@Runtime?5Error?$CB?6?6Program?3?5?$AA@ 00454590     LIBCMTD:crt0msg.obj
 0002:000035ac       ??_C@_09EMDO@_getbuf?4c?$AA@ 004545ac     LIBCMTD:_getbuf.obj
 0002:000035b8       ??_C@_08MOLN@mbtowc?4c?$AA@ 004545b8     LIBCMTD:mbtowc.obj
 0002:000035c4       ??_C@_0CD@NPPL@MB_CUR_MAX?5?$DN?$DN?51?5?$HM?$HM?5MB_CUR_MAX?5?$DN?$DN@ 004545c4     LIBCMTD:mbtowc.obj
 0002:000035e8       ??_C@_09DNOI@_filbuf?4c?$AA@ 004545e8     LIBCMTD:_filbuf.obj
 0002:000035f4       ??_C@_08JKP@ungetc?4c?$AA@ 004545f4     LIBCMTD:ungetc.obj
 0002:00003600       ??_C@_01A@?$AA?$AA@        00454600     LIBCMTD:a_str.obj
 0002:00003604       ??_C@_13A@?$AA?$AA?$AA?$AA@ 00454604     LIBCMTD:a_str.obj
 0002:00003614       ??_C@_09JNND@_sftbuf?4c?$AA@ 00454614     LIBCMTD:_sftbuf.obj
 0002:00003620       ??_C@_0BH@EOPG@flag?5?$DN?$DN?50?5?$HM?$HM?5flag?5?$DN?$DN?51?$AA@ 00454620     LIBCMTD:_sftbuf.obj
 0002:00003638       ??_C@_0L@JIE@_freebuf?4c?$AA@ 00454638     LIBCMTD:_freebuf.obj
 0002:00003644       ??_C@_0L@EEGJ@inittime?4c?$AA@ 00454644     LIBCMTD:inittime.obj
 0002:00003650       ??_C@_09IMJJ@initnum?4c?$AA@ 00454650     LIBCMTD:initnum.obj
 0002:0000365c       ??_C@_09KPNI@initmon?4c?$AA@ 0045465c     LIBCMTD:initmon.obj
 0002:00003668       ??_C@_0L@COIL@initctyp?4c?$AA@ 00454668     LIBCMTD:initctyp.obj
 0002:00003674       ??_C@_08OBJD@Paraguay?$AA@ 00454674     LIBCMTD:getqloc.obj
 0002:00003680       ??_C@_07GLKH@Uruguay?$AA@  00454680     LIBCMTD:getqloc.obj
 0002:00003688       ??_C@_05FPFC@Chile?$AA@    00454688     LIBCMTD:getqloc.obj
 0002:00003690       ??_C@_07IIGF@Ecuador?$AA@  00454690     LIBCMTD:getqloc.obj
 0002:00003698       ??_C@_09PKAL@Argentina?$AA@ 00454698     LIBCMTD:getqloc.obj
 0002:000036a4       ??_C@_04LKAH@Peru?$AA@     004546a4     LIBCMTD:getqloc.obj
 0002:000036ac       ??_C@_08NEEM@Colombia?$AA@ 004546ac     LIBCMTD:getqloc.obj
 0002:000036b8       ??_C@_09ODEB@Venezuela?$AA@ 004546b8     LIBCMTD:getqloc.obj
 0002:000036c4       ??_C@_0BD@CLEL@Dominican?5Republic?$AA@ 004546c4     LIBCMTD:getqloc.obj
 0002:000036d8       ??_C@_0N@MDGL@South?5Africa?$AA@ 004546d8     LIBCMTD:getqloc.obj
 0002:000036e8       ??_C@_06NKBG@Panama?$AA@   004546e8     LIBCMTD:getqloc.obj
 0002:000036f0       ??_C@_0L@BMHO@Luxembourg?$AA@ 004546f0     LIBCMTD:getqloc.obj
 0002:000036fc       ??_C@_0L@IMDK@Costa?5Rica?$AA@ 004546fc     LIBCMTD:getqloc.obj
 0002:00003708       ??_C@_0M@BLJF@Switzerland?$AA@ 00454708     LIBCMTD:getqloc.obj
 0002:00003714       ??_C@_09KBOL@Guatemala?$AA@ 00454714     LIBCMTD:getqloc.obj
 0002:00003720       ??_C@_06JNAK@Canada?$AA@   00454720     LIBCMTD:getqloc.obj
 0002:00003728       ??_C@_0BG@OLLP@Spanish?5?9?5Modern?5Sort?$AA@ 00454728     LIBCMTD:getqloc.obj
 0002:00003740       ??_C@_09IDKE@Australia?$AA@ 00454740     LIBCMTD:getqloc.obj
 0002:0000374c       ??_C@_07JJJJ@English?$AA@  0045474c     LIBCMTD:getqloc.obj
 0002:00003754       ??_C@_07NMDO@Austria?$AA@  00454754     LIBCMTD:getqloc.obj
 0002:0000375c       ??_C@_06DEFE@German?$AA@   0045475c     LIBCMTD:getqloc.obj
 0002:00003764       ??_C@_07JAIH@Belgium?$AA@  00454764     LIBCMTD:getqloc.obj
 0002:0000376c       ??_C@_06BNLJ@Mexico?$AA@   0045476c     LIBCMTD:getqloc.obj
 0002:00003774       ??_C@_07JHAG@Spanish?$AA@  00454774     LIBCMTD:getqloc.obj
 0002:0000377c       ??_C@_06DADE@Basque?$AA@   0045477c     LIBCMTD:getqloc.obj
 0002:00003784       ??_C@_06ENFP@Sweden?$AA@   00454784     LIBCMTD:getqloc.obj
 0002:0000378c       ??_C@_07JPMH@Swedish?$AA@  0045478c     LIBCMTD:getqloc.obj
 0002:00003794       ??_C@_07IEKF@Iceland?$AA@  00454794     LIBCMTD:getqloc.obj
 0002:0000379c       ??_C@_09KNEA@Icelandic?$AA@ 0045479c     LIBCMTD:getqloc.obj
 0002:000037a8       ??_C@_06IJOD@France?$AA@   004547a8     LIBCMTD:getqloc.obj
 0002:000037b0       ??_C@_06EINI@French?$AA@   004547b0     LIBCMTD:getqloc.obj
 0002:000037b8       ??_C@_07FOOE@Finland?$AA@  004547b8     LIBCMTD:getqloc.obj
 0002:000037c0       ??_C@_07OJOM@Finnish?$AA@  004547c0     LIBCMTD:getqloc.obj
 0002:000037c8       ??_C@_05FFAC@Spain?$AA@    004547c8     LIBCMTD:getqloc.obj
 0002:000037d0       ??_C@_0BL@BIHM@Spanish?5?9?5Traditional?5Sort?$AA@ 004547d0     LIBCMTD:getqloc.obj
 0002:000037ec       ??_C@_0O@GLHB@united?9states?$AA@ 004547ec     LIBCMTD:getqloc.obj
 0002:000037fc       ??_C@_0P@IIKK@united?9kingdom?$AA@ 004547fc     LIBCMTD:getqloc.obj
 0002:0000380c       ??_C@_0BC@FHBO@trinidad?5?$CG?5tobago?$AA@ 0045480c     LIBCMTD:getqloc.obj
 0002:00003820       ??_C@_0M@BDFM@south?9korea?$AA@ 00454820     LIBCMTD:getqloc.obj
 0002:0000382c       ??_C@_0N@CKFA@south?9africa?$AA@ 0045482c     LIBCMTD:getqloc.obj
 0002:0000383c       ??_C@_0M@HNHN@south?5korea?$AA@ 0045483c     LIBCMTD:getqloc.obj
 0002:00003848       ??_C@_0N@MKDO@south?5africa?$AA@ 00454848     LIBCMTD:getqloc.obj
 0002:00003858       ??_C@_06KFFJ@slovak?$AA@   00454858     LIBCMTD:getqloc.obj
 0002:00003860       ??_C@_0M@NMAC@puerto?9rico?$AA@ 00454860     LIBCMTD:getqloc.obj
 0002:0000386c       ??_C@_08EJOH@pr?9china?$AA@ 0045486c     LIBCMTD:getqloc.obj
 0002:00003878       ??_C@_08CHMG@pr?5china?$AA@ 00454878     LIBCMTD:getqloc.obj
 0002:00003884       ??_C@_02OCJK@nz?$AA@       00454884     LIBCMTD:getqloc.obj
 0002:00003888       ??_C@_0M@MMKA@new?9zealand?$AA@ 00454888     LIBCMTD:getqloc.obj
 0002:00003894       ??_C@_09MGEH@hong?9kong?$AA@ 00454894     LIBCMTD:getqloc.obj
 0002:000038a0       ??_C@_07CCAK@holland?$AA@  004548a0     LIBCMTD:getqloc.obj
 0002:000038a8       ??_C@_0O@MEPL@great?5britain?$AA@ 004548a8     LIBCMTD:getqloc.obj
 0002:000038b8       ??_C@_07LGIB@england?$AA@  004548b8     LIBCMTD:getqloc.obj
 0002:000038c0       ??_C@_05BMOA@czech?$AA@    004548c0     LIBCMTD:getqloc.obj
 0002:000038c8       ??_C@_05NMPB@china?$AA@    004548c8     LIBCMTD:getqloc.obj
 0002:000038d0       ??_C@_07GN@britain?$AA@    004548d0     LIBCMTD:getqloc.obj
 0002:000038d8       ??_C@_07DLAK@america?$AA@  004548d8     LIBCMTD:getqloc.obj
 0002:000038e0       ??_C@_03IPEP@usa?$AA@      004548e0     LIBCMTD:getqloc.obj
 0002:000038e4       ??_C@_02PILH@us?$AA@       004548e4     LIBCMTD:getqloc.obj
 0002:000038e8       ??_C@_02FHP@uk?$AA@        004548e8     LIBCMTD:getqloc.obj
 0002:000038ec       ??_C@_05DEAI@swiss?$AA@    004548ec     LIBCMTD:getqloc.obj
 0002:000038f4       ??_C@_0BA@LIAF@swedish?9finland?$AA@ 004548f4     LIBCMTD:getqloc.obj
 0002:00003904       ??_C@_0BC@FMEG@spanish?9venezuela?$AA@ 00454904     LIBCMTD:getqloc.obj
 0002:00003918       ??_C@_0BA@BNMG@spanish?9uruguay?$AA@ 00454918     LIBCMTD:getqloc.obj
 0002:00003928       ??_C@_0BE@BKDJ@spanish?9puerto?5rico?$AA@ 00454928     LIBCMTD:getqloc.obj
 0002:0000393c       ??_C@_0N@JIBL@spanish?9peru?$AA@ 0045493c     LIBCMTD:getqloc.obj
 0002:0000394c       ??_C@_0BB@OGOF@spanish?9paraguay?$AA@ 0045494c     LIBCMTD:getqloc.obj
 0002:00003960       ??_C@_0P@LLFA@spanish?9panama?$AA@ 00454960     LIBCMTD:getqloc.obj
 0002:00003970       ??_C@_0BC@BBJM@spanish?9nicaragua?$AA@ 00454970     LIBCMTD:getqloc.obj
 0002:00003984       ??_C@_0P@NJBN@spanish?9modern?$AA@ 00454984     LIBCMTD:getqloc.obj
 0002:00003994       ??_C@_0BA@NHDN@spanish?9mexican?$AA@ 00454994     LIBCMTD:getqloc.obj
 0002:000039a4       ??_C@_0BB@JHOJ@spanish?9honduras?$AA@ 004549a4     LIBCMTD:getqloc.obj
 0002:000039b8       ??_C@_0BC@BOOM@spanish?9guatemala?$AA@ 004549b8     LIBCMTD:getqloc.obj
 0002:000039cc       ??_C@_0BE@EELI@spanish?9el?5salvador?$AA@ 004549cc     LIBCMTD:getqloc.obj
 0002:000039e0       ??_C@_0BA@POAE@spanish?9ecuador?$AA@ 004549e0     LIBCMTD:getqloc.obj
 0002:000039f0       ??_C@_0BL@LDKN@spanish?9dominican?5republic?$AA@ 004549f0     LIBCMTD:getqloc.obj
 0002:00003a0c       ??_C@_0BD@HPMH@spanish?9costa?5rica?$AA@ 00454a0c     LIBCMTD:getqloc.obj
 0002:00003a20       ??_C@_0BB@NDDK@spanish?9colombia?$AA@ 00454a20     LIBCMTD:getqloc.obj
 0002:00003a34       ??_C@_0O@BJHA@spanish?9chile?$AA@ 00454a34     LIBCMTD:getqloc.obj
 0002:00003a44       ??_C@_0BA@OBNG@spanish?9bolivia?$AA@ 00454a44     LIBCMTD:getqloc.obj
 0002:00003a54       ??_C@_0BC@EFAM@spanish?9argentina?$AA@ 00454a54     LIBCMTD:getqloc.obj
 0002:00003a68       ??_C@_0BF@KMMM@portuguese?9brazilian?$AA@ 00454a68     LIBCMTD:getqloc.obj
 0002:00003a80       ??_C@_0BC@BAAE@norwegian?9nynorsk?$AA@ 00454a80     LIBCMTD:getqloc.obj
 0002:00003a94       ??_C@_0BB@PBHK@norwegian?9bokmal?$AA@ 00454a94     LIBCMTD:getqloc.obj
 0002:00003aa8       ??_C@_09EHKL@norwegian?$AA@ 00454aa8     LIBCMTD:getqloc.obj
 0002:00003ab4       ??_C@_0O@BEAN@italian?9swiss?$AA@ 00454ab4     LIBCMTD:getqloc.obj
 0002:00003ac4       ??_C@_0O@OIFK@irish?9english?$AA@ 00454ac4     LIBCMTD:getqloc.obj
 0002:00003ad4       ??_C@_0N@NBPL@german?9swiss?$AA@ 00454ad4     LIBCMTD:getqloc.obj
 0002:00003ae4       ??_C@_0BC@ICFJ@german?9luxembourg?$AA@ 00454ae4     LIBCMTD:getqloc.obj
 0002:00003af8       ??_C@_0BE@GGPC@german?9lichtenstein?$AA@ 00454af8     LIBCMTD:getqloc.obj
 0002:00003b0c       ??_C@_0BA@MKDC@german?9austrian?$AA@ 00454b0c     LIBCMTD:getqloc.obj
 0002:00003b1c       ??_C@_0N@ODNB@french?9swiss?$AA@ 00454b1c     LIBCMTD:getqloc.obj
 0002:00003b2c       ??_C@_0BC@MGCM@french?9luxembourg?$AA@ 00454b2c     LIBCMTD:getqloc.obj
 0002:00003b40       ??_C@_0BA@NABK@french?9canadian?$AA@ 00454b40     LIBCMTD:getqloc.obj
 0002:00003b50       ??_C@_0P@CJNO@french?9belgian?$AA@ 00454b50     LIBCMTD:getqloc.obj
 0002:00003b60       ??_C@_0M@LJOL@english?9usa?$AA@ 00454b60     LIBCMTD:getqloc.obj
 0002:00003b6c       ??_C@_0L@FMNC@english?9us?$AA@ 00454b6c     LIBCMTD:getqloc.obj
 0002:00003b78       ??_C@_0L@KBBK@english?9uk?$AA@ 00454b78     LIBCMTD:getqloc.obj
 0002:00003b84       ??_C@_0BK@NDDE@english?9trinidad?5y?5tobago?$AA@ 00454b84     LIBCMTD:getqloc.obj
 0002:00003ba0       ??_C@_0BF@LKML@english?9south?5africa?$AA@ 00454ba0     LIBCMTD:getqloc.obj
 0002:00003bb8       ??_C@_0L@EGPP@english?9nz?$AA@ 00454bb8     LIBCMTD:getqloc.obj
 0002:00003bc4       ??_C@_0BA@HLH@english?9jamaica?$AA@ 00454bc4     LIBCMTD:getqloc.obj
 0002:00003bd4       ??_C@_0M@PMJI@english?9ire?$AA@ 00454bd4     LIBCMTD:getqloc.obj
 0002:00003be0       ??_C@_0BC@HINE@english?9caribbean?$AA@ 00454be0     LIBCMTD:getqloc.obj
 0002:00003bf4       ??_C@_0M@DCFH@english?9can?$AA@ 00454bf4     LIBCMTD:getqloc.obj
 0002:00003c00       ??_C@_0P@DGHK@english?9belize?$AA@ 00454c00     LIBCMTD:getqloc.obj
 0002:00003c10       ??_C@_0M@FLHK@english?9aus?$AA@ 00454c10     LIBCMTD:getqloc.obj
 0002:00003c1c       ??_C@_0BB@HNCK@english?9american?$AA@ 00454c1c     LIBCMTD:getqloc.obj
 0002:00003c30       ??_C@_0O@PAMI@dutch?9belgian?$AA@ 00454c30     LIBCMTD:getqloc.obj
 0002:00003c40       ??_C@_0BE@FPEJ@chinese?9traditional?$AA@ 00454c40     LIBCMTD:getqloc.obj
 0002:00003c54       ??_C@_0BC@CHFL@chinese?9singapore?$AA@ 00454c54     LIBCMTD:getqloc.obj
 0002:00003c68       ??_C@_0BD@DCMH@chinese?9simplified?$AA@ 00454c68     LIBCMTD:getqloc.obj
 0002:00003c7c       ??_C@_0BB@JMOE@chinese?9hongkong?$AA@ 00454c7c     LIBCMTD:getqloc.obj
 0002:00003c90       ??_C@_07NGFN@chinese?$AA@  00454c90     LIBCMTD:getqloc.obj
 0002:00003c98       ??_C@_03PCOI@chi?$AA@      00454c98     LIBCMTD:getqloc.obj
 0002:00003c9c       ??_C@_03FIHP@chh?$AA@      00454c9c     LIBCMTD:getqloc.obj
 0002:00003ca0       ??_C@_08HFLO@canadian?$AA@ 00454ca0     LIBCMTD:getqloc.obj
 0002:00003cac       ??_C@_07INIJ@belgian?$AA@  00454cac     LIBCMTD:getqloc.obj
 0002:00003cb4       ??_C@_0L@LCCA@australian?$AA@ 00454cb4     LIBCMTD:getqloc.obj
 0002:00003cc0       ??_C@_0BB@BJIO@american?9english?$AA@ 00454cc0     LIBCMTD:getqloc.obj
 0002:00003cd4       ??_C@_0BB@DAGO@american?5english?$AA@ 00454cd4     LIBCMTD:getqloc.obj
 0002:00003ce8       ??_C@_08HENB@american?$AA@ 00454ce8     LIBCMTD:getqloc.obj
 0002:00003cf4       ??_C@_03DGJE@OCP?$AA@      00454cf4     LIBCMTD:getqloc.obj
 0002:00003cf8       ??_C@_03EKFG@ACP?$AA@      00454cf8     LIBCMTD:getqloc.obj
 0002:00003d18       ??_C@_09LNLM@osfinfo?4c?$AA@ 00454d18     LIBCMTD:osfinfo.obj
 0002:00003d24       ??_C@_08PHBD@fclose?4c?$AA@ 00454d24     LIBCMTD:fclose.obj
 0002:00003d30       ??_C@_07CJME@H?3mm?3ss?$AA@ 00454d30     LIBCMTD:strftime.obj
 0002:00003d38       ??_C@_0BE@MHI@dddd?0?5MMMM?5dd?0?5yyyy?$AA@ 00454d38     LIBCMTD:strftime.obj
 0002:00003d4c       ??_C@_06HCAD@M?1d?1yy?$AA@ 00454d4c     LIBCMTD:strftime.obj
 0002:00003d54       ??_C@_02DBLP@PM?$AA@       00454d54     LIBCMTD:strftime.obj
 0002:00003d58       ??_C@_02ENLM@AM?$AA@       00454d58     LIBCMTD:strftime.obj
 0002:00003d5c       ??_C@_08LIDF@December?$AA@ 00454d5c     LIBCMTD:strftime.obj
 0002:00003d68       ??_C@_08NJLI@November?$AA@ 00454d68     LIBCMTD:strftime.obj
 0002:00003d74       ??_C@_07IAMM@October?$AA@  00454d74     LIBCMTD:strftime.obj
 0002:00003d7c       ??_C@_09MKGD@September?$AA@ 00454d7c     LIBCMTD:strftime.obj
 0002:00003d88       ??_C@_06PADP@August?$AA@   00454d88     LIBCMTD:strftime.obj
 0002:00003d90       ??_C@_04PIJO@July?$AA@     00454d90     LIBCMTD:strftime.obj
 0002:00003d98       ??_C@_04ICFP@June?$AA@     00454d98     LIBCMTD:strftime.obj
 0002:00003da0       ??_C@_05JFGC@April?$AA@    00454da0     LIBCMTD:strftime.obj
 0002:00003da8       ??_C@_05FGPD@March?$AA@    00454da8     LIBCMTD:strftime.obj
 0002:00003db0       ??_C@_08PGBA@February?$AA@ 00454db0     LIBCMTD:strftime.obj
 0002:00003dbc       ??_C@_07BPKJ@January?$AA@  00454dbc     LIBCMTD:strftime.obj
 0002:00003dc4       ??_C@_03PGJO@Dec?$AA@      00454dc4     LIBCMTD:strftime.obj
 0002:00003dc8       ??_C@_03PDLM@Nov?$AA@      00454dc8     LIBCMTD:strftime.obj
 0002:00003dcc       ??_C@_03BLHK@Oct?$AA@      00454dcc     LIBCMTD:strftime.obj
 0002:00003dd0       ??_C@_03DPFM@Sep?$AA@      00454dd0     LIBCMTD:strftime.obj
 0002:00003dd4       ??_C@_03CMCH@Aug?$AA@      00454dd4     LIBCMTD:strftime.obj
 0002:00003dd8       ??_C@_03OBKI@Jul?$AA@      00454dd8     LIBCMTD:strftime.obj
 0002:00003ddc       ??_C@_03LEIG@Jun?$AA@      00454ddc     LIBCMTD:strftime.obj
 0002:00003de0       ??_C@_03MGHB@May?$AA@      00454de0     LIBCMTD:strftime.obj
 0002:00003de4       ??_C@_03MJJM@Apr?$AA@      00454de4     LIBCMTD:strftime.obj
 0002:00003de8       ??_C@_03GNHA@Mar?$AA@      00454de8     LIBCMTD:strftime.obj
 0002:00003dec       ??_C@_03PICE@Feb?$AA@      00454dec     LIBCMTD:strftime.obj
 0002:00003df0       ??_C@_03IEIF@Jan?$AA@      00454df0     LIBCMTD:strftime.obj
 0002:00003df4       ??_C@_08FAKH@Saturday?$AA@ 00454df4     LIBCMTD:strftime.obj
 0002:00003e00       ??_C@_06ONCK@Friday?$AA@   00454e00     LIBCMTD:strftime.obj
 0002:00003e08       ??_C@_08CCFO@Thursday?$AA@ 00454e08     LIBCMTD:strftime.obj
 0002:00003e14       ??_C@_09PBIN@Wednesday?$AA@ 00454e14     LIBCMTD:strftime.obj
 0002:00003e20       ??_C@_07BMBC@Tuesday?$AA@  00454e20     LIBCMTD:strftime.obj
 0002:00003e28       ??_C@_06CHLK@Monday?$AA@   00454e28     LIBCMTD:strftime.obj
 0002:00003e30       ??_C@_06OOEM@Sunday?$AA@   00454e30     LIBCMTD:strftime.obj
 0002:00003e38       ??_C@_03MPKK@Sat?$AA@      00454e38     LIBCMTD:strftime.obj
 0002:00003e3c       ??_C@_03FINJ@Fri?$AA@      00454e3c     LIBCMTD:strftime.obj
 0002:00003e40       ??_C@_03HIKC@Thu?$AA@      00454e40     LIBCMTD:strftime.obj
 0002:00003e44       ??_C@_03HECK@Wed?$AA@      00454e44     LIBCMTD:strftime.obj
 0002:00003e48       ??_C@_03ECCP@Tue?$AA@      00454e48     LIBCMTD:strftime.obj
 0002:00003e4c       ??_C@_03PIEP@Mon?$AA@      00454e4c     LIBCMTD:strftime.obj
 0002:00003e50       ??_C@_03FHEP@Sun?$AA@      00454e50     LIBCMTD:strftime.obj
 0002:00003e54       ??_C@_03MKGK@a?1p?$AA@     00454e54     LIBCMTD:strftime.obj
 0002:00003e58       ??_C@_05BDJK@am?1pm?$AA@   00454e58     LIBCMTD:strftime.obj
 0002:00003e60       ??_C@_0L@HKCB@inithelp?4c?$AA@ 00454e60     LIBCMTD:inithelp.obj
 0002:00003e88       ___dnames                  00454e88     LIBCMTD:timeset.obj
 0002:00003ea0       ___mnames                  00454ea0     LIBCMTD:timeset.obj
 0002:00003ec8       ??_C@_07DEKI@tzset?4c?$AA@ 00454ec8     LIBCMTD:tzset.obj
 0002:00003ed0       ??_C@_02JHIA@TZ?$AA@       00454ed0     LIBCMTD:tzset.obj
 0002:00003ef4       ??_C@_0L@EJNO@wtombenv?4c?$AA@ 00454ef4     LIBCMTD:wtombenv.obj
 0002:00003f00       ??_C@_07FOIK@a_cmp?4c?$AA@ 00454f00     LIBCMTD:a_cmp.obj
 0002:00003f08       ??_C@_0DN@PPKB@cchCount1?$DN?$DN0?5?$CG?$CG?5cchCount2?$DN?$DN1?5?$HM?$HM?5@ 00454f08     LIBCMTD:a_cmp.obj
 0002:00003f60       ??_C@_08FEIK@setenv?4c?$AA@ 00454f60     LIBCMTD:setenv.obj
 0002:000046a0       ??_R1A@?0A@A@type_info@@8  004556a0     LIBCMTD:typinfo.obj
 0002:000046b8       ??_R2type_info@@8          004556b8     LIBCMTD:typinfo.obj
 0002:000046c0       ??_R3type_info@@8          004556c0     LIBCMTD:typinfo.obj
 0002:000046d0       ??_R4type_info@@6B@        004556d0     LIBCMTD:typinfo.obj
 0002:00004948       __CT??_R0?AVException@@@8??0Exception@@QAE@ABV0@@Z8 00455948     ClientConnection.obj
 0002:00004968       __CT??_R0?AVQuietException@@@8??0QuietException@@QAE@ABV0@@Z8 00455968     ClientConnection.obj
 0002:00004988       __CTA2?AVQuietException@@  00455988     ClientConnection.obj
 0002:00004998       __TI2?AVQuietException@@   00455998     ClientConnection.obj
 0002:000049e0       __CT??_R0?AVWarningException@@@8??0WarningException@@QAE@ABV0@@Z12 004559e0     ClientConnection.obj
 0002:00004a00       __CTA2?AVWarningException@@ 00455a00     ClientConnection.obj
 0002:00004a10       __TI2?AVWarningException@@ 00455a10     ClientConnection.obj
 0002:00004a88       __CT??_R0?AVErrorException@@@8??0ErrorException@@QAE@ABV0@@Z8 00455a88     ClientConnection.obj
 0002:00004aa8       __CTA2?AVErrorException@@  00455aa8     ClientConnection.obj
 0002:00004ab8       __TI2?AVErrorException@@   00455ab8     ClientConnection.obj
 0002:00005518       __CT??_R0?AVomni_thread_fatal@@@84 00456518     omnithread:nt.obj
 0002:00005538       __CTA1?AVomni_thread_fatal@@ 00456538     omnithread:nt.obj
 0002:00005540       __TI1?AVomni_thread_fatal@@ 00456540     omnithread:nt.obj
 0002:00005740       __CT??_R0?AVomni_thread_invalid@@@81 00456740     omnithread:nt.obj
 0002:00005760       __CTA1?AVomni_thread_invalid@@ 00456760     omnithread:nt.obj
 0002:00005768       __TI1?AVomni_thread_invalid@@ 00456768     omnithread:nt.obj
 0003:00000000       ___xc_a                    00457000     LIBCMTD:crt0init.obj
 0003:00000278       ___xc_z                    00457278     LIBCMTD:crt0init.obj
 0003:0000037c       ___xi_a                    0045737c     LIBCMTD:crt0init.obj
 0003:00000694       ___xi_z                    00457694     LIBCMTD:crt0init.obj
 0003:00000798       ___xp_a                    00457798     LIBCMTD:crt0init.obj
 0003:000009a0       ___xp_z                    004579a0     LIBCMTD:crt0init.obj
 0003:00000aa4       ___xt_a                    00457aa4     LIBCMTD:crt0init.obj
 0003:00000cac       ___xt_z                    00457cac     LIBCMTD:crt0init.obj
 0003:00000db0       ??_R0?AVException@@@8      00457db0     ClientConnection.obj
 0003:00000dd0       ??_R0?AVQuietException@@@8 00457dd0     ClientConnection.obj
 0003:00000df8       ??_R0?AVWarningException@@@8 00457df8     ClientConnection.obj
 0003:00000e20       ??_R0?AVErrorException@@@8 00457e20     ClientConnection.obj
 0003:00000e48       ??_R0?AVomni_thread_invalid@@@8 00457e48     ClientConnection.obj
 0003:00001974       ?__LINE__Var@?1??WndProc@Daemon@@SGJPAUHWND__@@IIJ@Z@4FA@c741cf33 00458974     Daemon.obj
 0003:00001978       ?__LINE__Var@?1???0Exception@@QAE@PBD@Z@4FA 00458978     Exception.obj
 0003:0000197c       ?__LINE__Var@?1??Report@Exception@@UAEXXZ@4FA 0045897c     Exception.obj
 0003:00001980       ?__LINE__Var@?1??WndProc@Flasher@@SGJPAUHWND__@@IIJ@Z@4FA@53c060cf 00458980     Flasher.obj
 0003:00001988       _fixedkey                  00458988     vncauth.obj
 0003:00001994       ?BELL_APPL_KEY_NAME@@3PBDB 00458994     VNCviewerApp32.obj
 0003:00001998       ?BELL_LABEL@@3PBDB         00458998     VNCviewerApp32.obj
 0003:00001a00       ??_R0?AVomni_thread_fatal@@@8 00458a00     omnithread:nt.obj
 0003:00001a20       __NLG_Destination          00458a20     LIBCMTD:exsup.obj
 0003:00001a30       ??_R0?AVtype_info@@@8      00458a30     LIBCMTD:typinfo.obj
 0003:00001a48       ?__pMyUnhandledExceptionFilter@@3PAXA 00458a48     LIBCMTD:throw.obj
 0003:00001a4c       __crtDbgFlag               00458a4c     LIBCMTD:dbgheap.obj
 0003:00001a54       __crtBreakAlloc            00458a54     LIBCMTD:dbgheap.obj
 0003:00001aa4       __crtAssertBusy            00458aa4     LIBCMTD:dbgrpt.obj
 0003:00001aa8       __CrtDbgMode               00458aa8     LIBCMTD:dbgrpt.obj
 0003:00001ab4       __CrtDbgFile               00458ab4     LIBCMTD:dbgrpt.obj
 0003:00001ad0       __aexit_rtn                00458ad0     LIBCMTD:wincrt0.obj
 0003:00001ad4       ___app_type                00458ad4     LIBCMTD:wincrt0.obj
 0003:00001ad8       __locktable                00458ad8     LIBCMTD:mlock.obj
 0003:00001ba0       ___tlsindex                00458ba0     LIBCMTD:tidtable.obj
 0003:00001ba4       ?__pInconsistency@@3P6AXXZA 00458ba4     LIBCMTD:hooks.obj
 0003:00001ba8       ___nullstring              00458ba8     LIBCMTD:output.obj
 0003:00001bac       ___wnullstring             00458bac     LIBCMTD:output.obj
 0003:00001bbc       __pfnAllocHook             00458bbc     LIBCMTD:dbghook.obj
 0003:00001bc0       ___old_small_block_heap    00458bc0     LIBCMTD:sbheap.obj
 0003:00003be4       ___old_sbh_threshold       0045abe4     LIBCMTD:sbheap.obj
 0003:00003be8       __amblksiz                 0045abe8     LIBCMTD:heapinit.obj
 0003:00003bec       __pctype                   0045abec     LIBCMTD:ctype.obj
 0003:00003bf0       __pwctype                  0045abf0     LIBCMTD:ctype.obj
 0003:00003bf4       __ctype                    0045abf4     LIBCMTD:ctype.obj
 0003:00003df8       ___mb_cur_max              0045adf8     LIBCMTD:nlsdata1.obj
 0003:00003dfc       ___decimal_point           0045adfc     LIBCMTD:nlsdata1.obj
 0003:00003e00       ___decimal_point_length    0045ae00     LIBCMTD:nlsdata1.obj
 0003:00003e10       __iob                      0045ae10     LIBCMTD:_file.obj
 0003:00004308       ___lc_category             0045b308     LIBCMTD:setlocal.obj
 0003:00004350       __XcptActTab               0045b350     LIBCMTD:winxfltr.obj
 0003:000043c8       __First_FPE_Indx           0045b3c8     LIBCMTD:winxfltr.obj
 0003:000043cc       __Num_FPE                  0045b3cc     LIBCMTD:winxfltr.obj
 0003:000043d0       __XcptActTabSize           0045b3d0     LIBCMTD:winxfltr.obj
 0003:000043d4       __XcptActTabCount          0045b3d4     LIBCMTD:winxfltr.obj
 0003:000043d8       ___badioinfo               0045b3d8     LIBCMTD:ioinit.obj
 0003:00004490       __cfltcvt_tab              0045b490     LIBCMTD:cmiscdat.obj
 0003:000044b0       ___rgLocInfo               0045b4b0     LIBCMTD:getqloc.obj
 0003:00004954       ___rglangidNotDefault      0045b954     LIBCMTD:getqloc.obj
 0003:00004968       ___rg_country              0045b968     LIBCMTD:getqloc.obj
 0003:00004a20       ___rg_language             0045ba20     LIBCMTD:getqloc.obj
 0003:00004d20       ___lc_time_curr            0045bd20     LIBCMTD:strftime.obj
 0003:00004d28       ___lc_time_c               0045bd28     LIBCMTD:strftime.obj
 0003:00004dd8       ___lconv_static_decimal    0045bdd8     LIBCMTD:lconv.obj
 0003:00004de0       ___lconv_c                 0045bde0     LIBCMTD:lconv.obj
 0003:00004e10       ___lconv                   0045be10     LIBCMTD:lconv.obj
 0003:00004e20       __timezone                 0045be20     LIBCMTD:timeset.obj
 0003:00004e24       __daylight                 0045be24     LIBCMTD:timeset.obj
 0003:00004e28       __dstbias                  0045be28     LIBCMTD:timeset.obj
 0003:00004eac       __tzname                   0045beac     LIBCMTD:timeset.obj
 0003:00004ee0       __lpdays                   0045bee0     LIBCMTD:days.obj
 0003:00004f14       __days                     0045bf14     LIBCMTD:days.obj
 0003:00005d78       ?theLog@@3VLog@@A          0045cd78     Log.obj
 0003:00005d98       ?log@@3VLog@@A             0045cd98     vncviewer.obj
 0003:00005db0       ?pApp@@3PAVVNCviewerApp@@A 0045cdb0     VNCviewerApp.obj
 0003:00005dc0       ?cachelock@_internal_omni_thread_helper@@2Vomni_mutex@@A 0045cdc0     omnithread:nt.obj
 0003:00005de0       ?next_id_mutex@omni_thread@@0PAVomni_mutex@@A 0045cde0     omnithread:nt.obj
 0003:00005de4       ?cache@_internal_omni_thread_helper@@2PAV_internal_omni_thread_dummy@@A 0045cde4     omnithread:nt.obj
 0003:00005de8       ?count@init_t@omni_thread@@0HA 0045cde8     omnithread:nt.obj
 0003:00005dec       ?next_id@omni_thread@@0HA  0045cdec     omnithread:nt.obj
 0003:00005e08       __umaskval                 0045ce08     LIBCMTD:crt0dat.obj
 0003:00005e0c       __osver                    0045ce0c     LIBCMTD:crt0dat.obj
 0003:00005e10       __winver                   0045ce10     LIBCMTD:crt0dat.obj
 0003:00005e14       __winmajor                 0045ce14     LIBCMTD:crt0dat.obj
 0003:00005e18       __winminor                 0045ce18     LIBCMTD:crt0dat.obj
 0003:00005e1c       ___argc                    0045ce1c     LIBCMTD:crt0dat.obj
 0003:00005e20       ___argv                    0045ce20     LIBCMTD:crt0dat.obj
 0003:00005e24       ___wargv                   0045ce24     LIBCMTD:crt0dat.obj
 0003:00005e28       __environ                  0045ce28     LIBCMTD:crt0dat.obj
 0003:00005e2c       ___initenv                 0045ce2c     LIBCMTD:crt0dat.obj
 0003:00005e30       __wenviron                 0045ce30     LIBCMTD:crt0dat.obj
 0003:00005e34       ___winitenv                0045ce34     LIBCMTD:crt0dat.obj
 0003:00005e38       __pgmptr                   0045ce38     LIBCMTD:crt0dat.obj
 0003:00005e3c       __wpgmptr                  0045ce3c     LIBCMTD:crt0dat.obj
 0003:00005e40       __exitflag                 0045ce40     LIBCMTD:crt0dat.obj
 0003:00005e44       __C_Termination_Done       0045ce44     LIBCMTD:crt0dat.obj
 0003:00005e48       __C_Exit_Done              0045ce48     LIBCMTD:crt0dat.obj
 0003:00005e50       __aenvptr                  0045ce50     LIBCMTD:wincrt0.obj
 0003:00005e54       __wenvptr                  0045ce54     LIBCMTD:wincrt0.obj
 0003:00005e58       ___error_mode              0045ce58     LIBCMTD:wincrt0.obj
 0003:00005ec4       __newmode                  0045cec4     LIBCMTD:_newmode.obj
 0003:00005ec8       ?_pnhHeap@@3P6AHI@ZA       0045cec8     LIBCMTD:handler.obj
 0003:00005ef0       __cflush                   0045cef0     LIBCMTD:_file.obj
 0003:00005ef4       ___lc_handle               0045cef4     LIBCMTD:nlsdata2.obj
 0003:00005f0c       ___lc_codepage             0045cf0c     LIBCMTD:nlsdata2.obj
 0003:00005f10       ___lc_collate_cp           0045cf10     LIBCMTD:nlsdata2.obj
 0003:00006028       __adbgmsg                  0045d028     LIBCMTD:crt0msg.obj
 0003:00006030       __stdbuf                   0045d030     LIBCMTD:_sftbuf.obj
 0003:00006038       ___lc_time_intl            0045d038     LIBCMTD:inittime.obj
 0003:00006054       ___lc_id                   0045d054     LIBCMTD:nlsdata3.obj
 0003:000060ac       ___lconv_static_null       0045d0ac     LIBCMTD:lconv.obj
 0003:00006180       ___alternate_form          0045d180     <common>
 0003:00006190       ___no_lead_zeros           0045d190     <common>
 0003:00006194       ___mbcodepage              0045d194     <common>
 0003:00006210       ___mbulinfo                0045d210     <common>
 0003:0000621c       ___ismbcodepage            0045d21c     <common>
 0003:00006220       __mbcasemap                0045d220     <common>
 0003:00006320       __mbctype                  0045d320     <common>
 0003:00006424       ___mblcid                  0045d424     <common>
 0003:00006440       ___pioinfo                 0045d440     <common>
 0003:0000657c       __nhandle                  0045d57c     <common>
 0003:00006580       ___setlc_active            0045d580     <common>
 0003:00006590       ___unguarded_readlc_active 0045d590     <common>
 0003:00006594       ___piob                    0045d594     <common>
 0003:000068e0       __bufin                    0045d8e0     <common>
 0003:000078e0       __nstream                  0045e8e0     <common>
 0003:000078e4       __crtheap                  0045e8e4     <common>
 0003:000078f4       ___active_heap             0045e8f4     <common>
 0003:000078f8       ___sbh_sizeHeaderList      0045e8f8     <common>
 0003:0000790c       ___sbh_indGroupDefer       0045e90c     <common>
 0003:00007910       ___sbh_pHeaderScan         0045e910     <common>
 0003:00007914       ___sbh_initialized         0045e914     <common>
 0003:00007918       ___sbh_pHeaderDefer        0045e918     <common>
 0003:0000791c       ___sbh_cntHeaderList       0045e91c     <common>
 0003:00007920       ___sbh_pHeaderList         0045e920     <common>
 0003:00007924       ___sbh_threshold           0045e924     <common>
 0003:00007928       __FPmtinit                 0045e928     <common>
 0003:00007938       __FPmtterm                 0045e938     <common>
 0003:0000793c       __acmdln                   0045e93c     <common>
 0003:00007948       ___env_initialized         0045e948     <common>
 0003:00007958       ___mbctype_initialized     0045e958     <common>
 0003:0000795c       ___onexitend               0045e95c     <common>
 0003:00007960       ___onexitbegin             0045e960     <common>
 0003:00007964       __FPinit                   0045e964     <common>
 0003:00007968       __pfnReportHook            0045e968     <common>
 0003:00007974       __pfnDumpClient            0045e974     <common>
 0004:00000000       __IMPORT_DESCRIPTOR_WINMM  0045f000     winmm:WINMM.dll
 0004:00000014       __IMPORT_DESCRIPTOR_KERNEL32 0045f014     kernel32:KERNEL32.dll
 0004:00000028       __IMPORT_DESCRIPTOR_USER32 0045f028     user32:USER32.dll
 0004:0000003c       __IMPORT_DESCRIPTOR_GDI32  0045f03c     gdi32:GDI32.dll
 0004:00000050       __IMPORT_DESCRIPTOR_comdlg32 0045f050     comdlg32:comdlg32.dll
 0004:00000064       __IMPORT_DESCRIPTOR_ADVAPI32 0045f064     advapi32:ADVAPI32.dll
 0004:00000078       __IMPORT_DESCRIPTOR_SHELL32 0045f078     shell32:SHELL32.dll
 0004:0000008c       __IMPORT_DESCRIPTOR_WSOCK32 0045f08c     wsock32:WSOCK32.dll
 0004:000000a0       __NULL_IMPORT_DESCRIPTOR   0045f0a0     winmm:WINMM.dll
 0004:00000690       __imp__RegEnumValueA@32    0045f690     advapi32:ADVAPI32.dll
 0004:00000694       __imp__RegOpenKeyA@12      0045f694     advapi32:ADVAPI32.dll
 0004:00000698       __imp__RegSetValueA@20     0045f698     advapi32:ADVAPI32.dll
 0004:0000069c       __imp__RegQueryInfoKeyA@48 0045f69c     advapi32:ADVAPI32.dll
 0004:000006a0       __imp__RegCloseKey@4       0045f6a0     advapi32:ADVAPI32.dll
 0004:000006a4       __imp__RegDeleteValueA@8   0045f6a4     advapi32:ADVAPI32.dll
 0004:000006a8       __imp__RegCreateKeyA@12    0045f6a8     advapi32:ADVAPI32.dll
 0004:000006ac       __imp__RegCreateKeyExA@36  0045f6ac     advapi32:ADVAPI32.dll
 0004:000006b0       __imp__RegQueryValueExA@24 0045f6b0     advapi32:ADVAPI32.dll
 0004:000006b4       __imp__RegSetValueExA@24   0045f6b4     advapi32:ADVAPI32.dll
 0004:000006b8       \177ADVAPI32_NULL_THUNK_DATA 0045f6b8     advapi32:ADVAPI32.dll
 0004:000006ec       __imp__GetDeviceCaps@8     0045f6ec     gdi32:GDI32.dll
 0004:000006f0       __imp__ExtTextOutA@32      0045f6f0     gdi32:GDI32.dll
 0004:000006f4       __imp__CreatePalette@4     0045f6f4     gdi32:GDI32.dll
 0004:000006f8       __imp__CreateCompatibleDC@4 0045f6f8     gdi32:GDI32.dll
 0004:000006fc       __imp__GetStockObject@4    0045f6fc     gdi32:GDI32.dll
 0004:00000700       __imp__SetTextColor@8      0045f700     gdi32:GDI32.dll
 0004:00000704       __imp__SetBkColor@8        0045f704     gdi32:GDI32.dll
 0004:00000708       __imp__CreateCompatibleBitmap@12 0045f708     gdi32:GDI32.dll
 0004:0000070c       __imp__SelectObject@8      0045f70c     gdi32:GDI32.dll
 0004:00000710       __imp__RealizePalette@4    0045f710     gdi32:GDI32.dll
 0004:00000714       __imp__SelectPalette@12    0045f714     gdi32:GDI32.dll
 0004:00000718       __imp__DeleteObject@4      0045f718     gdi32:GDI32.dll
 0004:0000071c       __imp__DeleteDC@4          0045f71c     gdi32:GDI32.dll
 0004:00000720       __imp__UpdateColors@4      0045f720     gdi32:GDI32.dll
 0004:00000724       __imp__BitBlt@36           0045f724     gdi32:GDI32.dll
 0004:00000728       __imp__StretchBlt@44       0045f728     gdi32:GDI32.dll
 0004:0000072c       __imp__SetBrushOrgEx@16    0045f72c     gdi32:GDI32.dll
 0004:00000730       __imp__SetStretchBltMode@8 0045f730     gdi32:GDI32.dll
 0004:00000734       __imp__SetPixelV@16        0045f734     gdi32:GDI32.dll
 0004:00000738       __imp__CreateFontIndirectA@4 0045f738     gdi32:GDI32.dll
 0004:0000073c       __imp__GdiFlush@0          0045f73c     gdi32:GDI32.dll
 0004:00000740       __imp__SetBkMode@8         0045f740     gdi32:GDI32.dll
 0004:00000744       __imp__Rectangle@20        0045f744     gdi32:GDI32.dll
 0004:00000748       __imp__GetClipBox@8        0045f748     gdi32:GDI32.dll
 0004:0000074c       \177GDI32_NULL_THUNK_DATA  0045f74c     gdi32:GDI32.dll
 0004:00000788       __imp__TlsAlloc@0          0045f788     kernel32:KERNEL32.dll
 0004:0000078c       __imp__DuplicateHandle@28  0045f78c     kernel32:KERNEL32.dll
 0004:00000790       __imp__GetCurrentThreadId@0 0045f790     kernel32:KERNEL32.dll
 0004:00000794       __imp__GetSystemTime@4     0045f794     kernel32:KERNEL32.dll
 0004:00000798       __imp__GetCurrentProcess@0 0045f798     kernel32:KERNEL32.dll
 0004:0000079c       __imp__GetCurrentThread@0  0045f79c     kernel32:KERNEL32.dll
 0004:000007a0       __imp__TlsSetValue@8       0045f7a0     kernel32:KERNEL32.dll
 0004:000007a4       __imp__SetThreadPriority@8 0045f7a4     kernel32:KERNEL32.dll
 0004:000007a8       __imp__CreateSemaphoreA@16 0045f7a8     kernel32:KERNEL32.dll
 0004:000007ac       __imp__ReleaseSemaphore@12 0045f7ac     kernel32:KERNEL32.dll
 0004:000007b0       __imp__WaitForSingleObject@8 0045f7b0     kernel32:KERNEL32.dll
 0004:000007b4       __imp__LeaveCriticalSection@4 0045f7b4     kernel32:KERNEL32.dll
 0004:000007b8       __imp__EnterCriticalSection@4 0045f7b8     kernel32:KERNEL32.dll
 0004:000007bc       __imp__DeleteCriticalSection@4 0045f7bc     kernel32:KERNEL32.dll
 0004:000007c0       __imp__InitializeCriticalSection@4 0045f7c0     kernel32:KERNEL32.dll
 0004:000007c4       __imp__GetModuleFileNameA@12 0045f7c4     kernel32:KERNEL32.dll
 0004:000007c8       __imp__OutputDebugStringA@4 0045f7c8     kernel32:KERNEL32.dll
 0004:000007cc       __imp__GetStdHandle@4      0045f7cc     kernel32:KERNEL32.dll
 0004:000007d0       __imp__WriteConsoleA@20    0045f7d0     kernel32:KERNEL32.dll
 0004:000007d4       __imp__WriteFile@20        0045f7d4     kernel32:KERNEL32.dll
 0004:000007d8       __imp__CloseHandle@4       0045f7d8     kernel32:KERNEL32.dll
 0004:000007dc       __imp__CreateFileA@28      0045f7dc     kernel32:KERNEL32.dll
 0004:000007e0       __imp__SetFilePointer@16   0045f7e0     kernel32:KERNEL32.dll
 0004:000007e4       __imp__SetEndOfFile@4      0045f7e4     kernel32:KERNEL32.dll
 0004:000007e8       __imp__AllocConsole@0      0045f7e8     kernel32:KERNEL32.dll
 0004:000007ec       __imp__TlsGetValue@4       0045f7ec     kernel32:KERNEL32.dll
 0004:000007f0       __imp__ResumeThread@4      0045f7f0     kernel32:KERNEL32.dll
 0004:000007f4       __imp__GetPrivateProfileStringA@24 0045f7f4     kernel32:KERNEL32.dll
 0004:000007f8       __imp__FormatMessageA@28   0045f7f8     kernel32:KERNEL32.dll
 0004:000007fc       __imp__LocalFree@4         0045f7fc     kernel32:KERNEL32.dll
 0004:00000800       __imp__GetEnvironmentStrings@0 0045f800     kernel32:KERNEL32.dll
 0004:00000804       __imp__WideCharToMultiByte@32 0045f804     kernel32:KERNEL32.dll
 0004:00000808       __imp__FreeEnvironmentStringsW@4 0045f808     kernel32:KERNEL32.dll
 0004:0000080c       __imp__FreeEnvironmentStringsA@4 0045f80c     kernel32:KERNEL32.dll
 0004:00000810       __imp__UnhandledExceptionFilter@4 0045f810     kernel32:KERNEL32.dll
 0004:00000814       __imp__GetDriveTypeA@4     0045f814     kernel32:KERNEL32.dll
 0004:00000818       __imp__GetCurrentDirectoryA@8 0045f818     kernel32:KERNEL32.dll
 0004:0000081c       __imp__SetConsoleCtrlHandler@8 0045f81c     kernel32:KERNEL32.dll
 0004:00000820       __imp__HeapCreate@12       0045f820     kernel32:KERNEL32.dll
 0004:00000824       __imp__HeapDestroy@4       0045f824     kernel32:KERNEL32.dll
 0004:00000828       __imp__GetEnvironmentVariableA@12 0045f828     kernel32:KERNEL32.dll
 0004:0000082c       __imp__VirtualAlloc@16     0045f82c     kernel32:KERNEL32.dll
 0004:00000830       __imp__VirtualFree@12      0045f830     kernel32:KERNEL32.dll
 0004:00000834       __imp__HeapReAlloc@16      0045f834     kernel32:KERNEL32.dll
 0004:00000838       __imp__HeapAlloc@12        0045f838     kernel32:KERNEL32.dll
 0004:0000083c       __imp__SetUnhandledExceptionFilter@4 0045f83c     kernel32:KERNEL32.dll
 0004:00000840       __imp__HeapFree@12         0045f840     kernel32:KERNEL32.dll
 0004:00000844       __imp__SetLastError@4      0045f844     kernel32:KERNEL32.dll
 0004:00000848       __imp__TlsFree@4           0045f848     kernel32:KERNEL32.dll
 0004:0000084c       __imp__FatalAppExitA@8     0045f84c     kernel32:KERNEL32.dll
 0004:00000850       __imp__ExitThread@4        0045f850     kernel32:KERNEL32.dll
 0004:00000854       __imp__CreateThread@24     0045f854     kernel32:KERNEL32.dll
 0004:00000858       __imp__GetVersion@0        0045f858     kernel32:KERNEL32.dll
 0004:0000085c       __imp__GetCommandLineA@0   0045f85c     kernel32:KERNEL32.dll
 0004:00000860       __imp__GetStartupInfoA@4   0045f860     kernel32:KERNEL32.dll
 0004:00000864       __imp__GetModuleHandleA@4  0045f864     kernel32:KERNEL32.dll
 0004:00000868       __imp__TerminateProcess@8  0045f868     kernel32:KERNEL32.dll
 0004:0000086c       __imp__ExitProcess@4       0045f86c     kernel32:KERNEL32.dll
 0004:00000870       __imp__GetFullPathNameA@16 0045f870     kernel32:KERNEL32.dll
 0004:00000874       __imp__GetFileAttributesA@4 0045f874     kernel32:KERNEL32.dll
 0004:00000878       __imp__InterlockedIncrement@4 0045f878     kernel32:KERNEL32.dll
 0004:0000087c       __imp__LoadLibraryA@4      0045f87c     kernel32:KERNEL32.dll
 0004:00000880       __imp__GetProcAddress@8    0045f880     kernel32:KERNEL32.dll
 0004:00000884       __imp__InterlockedDecrement@4 0045f884     kernel32:KERNEL32.dll
 0004:00000888       __imp__DebugBreak@0        0045f888     kernel32:KERNEL32.dll
 0004:0000088c       __imp__HeapValidate@12     0045f88c     kernel32:KERNEL32.dll
 0004:00000890       __imp__IsBadReadPtr@8      0045f890     kernel32:KERNEL32.dll
 0004:00000894       __imp__IsBadWritePtr@8     0045f894     kernel32:KERNEL32.dll
 0004:00000898       __imp__RaiseException@16   0045f898     kernel32:KERNEL32.dll
 0004:0000089c       __imp__RtlUnwind@16        0045f89c     kernel32:KERNEL32.dll
 0004:000008a0       __imp__GetEnvironmentStringsW@0 0045f8a0     kernel32:KERNEL32.dll
 0004:000008a4       __imp__SetHandleCount@4    0045f8a4     kernel32:KERNEL32.dll
 0004:000008a8       __imp__GetFileType@4       0045f8a8     kernel32:KERNEL32.dll
 0004:000008ac       __imp__IsBadCodePtr@4      0045f8ac     kernel32:KERNEL32.dll
 0004:000008b0       __imp__MultiByteToWideChar@24 0045f8b0     kernel32:KERNEL32.dll
 0004:000008b4       __imp__GetStringTypeA@20   0045f8b4     kernel32:KERNEL32.dll
 0004:000008b8       __imp__GetStringTypeW@16   0045f8b8     kernel32:KERNEL32.dll
 0004:000008bc       __imp__FlushFileBuffers@4  0045f8bc     kernel32:KERNEL32.dll
 0004:000008c0       __imp__GetCPInfo@8         0045f8c0     kernel32:KERNEL32.dll
 0004:000008c4       __imp__IsValidLocale@8     0045f8c4     kernel32:KERNEL32.dll
 0004:000008c8       __imp__IsValidCodePage@4   0045f8c8     kernel32:KERNEL32.dll
 0004:000008cc       __imp__GetLocaleInfoA@16   0045f8cc     kernel32:KERNEL32.dll
 0004:000008d0       __imp__EnumSystemLocalesA@8 0045f8d0     kernel32:KERNEL32.dll
 0004:000008d4       __imp__GetUserDefaultLCID@0 0045f8d4     kernel32:KERNEL32.dll
 0004:000008d8       __imp__LCMapStringA@24     0045f8d8     kernel32:KERNEL32.dll
 0004:000008dc       __imp__LCMapStringW@24     0045f8dc     kernel32:KERNEL32.dll
 0004:000008e0       __imp__GetACP@0            0045f8e0     kernel32:KERNEL32.dll
 0004:000008e4       __imp__GetOEMCP@0          0045f8e4     kernel32:KERNEL32.dll
 0004:000008e8       __imp__SetEnvironmentVariableA@8 0045f8e8     kernel32:KERNEL32.dll
 0004:000008ec       __imp__ReadFile@20         0045f8ec     kernel32:KERNEL32.dll
 0004:000008f0       __imp__GlobalLock@4        0045f8f0     kernel32:KERNEL32.dll
 0004:000008f4       __imp__GetTimeZoneInformation@4 0045f8f4     kernel32:KERNEL32.dll
 0004:000008f8       __imp__GetLastError@0      0045f8f8     kernel32:KERNEL32.dll
 0004:000008fc       __imp__Sleep@4             0045f8fc     kernel32:KERNEL32.dll
 0004:00000900       __imp__GetVersionExA@4     0045f900     kernel32:KERNEL32.dll
 0004:00000904       __imp__Beep@8              0045f904     kernel32:KERNEL32.dll
 0004:00000908       __imp__GlobalUnlock@4      0045f908     kernel32:KERNEL32.dll
 0004:0000090c       __imp__SetStdHandle@8      0045f90c     kernel32:KERNEL32.dll
 0004:00000910       __imp__GlobalAlloc@8       0045f910     kernel32:KERNEL32.dll
 0004:00000914       __imp__WritePrivateProfileStringA@16 0045f914     kernel32:KERNEL32.dll
 0004:00000918       __imp__GetPrivateProfileIntA@16 0045f918     kernel32:KERNEL32.dll
 0004:0000091c       __imp__GetLocaleInfoW@16   0045f91c     kernel32:KERNEL32.dll
 0004:00000920       __imp__CompareStringA@24   0045f920     kernel32:KERNEL32.dll
 0004:00000924       __imp__CompareStringW@24   0045f924     kernel32:KERNEL32.dll
 0004:00000928       \177KERNEL32_NULL_THUNK_DATA 0045f928     kernel32:KERNEL32.dll
 0004:000009a4       __imp__Shell_NotifyIconA@8 0045f9a4     shell32:SHELL32.dll
 0004:000009a8       \177SHELL32_NULL_THUNK_DATA 0045f9a8     shell32:SHELL32.dll
 0004:000009d4       __imp__SetWindowLongA@12   0045f9d4     user32:USER32.dll
 0004:000009d8       __imp__SetRect@20          0045f9d8     user32:USER32.dll
 0004:000009dc       __imp__DrawMenuBar@4       0045f9dc     user32:USER32.dll
 0004:000009e0       __imp__GetWindowLongA@8    0045f9e0     user32:USER32.dll
 0004:000009e4       __imp__EndDialog@8         0045f9e4     user32:USER32.dll
 0004:000009e8       __imp__DialogBoxParamA@20  0045f9e8     user32:USER32.dll
 0004:000009ec       __imp__AppendMenuA@16      0045f9ec     user32:USER32.dll
 0004:000009f0       __imp__GetSystemMenu@8     0045f9f0     user32:USER32.dll
 0004:000009f4       __imp__ShowWindow@8        0045f9f4     user32:USER32.dll
 0004:000009f8       __imp__CreateWindowExA@48  0045f9f8     user32:USER32.dll
 0004:000009fc       __imp__SetClipboardViewer@4 0045f9fc     user32:USER32.dll
 0004:00000a00       __imp__LoadCursorA@8       0045fa00     user32:USER32.dll
 0004:00000a04       __imp__LoadIconA@8         0045fa04     user32:USER32.dll
 0004:00000a08       __imp__MessageBoxA@16      0045fa08     user32:USER32.dll
 0004:00000a0c       __imp__DrawTextA@20        0045fa0c     user32:USER32.dll
 0004:00000a10       __imp__ReleaseDC@8         0045fa10     user32:USER32.dll
 0004:00000a14       __imp__SetWindowTextA@8    0045fa14     user32:USER32.dll
 0004:00000a18       __imp__SetForegroundWindow@4 0045fa18     user32:USER32.dll
 0004:00000a1c       __imp__SetWindowPos@28     0045fa1c     user32:USER32.dll
 0004:00000a20       __imp__AdjustWindowRectEx@16 0045fa20     user32:USER32.dll
 0004:00000a24       __imp__RegisterClassA@4    0045fa24     user32:USER32.dll
 0004:00000a28       __imp__InvalidateRect@12   0045fa28     user32:USER32.dll
 0004:00000a2c       __imp__SystemParametersInfoA@16 0045fa2c     user32:USER32.dll
 0004:00000a30       __imp__LoadKeyboardLayoutA@8 0045fa30     user32:USER32.dll
 0004:00000a34       __imp__GetMessageA@16      0045fa34     user32:USER32.dll
 0004:00000a38       __imp__DispatchMessageA@4  0045fa38     user32:USER32.dll
 0004:00000a3c       __imp__EnableWindow@8      0045fa3c     user32:USER32.dll
 0004:00000a40       __imp__SetDlgItemInt@16    0045fa40     user32:USER32.dll
 0004:00000a44       __imp__GetDlgItemInt@16    0045fa44     user32:USER32.dll
 0004:00000a48       __imp__GetDlgItem@8        0045fa48     user32:USER32.dll
 0004:00000a4c       __imp__GetKeyboardState@4  0045fa4c     user32:USER32.dll
 0004:00000a50       __imp__ToAscii@20          0045fa50     user32:USER32.dll
 0004:00000a54       __imp__GetKeyState@4       0045fa54     user32:USER32.dll
 0004:00000a58       __imp__FindWindowA@8       0045fa58     user32:USER32.dll
 0004:00000a5c       __imp__OpenDesktopA@16     0045fa5c     user32:USER32.dll
 0004:00000a60       __imp__EnumDesktopWindows@12 0045fa60     user32:USER32.dll
 0004:00000a64       __imp__CloseDesktop@4      0045fa64     user32:USER32.dll
 0004:00000a68       __imp__DestroyMenu@4       0045fa68     user32:USER32.dll
 0004:00000a6c       __imp__GetSubMenu@8        0045fa6c     user32:USER32.dll
 0004:00000a70       __imp__GetMenuItemID@8     0045fa70     user32:USER32.dll
 0004:00000a74       __imp__SetMenuDefaultItem@12 0045fa74     user32:USER32.dll
 0004:00000a78       __imp__TrackPopupMenu@28   0045fa78     user32:USER32.dll
 0004:00000a7c       __imp__LoadStringA@16      0045fa7c     user32:USER32.dll
 0004:00000a80       __imp__RegisterClassExA@4  0045fa80     user32:USER32.dll
 0004:00000a84       __imp__LoadMenuA@8         0045fa84     user32:USER32.dll
 0004:00000a88       __imp__GetCursorPos@4      0045fa88     user32:USER32.dll
 0004:00000a8c       __imp__SetCursorPos@8      0045fa8c     user32:USER32.dll
 0004:00000a90       __imp__GetSystemMetrics@4  0045fa90     user32:USER32.dll
 0004:00000a94       __imp__CheckMenuItem@12    0045fa94     user32:USER32.dll
 0004:00000a98       __imp__EmptyClipboard@0    0045fa98     user32:USER32.dll
 0004:00000a9c       __imp__SetClipboardData@8  0045fa9c     user32:USER32.dll
 0004:00000aa0       __imp__GetClipboardOwner@0 0045faa0     user32:USER32.dll
 0004:00000aa4       __imp__OpenClipboard@4     0045faa4     user32:USER32.dll
 0004:00000aa8       __imp__GetClipboardData@4  0045faa8     user32:USER32.dll
 0004:00000aac       __imp__CloseClipboard@0    0045faac     user32:USER32.dll
 0004:00000ab0       __imp__IsIconic@4          0045fab0     user32:USER32.dll
 0004:00000ab4       __imp__GetKeyboardLayoutNameA@4 0045fab4     user32:USER32.dll
 0004:00000ab8       __imp__SetScrollInfo@16    0045fab8     user32:USER32.dll
 0004:00000abc       __imp__BeginPaint@8        0045fabc     user32:USER32.dll
 0004:00000ac0       __imp__EndPaint@8          0045fac0     user32:USER32.dll
 0004:00000ac4       __imp__GetKeyNameTextA@12  0045fac4     user32:USER32.dll
 0004:00000ac8       __imp__SetTimer@16         0045fac8     user32:USER32.dll
 0004:00000acc       __imp__PostMessageA@16     0045facc     user32:USER32.dll
 0004:00000ad0       __imp__KillTimer@8         0045fad0     user32:USER32.dll
 0004:00000ad4       __imp__GetFocus@0          0045fad4     user32:USER32.dll
 0004:00000ad8       __imp__GetForegroundWindow@0 0045fad8     user32:USER32.dll
 0004:00000adc       __imp__GetWindow@8         0045fadc     user32:USER32.dll
 0004:00000ae0       __imp__ChangeClipboardChain@8 0045fae0     user32:USER32.dll
 0004:00000ae4       __imp__GetWindowRect@8     0045fae4     user32:USER32.dll
 0004:00000ae8       __imp__ShowScrollBar@12    0045fae8     user32:USER32.dll
 0004:00000aec       __imp__SetCursor@4         0045faec     user32:USER32.dll
 0004:00000af0       __imp__PostQuitMessage@4   0045faf0     user32:USER32.dll
 0004:00000af4       __imp__SendMessageA@16     0045faf4     user32:USER32.dll
 0004:00000af8       __imp__DefWindowProcA@16   0045faf8     user32:USER32.dll
 0004:00000afc       __imp__GetClientRect@8     0045fafc     user32:USER32.dll
 0004:00000b00       __imp__ScrollWindowEx@32   0045fb00     user32:USER32.dll
 0004:00000b04       __imp__UpdateWindow@4      0045fb04     user32:USER32.dll
 0004:00000b08       __imp__DestroyWindow@4     0045fb08     user32:USER32.dll
 0004:00000b0c       __imp__GetDlgItemTextA@16  0045fb0c     user32:USER32.dll
 0004:00000b10       __imp__SetDlgItemTextA@12  0045fb10     user32:USER32.dll
 0004:00000b14       __imp__GetDC@4             0045fb14     user32:USER32.dll
 0004:00000b18       \177USER32_NULL_THUNK_DATA 0045fb18     user32:USER32.dll
 0004:00000b84       __imp__PlaySoundA@12       0045fb84     winmm:WINMM.dll
 0004:00000b88       \177WINMM_NULL_THUNK_DATA  0045fb88     winmm:WINMM.dll
 0004:00000bb4       __imp__shutdown@8          0045fbb4     wsock32:WSOCK32.dll
 0004:00000bb8       __imp__accept@12           0045fbb8     wsock32:WSOCK32.dll
 0004:00000bbc       __imp__ioctlsocket@12      0045fbbc     wsock32:WSOCK32.dll
 0004:00000bc0       __imp__bind@12             0045fbc0     wsock32:WSOCK32.dll
 0004:00000bc4       __imp__listen@8            0045fbc4     wsock32:WSOCK32.dll
 0004:00000bc8       __imp__WSAAsyncSelect@16   0045fbc8     wsock32:WSOCK32.dll
 0004:00000bcc       __imp__send@16             0045fbcc     wsock32:WSOCK32.dll
 0004:00000bd0       __imp__recv@16             0045fbd0     wsock32:WSOCK32.dll
 0004:00000bd4       __imp__WSAStartup@8        0045fbd4     wsock32:WSOCK32.dll
 0004:00000bd8       __imp__WSACleanup@0        0045fbd8     wsock32:WSOCK32.dll
 0004:00000bdc       __imp__setsockopt@20       0045fbdc     wsock32:WSOCK32.dll
 0004:00000be0       __imp__socket@12           0045fbe0     wsock32:WSOCK32.dll
 0004:00000be4       __imp__inet_addr@4         0045fbe4     wsock32:WSOCK32.dll
 0004:00000be8       __imp__gethostbyname@4     0045fbe8     wsock32:WSOCK32.dll
 0004:00000bec       __imp__htons@4             0045fbec     wsock32:WSOCK32.dll
 0004:00000bf0       __imp__connect@12          0045fbf0     wsock32:WSOCK32.dll
 0004:00000bf4       __imp__getpeername@12      0045fbf4     wsock32:WSOCK32.dll
 0004:00000bf8       __imp__WSAGetLastError@0   0045fbf8     wsock32:WSOCK32.dll
 0004:00000bfc       __imp__closesocket@4       0045fbfc     wsock32:WSOCK32.dll
 0004:00000c00       \177WSOCK32_NULL_THUNK_DATA 0045fc00     wsock32:WSOCK32.dll
 0004:00000c38       __imp__CommDlgExtendedError@0 0045fc38     comdlg32:comdlg32.dll
 0004:00000c3c       __imp__GetSaveFileNameA@4  0045fc3c     comdlg32:comdlg32.dll
 0004:00000c40       \177comdlg32_NULL_THUNK_DATA 0045fc40     comdlg32:comdlg32.dll

 entry point at        0001:00019dc0

